 HlfViewer

 Timestamp is 640bd5e7 (Sat Mar 11 01:14:15 2023)

 Preferred load address is 10000000

 Start         Length     Name                   Class
 0001:00000000 0000e7d0H .text$mn                CODE
 0001:0000e7d0 000000b0H .text$x                 CODE
 0001:0000e880 0000003dH .text$yd                CODE
 0002:00000000 00000134H .idata$5                DATA
 0002:00000134 00000004H .00cfg                  DATA
 0002:00000138 00000004H .CRT$XCA                DATA
 0002:0000013c 00000004H .CRT$XCZ                DATA
 0002:00000140 00000004H .CRT$XIA                DATA
 0002:00000144 0000000cH .CRT$XIC                DATA
 0002:00000150 00000004H .CRT$XIZ                DATA
 0002:00000154 00000004H .CRT$XPA                DATA
 0002:00000158 00000008H .CRT$XPX                DATA
 0002:00000160 00000004H .CRT$XPXA               DATA
 0002:00000164 00000004H .CRT$XPZ                DATA
 0002:00000168 00000004H .CRT$XTA                DATA
 0002:0000016c 00000004H .CRT$XTZ                DATA
 0002:00000170 00000000H .gfids$y                DATA
 0002:00000170 00004fd0H .rdata                  DATA
 0002:00005140 00000000H .rdata$CastGuardVftablesA DATA
 0002:00005140 00000000H .rdata$CastGuardVftablesC DATA
 0002:00005140 0000032cH .rdata$r                DATA
 0002:0000546c 00000020H .rdata$sxdata           DATA
 0002:0000548c 00000030H .rdata$voltmd           DATA
 0002:000054bc 00000314H .rdata$zzzdbg           DATA
 0002:000057d0 00000004H .rtc$IAA                DATA
 0002:000057d4 00000004H .rtc$IZZ                DATA
 0002:000057d8 00000004H .rtc$TAA                DATA
 0002:000057dc 00000004H .rtc$TZZ                DATA
 0002:000057e0 00000680H .xdata$x                DATA
 0002:00005e60 000000c8H .edata                  DATA
 0002:00005f28 00000028H .idata$2                DATA
 0002:00005f50 00000014H .idata$3                DATA
 0002:00005f64 00000134H .idata$4                DATA
 0002:00006098 00000570H .idata$6                DATA
 0003:00000000 00000860H .data                   DATA
 0003:00000860 000000c0H .data$r                 DATA
 0003:00000920 000000b0H .data$rs                DATA
 0003:000009d0 00001908H .bss                    DATA
 0004:00000000 00000060H .rsrc$01                DATA
 0004:00000060 00000348H .rsrc$02                DATA

  Address         Publics by Value              Rva+Base       Lib:Object

 0000:00000000       ___guard_eh_cont_table     00000000     <absolute>
 0000:00000000       ___guard_fids_count        00000000     <absolute>
 0000:00000000       __except_list              00000000     <absolute>
 0000:00000000       ___arm64x_native_entrypoint 00000000     <absolute>
 0000:00000000       ___x64_code_ranges_to_entry_points_count 00000000     <absolute>
 0000:00000000       ___guard_longjmp_table     00000000     <absolute>
 0000:00000000       ___arm64x_extra_rfe_table  00000000     <absolute>
 0000:00000000       ___arm64x_redirection_metadata 00000000     <absolute>
 0000:00000000       ___guard_eh_cont_count     00000000     <absolute>
 0000:00000000       ___guard_iat_table         00000000     <absolute>
 0000:00000000       ___hybrid_code_map_count   00000000     <absolute>
 0000:00000000       ___x64_code_ranges_to_entry_points 00000000     <absolute>
 0000:00000000       ___guard_iat_count         00000000     <absolute>
 0000:00000000       ___hybrid_code_map         00000000     <absolute>
 0000:00000000       ___guard_longjmp_count     00000000     <absolute>
 0000:00000000       ___arm64x_extra_rfe_table_size 00000000     <absolute>
 0000:00000000       ___guard_check_icall_a64n_fptr 00000000     <absolute>
 0000:00000000       ___arm64x_redirection_metadata_count 00000000     <absolute>
 0000:00000000       ___hybrid_auxiliary_iat    00000000     <absolute>
 0000:00000000       ___dynamic_value_reloc_table 00000000     <absolute>
 0000:00000000       ___enclave_config          00000000     <absolute>
 0000:00000000       ___AbsoluteZero            00000000     <absolute>
 0000:00000000       ___guard_fids_table        00000000     <absolute>
 0000:00000000       ___hybrid_auxiliary_iat_copy 00000000     <absolute>
 0000:00000008       ___safe_se_handler_count   00000008     <absolute>
 0000:00000100       ___guard_flags             00000100     <absolute>
 0000:00000000       ___ImageBase               10000000     <linker-defined>
 0001:00000000       ??1PluginSettings@@QAE@XZ  10001000 f i HlfViewer.obj
 0001:00000050       ?Get@PluginSettings@@QAEHIPB_WH@Z 10001050 f i HlfViewer.obj
 0001:000000b0       ??0exception@std@@QAE@ABV01@@Z 100010b0 f i HlfViewer.obj
 0001:000000e0       ?what@exception@std@@UBEPBDXZ 100010e0 f i HlfViewer.obj
 0001:000000f0       ??_Ebad_alloc@std@@UAEPAXI@Z 100010f0 f i * CIL library *:* CIL module *
 0001:000000f0       ??_Gexception@std@@UAEPAXI@Z 100010f0 f i HlfViewer.obj
 0001:000000f0       ??_Gbad_alloc@std@@UAEPAXI@Z 100010f0 f i HlfViewer.obj
 0001:000000f0       ??_Gbad_array_new_length@std@@UAEPAXI@Z 100010f0 f i HlfViewer.obj
 0001:000000f0       ??_Ebad_array_new_length@std@@UAEPAXI@Z 100010f0 f i * CIL library *:* CIL module *
 0001:000000f0       ??_Eexception@std@@UAEPAXI@Z 100010f0 f i * CIL library *:* CIL module *
 0001:00000120       ??1length_error@std@@UAE@XZ 10001120 f i libcpmt:xthrow.obj
 0001:00000120       ??1bad_array_new_length@std@@UAE@XZ 10001120 f i HlfViewer.obj
 0001:00000120       ??1bad_exception@std@@UAE@XZ 10001120 f i libvcruntime:frame.obj
 0001:00000120       ??1bad_alloc@std@@UAE@XZ   10001120 f i HlfViewer.obj
 0001:00000140       ??0bad_array_new_length@std@@QAE@XZ 10001140 f i HlfViewer.obj
 0001:00000160       ?_Throw_bad_array_new_length@std@@YAXXZ 10001160 f i HlfViewer.obj
 0001:00000160       ?__scrt_throw_std_bad_array_new_length@@YAXXZ 10001160 f i LIBCMT:throw_bad_alloc.obj
 0001:00000180       ??0bad_array_new_length@std@@QAE@ABV01@@Z 10001180 f i HlfViewer.obj
 0001:000001c0       ??0bad_alloc@std@@QAE@ABV01@@Z 100011c0 f i HlfViewer.obj
 0001:00000200       ?_Xlen_string@std@@YAXXZ   10001200 f i HlfViewer.obj
 0001:00000210       ?SaveValue@PluginCheckBoxBinding@@UAEXPBUFarDialogItem@@H@Z 10001210 f i HlfViewer.obj
 0001:00000260       ??_GPluginEditFieldBinding@@UAEPAXI@Z 10001260 f i HlfViewer.obj
 0001:00000260       ??_EPluginEditFieldBinding@@UAEPAXI@Z 10001260 f i * CIL library *:* CIL module *
 0001:00000260       ??_GPluginCheckBoxBinding@@UAEPAXI@Z 10001260 f i HlfViewer.obj
 0001:00000260       ??_EPluginCheckBoxBinding@@UAEPAXI@Z 10001260 f i * CIL library *:* CIL module *
 0001:00000280       ?SaveValue@PluginRadioButtonBinding@@UAEXPBUFarDialogItem@@H@Z 10001280 f i HlfViewer.obj
 0001:000002b0       ??_GPluginRadioButtonBinding@@UAEPAXI@Z 100012b0 f i HlfViewer.obj
 0001:000002b0       ??_EPluginRadioButtonBinding@@UAEPAXI@Z 100012b0 f i * CIL library *:* CIL module *
 0001:000002d0       ?SaveValue@PluginEditFieldBinding@@UAEXPBUFarDialogItem@@H@Z 100012d0 f i HlfViewer.obj
 0001:00000330       ??0PluginDialogBuilder@@QAE@ABUPluginStartupInfo@@ABU_GUID@@1HPB_WP6GHPAXHH3@Z3_K@Z 10001330 f i HlfViewer.obj
 0001:00000540       ?AddCheckbox@PluginDialogBuilder@@QAEPAUFarDialogItem@@HPAHH_N@Z 10001540 f i HlfViewer.obj
 0001:00000650       ?AddRadioButtons@PluginDialogBuilder@@QAEPAUFarDialogItem@@PAHHQBH_N@Z 10001650 f i HlfViewer.obj
 0001:00000890       ?AddEditField@PluginDialogBuilder@@QAEPAUFarDialogItem@@PA_WHHPB_W_N@Z 10001890 f i HlfViewer.obj
 0001:00000930       ?AddButtons@PluginDialogBuilder@@QAEXHPBHHH@Z 10001930 f i HlfViewer.obj
 0001:00000b50       ?ShowDialogEx@PluginDialogBuilder@@QAEHXZ 10001b50 f i HlfViewer.obj
 0001:00000db0       ?AddDialogItem@PluginDialogBuilder@@AAEPAUFarDialogItem@@W4FARDIALOGITEMTYPES@@PB_W@Z 10001db0 f i HlfViewer.obj
 0001:00000f10       _GetGlobalInfoW@4          10001f10 f   HlfViewer.obj
 0001:00000fa0       _SetStartupInfoW@4         10001fa0 f   HlfViewer.obj
 0001:00000fe0       _OpenW@4                   10001fe0 f   HlfViewer.obj
 0001:000015d0       _GetPluginInfoW@4          100025d0 f   HlfViewer.obj
 0001:00001650       _ProcessEditorInputW@4     10002650 f   HlfViewer.obj
 0001:00001730       ?GetEditorFileName@@YAPA_WXZ 10002730 f   HlfViewer.obj
 0001:00001780       ?ShowCurrentHelpTopic@@YA_NXZ 10002780 f   HlfViewer.obj
 0001:00001ad0       ?IsHlf@@YAHXZ              10002ad0 f   HlfViewer.obj
 0001:00001cf0       ?FindTopic@@YAPB_W_N0@Z    10002cf0 f   HlfViewer.obj
 0001:00001ea0       _ConfigureW@4              10002ea0 f   HlfViewer.obj
 0001:000023f0       ?GetPluginConfig@@YAXXZ    100033f0 f   HlfViewer.obj
 0001:000025d0       ?assign@?$basic_string@_WU?$char_traits@_W@std@@V?$allocator@_W@2@@std@@QAEAAV12@QB_WI@Z 100035d0 f i HlfViewer.obj
 0001:00002730       _EncodePointerWrapper@4    10003730 f   vc_crt_fix_impl.obj
 0001:000027f0       _DecodePointerWrapper@4    100037f0 f   vc_crt_fix_impl.obj
 0001:00002840       _GetModuleHandleExWWrapper@12 10003840 f   vc_crt_fix_impl.obj
 0001:00002b80       _InitializeSListHeadWrapper@4 10003b80 f   vc_crt_fix_impl.obj
 0001:00002bd0       _InterlockedFlushSListWrapper@4 10003bd0 f   vc_crt_fix_impl.obj
 0001:00002c20       _InterlockedPopEntrySListWrapper@4 10003c20 f   vc_crt_fix_impl.obj
 0001:00002c70       _InterlockedPushEntrySListWrapper@8 10003c70 f   vc_crt_fix_impl.obj
 0001:00002cc0       _InterlockedPushListSListExWrapper@16 10003cc0 f   vc_crt_fix_impl.obj
 0001:00002d10       _RtlFirstEntrySListWrapper@4 10003d10 f   vc_crt_fix_impl.obj
 0001:00002d60       _QueryDepthSListWrapper@4  10003d60 f   vc_crt_fix_impl.obj
 0001:00002db0       _GetNumaHighestNodeNumberWrapper@4 10003db0 f   vc_crt_fix_impl.obj
 0001:00002e20       _GetLogicalProcessorInformationWrapper@8 10003e20 f   vc_crt_fix_impl.obj
 0001:00002e80       _SetThreadStackGuaranteeWrapper@4 10003e80 f   vc_crt_fix_impl.obj
 0001:00002ee0       _InitializeCriticalSectionExWrapper@12 10003ee0 f   vc_crt_fix_impl.obj
 0001:00002f60       _CompareStringExWrapper@36 10003f60 f   vc_crt_fix_impl.obj
 0001:00002fe0       _LCMapStringExWrapper@36   10003fe0 f   vc_crt_fix_impl.obj
 0001:00003060       ??0bad_alloc@std@@QAE@XZ   10004060 f i libcpmt:xthrow.obj
 0001:00003078       ??0exception@std@@QAE@QBD@Z 10004078 f i libcpmt:xthrow.obj
 0001:000030ad       ??0length_error@std@@QAE@ABV01@@Z 100040ad f i libcpmt:xthrow.obj
 0001:000030c8       ??0length_error@std@@QAE@PBD@Z 100040c8 f i libcpmt:xthrow.obj
 0001:000030e7       ??0logic_error@std@@QAE@ABV01@@Z 100040e7 f i libcpmt:xthrow.obj
 0001:00003102       ??_Gbad_exception@std@@UAEPAXI@Z 10004102 f i libvcruntime:frame.obj
 0001:00003102       ??_Ebad_exception@std@@UAEPAXI@Z 10004102 f i libvcruntime:frame.obj
 0001:00003102       ??_Glogic_error@std@@UAEPAXI@Z 10004102 f i libcpmt:xthrow.obj
 0001:00003102       ??_Elength_error@std@@UAEPAXI@Z 10004102 f i libcpmt:xthrow.obj
 0001:00003102       ??_Glength_error@std@@UAEPAXI@Z 10004102 f i libcpmt:xthrow.obj
 0001:00003102       ??_Elogic_error@std@@UAEPAXI@Z 10004102 f i libcpmt:xthrow.obj
 0001:0000312f       ?_Xlength_error@std@@YAXPBD@Z 1000412f f   libcpmt:xthrow.obj
 0001:0000314f       @__security_check_cookie@4 1000414f f   LIBCMT:secchk.obj
 0001:0000315d       ??_V@YAXPAX@Z              1000415d f   LIBCMT:delete_array.obj
 0001:00003162       ___raise_securityfailure   10004162 f   LIBCMT:gs_report.obj
 0001:0000318a       ___report_gsfailure        1000418a f   LIBCMT:gs_report.obj
 0001:00003284       ??2@YAPAXI@Z               10004284 f   LIBCMT:new_scalar.obj
 0001:000032b4       ??3@YAXPAX@Z               100042b4 f   LIBCMT:delete_scalar.obj
 0001:000032b9       ??3@YAXPAXI@Z              100042b9 f   LIBCMT:delete_scalar_size.obj
 0001:000032c7       ??_U@YAPAXI@Z              100042c7 f   LIBCMT:new_array.obj
 0001:000032d0       ??_Gtype_info@@UAEPAXI@Z   100042d0 f i LIBCMT:std_type_info_static.obj
 0001:000032d0       ??_Etype_info@@UAEPAXI@Z   100042d0 f i LIBCMT:std_type_info_static.obj
 0001:00003337       ___scrt_acquire_startup_lock 10004337 f   LIBCMT:utility.obj
 0001:00003369       ___scrt_dllmain_after_initialize_c 10004369 f   LIBCMT:utility.obj
 0001:00003394       ___scrt_dllmain_before_initialize_c 10004394 f   LIBCMT:utility.obj
 0001:000033a2       ___scrt_dllmain_crt_thread_attach 100043a2 f   LIBCMT:utility.obj
 0001:000033c1       ___scrt_dllmain_crt_thread_detach 100043c1 f   LIBCMT:utility.obj
 0001:000033ce       ___scrt_dllmain_exception_filter 100043ce f   LIBCMT:utility.obj
 0001:00003402       ___scrt_dllmain_uninitialize_c 10004402 f   LIBCMT:utility.obj
 0001:00003425       ___scrt_dllmain_uninitialize_critical 10004425 f   LIBCMT:utility.obj
 0001:00003432       ___scrt_initialize_crt     10004432 f   LIBCMT:utility.obj
 0001:0000346b       ___scrt_initialize_onexit_tables 1000446b f   LIBCMT:utility.obj
 0001:000034f2       ___scrt_is_nonwritable_in_current_image 100044f2 f   LIBCMT:utility.obj
 0001:00003586       ___scrt_release_startup_lock 10004586 f   LIBCMT:utility.obj
 0001:000035a3       ___scrt_uninitialize_crt   100045a3 f   LIBCMT:utility.obj
 0001:000035cb       __onexit                   100045cb f   LIBCMT:utility.obj
 0001:000035f8       _atexit                    100045f8 f   LIBCMT:utility.obj
 0001:0000394d       __DllMainCRTStartup@12     1000494d f   LIBCMT:dll_dllmain.obj
 0001:00003970       ?__scrt_throw_std_bad_alloc@@YAXXZ 10004970 f   LIBCMT:throw_bad_alloc.obj
 0001:0000398d       ___isa_available_init      1000498d f   LIBCMT:cpu_disp.obj
 0001:00003b5e       __get_startup_argv_mode    10004b5e f   LIBCMT:argv_mode.obj
 0001:00003b62       ___scrt_is_ucrt_dll_in_use 10004b62 f   LIBCMT:ucrt_detection.obj
 0001:00003b6e       ___scrt_fastfail           10004b6e f   LIBCMT:utility_desktop.obj
 0001:00003c89       __crt_debugger_hook        10004c89 f   LIBCMT:utility_desktop.obj
 0001:00003ca0       __SEH_prolog4              10004ca0 f   LIBCMT:sehprolg4.obj
 0001:00003ce5       @_guard_check_icall_nop@4  10004ce5 f i LIBCMT:guard_support.obj
 0001:00003d35       ___security_init_cookie    10004d35 f   LIBCMT:gs_support.obj
 0001:00003d80       _DllMain@12                10004d80 f   LIBCMT:dll_dllmain_stub.obj
 0001:00003d86       ?__scrt_initialize_type_info@@YAXXZ 10004d86 f   LIBCMT:tncleanup.obj
 0001:00003d92       ?__scrt_uninitialize_type_info@@YAXXZ 10004d92 f   LIBCMT:tncleanup.obj
 0001:00003d9e       ___local_stdio_printf_options 10004d9e f i LIBCMT:default_local_stdio_options.obj
 0001:00003da4       ___local_stdio_scanf_options 10004da4 f i LIBCMT:default_local_stdio_options.obj
 0001:00003daa       ___scrt_initialize_default_local_stdio_options 10004daa f   LIBCMT:default_local_stdio_options.obj
 0001:00003dc7       ___scrt_get_dyn_tls_init_callback 10004dc7 f   LIBCMT:dyn_tls_init.obj
 0001:00003dcd       __RTC_Initialize           10004dcd f   LIBCMT:initsect.obj
 0001:00003df9       __RTC_Terminate            10004df9 f   LIBCMT:initsect.obj
 0001:00003e25       ?GetRangeOfTrysToCheck@__FrameHandler3@@SA?AU?$pair@Viterator@TryBlockMap@__FrameHandler3@@V123@@std@@AAVTryBlockMap@1@HPAXPBU_s_FuncInfo@@H@Z 10004e25 f   libvcruntime:trnsctrl.obj
 0001:00003e95       ?_CallCatchBlock2@@YAPAXPAUEHRegistrationNode@@PBU_s_FuncInfo@@PAXHK@Z 10004e95 f   libvcruntime:trnsctrl.obj
 0001:00003ef2       ?_CallSETranslator@@YAHPAUEHExceptionRecord@@PAUEHRegistrationNode@@PAX2PBU_s_FuncInfo@@H1@Z 10004ef2 f   libvcruntime:trnsctrl.obj
 0001:00003fe8       ?_JumpToContinuation@@YGXPAXPAUEHRegistrationNode@@@Z 10004fe8 f   libvcruntime:trnsctrl.obj
 0001:00004018       ?_UnwindNestedFrames@@YGXPAUEHRegistrationNode@@PAUEHExceptionRecord@@@Z 10005018 f   libvcruntime:trnsctrl.obj
 0001:0000406b       __CatchGuardHandler        1000506b f   libvcruntime:trnsctrl.obj
 0001:0000409c       __CreateFrameInfo          1000509c f   libvcruntime:trnsctrl.obj
 0001:000040c0       __FindAndUnlinkFrame       100050c0 f   libvcruntime:trnsctrl.obj
 0001:00004108       __TranslatorGuardHandler   10005108 f   libvcruntime:trnsctrl.obj
 0001:000041a5       ___CxxFrameHandler3        100051a5 f   libvcruntime:trnsctrl.obj
 0001:000041db       ___std_exception_copy      100051db f   libvcruntime:std_exception.obj
 0001:0000423e       ___std_exception_destroy   1000523e f   libvcruntime:std_exception.obj
 0001:0000425d       _wcschr                    1000525d f   libvcruntime:wcschr.obj
 0001:00004324       ___DestructExceptionObject 10005324 f   libvcruntime:ehhelpers.obj
 0001:000043c5       ?_CallMemberFunction0@@YGXQAX0@Z 100053c5 f i libvcruntime:ehhelpers.obj
 0001:0000442a       __IsExceptionObjectToBeDestroyed 1000542a f   libvcruntime:ehhelpers.obj
 0001:00004450       ___AdjustPointer           10005450 f   libvcruntime:ehhelpers.obj
 0001:00004475       ___FrameUnwindFilter       10005475 f   libvcruntime:ehhelpers.obj
 0001:000044cb       ___std_terminate           100054cb f   libvcruntime:ehhelpers.obj
 0001:000044d0       __CxxThrowException@8      100054d0 f   libvcruntime:throw.obj
 0001:0000453c       ___vcrt_initialize         1000553c f   libvcruntime:initialization.obj
 0001:0000455b       ___vcrt_thread_attach      1000555b f   libvcruntime:initialization.obj
 0001:00004566       ___vcrt_thread_detach      10005566 f   libvcruntime:initialization.obj
 0001:00004571       ___vcrt_uninitialize       10005571 f   libvcruntime:initialization.obj
 0001:00004588       ___vcrt_uninitialize_critical 10005588 f   libvcruntime:initialization.obj
 0001:000045d0       __except_handler4          100055d0 f   libvcruntime:chandler4.obj
 0001:00004730       _memset                    10005730 f   libvcruntime:memset.obj
 0001:0000488a       ___std_type_info_compare   1000588a f   libvcruntime:std_type_info.obj
 0001:000048c6       ___std_type_info_destroy_list 100058c6 f   libvcruntime:std_type_info.obj
 0001:000048e9       ___vcrt_freefls@4          100058e9 f   libvcruntime:per_thread_data.obj
 0001:00004905       ___vcrt_freeptd            10005905 f   libvcruntime:per_thread_data.obj
 0001:0000493b       ___vcrt_getptd             1000593b f   libvcruntime:per_thread_data.obj
 0001:00004949       ___vcrt_getptd_noexit      10005949 f   libvcruntime:per_thread_data.obj
 0001:000049db       ___vcrt_initialize_ptd     100059db f   libvcruntime:per_thread_data.obj
 0001:00004a0e       ___vcrt_uninitialize_ptd   10005a0e f   libvcruntime:per_thread_data.obj
 0001:00005160       ??$TypeMatchHelper@V__FrameHandler3@@@@YAHPBU_s_HandlerType@@PBU_s_CatchableType@@PBU_s_ThrowInfo@@@Z 10006160 f i libvcruntime:frame.obj
 0001:000051ee       ??$__InternalCxxFrameHandler@V__FrameHandler3@@@@YA?AW4_EXCEPTION_DISPOSITION@@PAUEHExceptionRecord@@PAUEHRegistrationNode@@PAU_CONTEXT@@PAXPBU_s_FuncInfo@@H1E@Z 100061ee f i libvcruntime:frame.obj
 0001:000052f0       ??0bad_exception@std@@QAE@ABV01@@Z 100062f0 f i libvcruntime:frame.obj
 0001:0000530b       ??0bad_exception@std@@QAE@XZ 1000630b f i libvcruntime:frame.obj
 0001:00005323       ??8type_info@@QBE_NABV0@@Z 10006323 f i libvcruntime:frame.obj
 0001:0000558f       ?FrameUnwindToEmptyState@__FrameHandler3@@SAXPAUEHRegistrationNode@@PAXPBU_s_FuncInfo@@@Z 1000658f f   libvcruntime:frame.obj
 0001:000055a7       ?FrameUnwindToState@__FrameHandler3@@SAXPAUEHRegistrationNode@@PAXPBU_s_FuncInfo@@H@Z 100065a7 f   libvcruntime:frame.obj
 0001:00005729       ?_CallMemberFunction1@@YGXQAX00@Z 10006729 f i libvcruntime:frame.obj
 0001:00005739       ?_CallMemberFunction2@@YGXQAX00H@Z 10006739 f i libvcruntime:frame.obj
 0001:0000574c       ?getESTypes@__FrameHandler3@@SAPBU_s_ESTypeList@@PBU_s_FuncInfo@@@Z 1000674c f i libvcruntime:frame.obj
 0001:00005760       __CallSettingFrame@12      10006760 f   libvcruntime:lowhelpr.obj
 0001:00005787       __NLG_Return               10006787     libvcruntime:lowhelpr.obj
 0001:000057ac       ___except_validate_context_record 100067ac f   libvcruntime:jbcxrval.obj
 0001:000057dc       ___vcrt_initialize_locks   100067dc f   libvcruntime:locks.obj
 0001:00005818       ___vcrt_uninitialize_locks 10006818 f   libvcruntime:locks.obj
 0001:00005850       __local_unwind4            10006850 f   libvcruntime:exsup4.obj
 0001:00005940       @_EH4_CallFilterFunc@8     10006940 f   libvcruntime:exsup4.obj
 0001:00005960       @_EH4_TransferToHandler@8  10006960 f   libvcruntime:exsup4.obj
 0001:00005980       @_EH4_GlobalUnwind2@8      10006980 f   libvcruntime:exsup4.obj
 0001:000059a0       @_EH4_LocalUnwind@16       100069a0 f   libvcruntime:exsup4.obj
 0001:00005a9a       ___vcrt_FlsAlloc           10006a9a f   libvcruntime:winapi_downlevel.obj
 0001:00005ad5       ___vcrt_FlsFree            10006ad5 f   libvcruntime:winapi_downlevel.obj
 0001:00005b10       ___vcrt_FlsGetValue        10006b10 f   libvcruntime:winapi_downlevel.obj
 0001:00005b4b       ___vcrt_FlsSetValue        10006b4b f   libvcruntime:winapi_downlevel.obj
 0001:00005b89       ___vcrt_InitializeCriticalSectionEx 10006b89 f   libvcruntime:winapi_downlevel.obj
 0001:00005bd0       _unexpected                10006bd0 f   libvcruntime:unexpected.obj
 0001:00005bed       ?GetCurrentState@__FrameHandler3@@SAHPAUEHRegistrationNode@@PAXPBU_s_FuncInfo@@@Z 10006bed f   libvcruntime:ehstate.obj
 0001:00005c0a       ?SetState@__FrameHandler3@@SAXPAUEHRegistrationNode@@PBU_s_FuncInfo@@H@Z 10006c0a f   libvcruntime:ehstate.obj
 0001:00005c20       _memcpy                    10006c20 f   libvcruntime:memcpy.obj
 0001:00005c20       _memmove                   10006c20 f   libvcruntime:memmove.obj
 0001:000061a0       __NLG_Notify1              100071a0 f   libvcruntime:exsup.obj
 0001:000061b0       __NLG_Notify               100071b0 f   libvcruntime:exsup.obj
 0001:000061c7       __NLG_Dispatch2            100071c7     libvcruntime:exsup.obj
 0001:000061c7       __NLG_Dispatch             100071c7     libvcruntime:exsup.obj
 0001:000061d0       __NLG_Call                 100071d0 f   libvcruntime:exsup.obj
 0001:000061d2       __NLG_Return2              100071d2     libvcruntime:exsup.obj
 0001:000061e0       ___acrt_call_reportfault   100071e0 f   libucrt:invalid_parameter.obj
 0001:00006319       ___acrt_initialize_invalid_parameter_handler 10007319 f   libucrt:invalid_parameter.obj
 0001:00006328       __invalid_parameter        10007328 f   libucrt:invalid_parameter.obj
 0001:0000638c       __invalid_parameter_noinfo 1000738c f   libucrt:invalid_parameter.obj
 0001:0000639c       __invalid_parameter_noinfo_noreturn 1000739c f   libucrt:invalid_parameter.obj
 0001:000063b9       __invoke_watson            100073b9 f   libucrt:invalid_parameter.obj
 0001:000063ed       _free                      100073ed f   libucrt:free.obj
 0001:00006408       _malloc                    10007408 f   libucrt:malloc.obj
 0001:00006413       ___acrt_initialize_new_handler 10007413 f   libucrt:new_handler.obj
 0001:00006422       __callnewh                 10007422 f   libucrt:new_handler.obj
 0001:0000644f       __query_new_handler        1000744f f   libucrt:new_handler.obj
 0001:000064ab       __seh_filter_dll           100074ab f   libucrt:exception_filter.obj
 0001:000064cb       __seh_filter_exe           100074cb f   libucrt:exception_filter.obj
 0001:00006899       ___acrt_initialize_thread_local_exit_callback 10007899 f   libucrt:exit.obj
 0001:000068a8       __cexit                    100078a8 f   libucrt:exit.obj
 0001:000068b7       __exit                     100078b7 f   libucrt:exit.obj
 0001:000068cd       __is_c_termination_complete 100078cd f   libucrt:exit.obj
 0001:00006b81       ___acrt_allocate_buffer_for_argv 10007b81 f   libucrt:argv_parsing.obj
 0001:00006bd0       __configure_narrow_argv    10007bd0 f   libucrt:argv_parsing.obj
 0001:00006d2d       ??$uninitialize@A6AXAAPAPA_W@Z@?$dual_state_global@PAPA_W@__crt_state_management@@QAEXA6AXAAPAPA_W@Z@Z 10007d2d f i libucrt:environment_initialization.obj
 0001:00006d2d       ??$uninitialize@A6AXAAPAPAD@Z@?$dual_state_global@PAPAD@__crt_state_management@@QAEXA6AXAAPAPAD@Z@Z 10007d2d f i libucrt:environment_initialization.obj
 0001:00006d8c       ___dcrt_uninitialize_environments_nolock 10007d8c f   libucrt:environment_initialization.obj
 0001:00006dc3       __initialize_narrow_environment 10007dc3 f   libucrt:environment_initialization.obj
 0001:00006e7e       ??$__crt_fast_encode_pointer@P6AHXZ@@YAP6AHXZQ6AHXZ@Z 10007e7e f i libucrt:onexit.obj
 0001:00006e7e       ??$__crt_fast_encode_pointer@PAX@@YAPAXQAX@Z 10007e7e f i libucrt:initialization.obj
 0001:00006e7e       ??$__crt_fast_encode_pointer@PAP6AXXZ@@YAPAP6AXXZQAP6AXXZ@Z 10007e7e f i libucrt:onexit.obj
 0001:000070a0       __crt_atexit               100080a0 f   libucrt:onexit.obj
 0001:000070b6       __execute_onexit_table     100080b6 f   libucrt:onexit.obj
 0001:000070e3       __initialize_onexit_table  100080e3 f   libucrt:onexit.obj
 0001:0000710c       __register_onexit_function 1000810c f   libucrt:onexit.obj
 0001:0000713f       ___acrt_uninitialize_command_line 1000813f f   libucrt:argv_data.obj
 0001:0000723d       ___acrt_initialize         1000823d f   libucrt:initialization.obj
 0001:0000724f       ___acrt_thread_attach      1000824f f   libucrt:initialization.obj
 0001:0000725a       ___acrt_thread_detach      1000825a f   libucrt:initialization.obj
 0001:00007262       ___acrt_uninitialize       10008262 f   libucrt:initialization.obj
 0001:00007292       ___acrt_uninitialize_critical 10008292 f   libucrt:initialization.obj
 0001:000072a4       __initterm                 100082a4 f   libucrt:initterm.obj
 0001:000072e9       __initterm_e               100082e9 f   libucrt:initterm.obj
 0001:00007317       _terminate                 10008317 f   libucrt:terminate.obj
 0001:00007353       _abort                     10008353 f   libucrt:abort.obj
 0001:00007397       _strcpy_s                  10008397 f   libucrt:strcpy_s.obj
 0001:000073f1       _calloc                    100083f1 f   libucrt:calloc.obj
 0001:000073fc       ??0_LocaleUpdate@@QAE@QAU__crt_locale_pointers@@@Z 100083fc f i libucrt:output.obj
 0001:0000747f       ___acrt_locale_get_ctype_array_value 1000847f f i libucrt:output.obj
 0001:000074b0       _strncmp                   100084b0 f   libucrt:strncmp.obj
 0001:00007528       _wcsncmp                   10008528 f   libucrt:wcsncmp.obj
 0001:000078a0       ___acrt_freeptd            100088a0 f   libucrt:per_thread_data.obj
 0001:000078cc       ___acrt_getptd             100088cc f   libucrt:per_thread_data.obj
 0001:00007989       ___acrt_getptd_head        10008989 f   libucrt:per_thread_data.obj
 0001:00007a23       ___acrt_getptd_noexit      10008a23 f   libucrt:per_thread_data.obj
 0001:00007ad8       ___acrt_initialize_ptd     10008ad8 f   libucrt:per_thread_data.obj
 0001:00007b04       ___acrt_uninitialize_ptd   10008b04 f   libucrt:per_thread_data.obj
 0001:00007b1e       __free_base                10008b1e f   libucrt:free_base.obj
 0001:00007b58       __malloc_base              10008b58 f   libucrt:malloc_base.obj
 0001:00007ba6       ___acrt_initialize_locks   10008ba6 f   libucrt:locks.obj
 0001:00007be7       ___acrt_lock               10008be7 f   libucrt:locks.obj
 0001:00007bfe       ___acrt_uninitialize_locks 10008bfe f   libucrt:locks.obj
 0001:00007c2f       ___acrt_unlock             10008c2f f   libucrt:locks.obj
 0001:00007c46       ___acrt_get_process_end_policy 10008c46 f   libucrt:win_policies.obj
 0001:00007c77       ___acrt_errno_from_os_error 10008c77 f   libucrt:errno.obj
 0001:00007cba       ___acrt_errno_map_os_error 10008cba f   libucrt:errno.obj
 0001:00007cdd       ___doserrno                10008cdd f   libucrt:errno.obj
 0001:00007cf0       __errno                    10008cf0 f   libucrt:errno.obj
 0001:00007d03       __calloc_base              10008d03 f   libucrt:calloc_base.obj
 0001:00007ef9       ??$__acrt_mbs_to_wcs_cp@U__crt_win32_buffer_internal_dynamic_resizing@@@@YAHQBDAAV?$__crt_win32_buffer@_WU__crt_win32_buffer_internal_dynamic_resizing@@@@I@Z 10008ef9 f i libucrt:argv_wildcards.obj
 0001:0000840d       ?__acrt_get_utf8_acp_compatibility_codepage@@YAIXZ 1000940d f i libucrt:argv_wildcards.obj
 0001:0000844c       ?_deallocate@?$__crt_win32_buffer@DU__crt_win32_buffer_internal_dynamic_resizing@@@@AAEXXZ 1000944c f i libucrt:argv_wildcards.obj
 0001:0000844c       ?_deallocate@?$__crt_win32_buffer@_WU__crt_win32_buffer_internal_dynamic_resizing@@@@AAEXXZ 1000944c f i libucrt:argv_wildcards.obj
 0001:00008466       ?allocate@?$__crt_win32_buffer@DU__crt_win32_buffer_internal_dynamic_resizing@@@@QAEHI@Z 10009466 f i libucrt:argv_wildcards.obj
 0001:000084a2       ?allocate@?$__crt_win32_buffer@_WU__crt_win32_buffer_internal_dynamic_resizing@@@@QAEHI@Z 100094a2 f i libucrt:argv_wildcards.obj
 0001:000084e1       ?allocate@__crt_win32_buffer_internal_dynamic_resizing@@SAHQAPAXIABV__crt_win32_buffer_empty_debug_info@@@Z 100094e1 f i libucrt:argv_wildcards.obj
 0001:00008587       ___acrt_expand_narrow_argv_wildcards 10009587 f   libucrt:argv_wildcards.obj
 0001:00008659       ?allocate@?$__crt_win32_buffer@DU__crt_win32_buffer_no_resizing@@@@QAEHI@Z 10009659 f i libucrt:getmodulefilenamea.obj
 0001:00008680       ?set_to_nullptr@?$__crt_win32_buffer@DU__crt_win32_buffer_no_resizing@@@@QAEXXZ 10009680 f i libucrt:getmodulefilenamea.obj
 0001:00008694       ___acrt_GetModuleFileNameA 10009694 f   libucrt:getmodulefilenamea.obj
 0001:00008c53       ___acrt_initialize_multibyte 10009c53 f   libucrt:mbctype.obj
 0001:00008c9b       ___acrt_update_thread_multibyte_data 10009c9b f   libucrt:mbctype.obj
 0001:00008cae       __setmbcp_nolock           10009cae f   libucrt:mbctype.obj
 0001:00008f79       __ismbblead                10009f79 f   libucrt:ismbbyte.obj
 0001:00008f91       ___acrt_initialize_command_line 10009f91 f   libucrt:argv_data.obj
 0001:00008faa       ___acrt_MultiByteToWideChar 10009faa f   libucrt:multibytetowidechar.obj
 0001:00009026       ___acrt_WideCharToMultiByte 1000a026 f   libucrt:widechartomultibyte.obj
 0001:0000910a       ___dcrt_get_narrow_environment_from_os 1000a10a f   libucrt:get_environment_from_os.obj
 0001:0000918e       __recalloc_base            1000a18e f   libucrt:recalloc.obj
 0001:00009393       ___acrt_AppPolicyGetProcessTerminationMethodInternal@4 1000a393 f   libucrt:winapi_thunks.obj
 0001:000093d3       ___acrt_AreFileApisANSI@0  1000a3d3 f   libucrt:winapi_thunks.obj
 0001:000093f2       ___acrt_FlsAlloc@4         1000a3f2 f   libucrt:winapi_thunks.obj
 0001:00009431       ___acrt_FlsFree@4          1000a431 f   libucrt:winapi_thunks.obj
 0001:00009470       ___acrt_FlsGetValue@4      1000a470 f   libucrt:winapi_thunks.obj
 0001:000094af       ___acrt_FlsSetValue@8      1000a4af f   libucrt:winapi_thunks.obj
 0001:000094f1       ___acrt_InitializeCriticalSectionEx@12 1000a4f1 f   libucrt:winapi_thunks.obj
 0001:0000953c       ___acrt_LCMapStringEx@36   1000a53c f   libucrt:winapi_thunks.obj
 0001:00009599       ___acrt_LocaleNameToLCID@8 1000a599 f   libucrt:winapi_thunks.obj
 0001:000095ca       ___acrt_initialize_winapi_thunks 1000a5ca f   libucrt:winapi_thunks.obj
 0001:000095f5       ___acrt_uninitialize_winapi_thunks 1000a5f5 f   libucrt:winapi_thunks.obj
 0001:0000962b       ___acrt_initialize_heap    1000a62b f   libucrt:heap_handle.obj
 0001:0000963c       ___acrt_uninitialize_heap  1000a63c f   libucrt:heap_handle.obj
 0001:000097b0       ___acrt_initialize_lowio   1000a7b0 f   libucrt:ioinit.obj
 0001:00009810       ___acrt_uninitialize_lowio 1000a810 f   libucrt:ioinit.obj
 0001:0000983c       ___acrt_execute_initializers 1000a83c f   libucrt:shared_initialization.obj
 0001:000098a4       ___acrt_execute_uninitializers 1000a8a4 f   libucrt:shared_initialization.obj
 0001:000099a3       ___acrt_get_sigabrt_handler 1000a9a3 f   libucrt:signal.obj
 0001:000099ca       ___acrt_initialize_signal_handlers 1000a9ca f   libucrt:signal.obj
 0001:000099e8       ___fpecode                 1000a9e8 f   libucrt:signal.obj
 0001:000099f1       _raise                     1000a9f1 f   libucrt:signal.obj
 0001:00009bec       ___acrt_has_user_matherr   1000abec f   libucrt:matherr.obj
 0001:00009c04       ___acrt_initialize_user_matherr 1000ac04 f   libucrt:matherr.obj
 0001:00009c13       ___acrt_invoke_user_matherr 1000ac13 f   libucrt:matherr.obj
 0001:00009e22       ___acrt_stdio_flush_nolock 1000ae22 f   libucrt:fflush.obj
 0001:00009e87       __fflush_nolock            1000ae87 f   libucrt:fflush.obj
 0001:00009ecf       __flushall                 1000aecf f   libucrt:fflush.obj
 0001:00009ed8       ___acrt_initialize_stdio   1000aed8 f   libucrt:_file.obj
 0001:00009fa0       ___acrt_uninitialize_stdio 1000afa0 f   libucrt:_file.obj
 0001:00009fec       __lock_file                1000afec f   libucrt:_file.obj
 0001:0000a000       __unlock_file              1000b000 f   libucrt:_file.obj
 0001:0000a014       __mbtowc_l                 1000b014 f   libucrt:mbtowc.obj
 0001:0000a156       _mbtowc                    1000b156 f   libucrt:mbtowc.obj
 0001:0000a170       ___acrt_update_locale_info 1000b170 f   libucrt:locale_update.obj
 0001:0000a19d       ___acrt_update_multibyte_info 1000b19d f   libucrt:locale_update.obj
 0001:0000a1ca       __fileno                   1000b1ca f   libucrt:fileno.obj
 0001:0000a25f       ___acrt_set_locale_changed 1000b25f f   libucrt:wsetlocale.obj
 0001:0000a26a       ___acrt_uninitialize_locale 1000b26a f   libucrt:wsetlocale.obj
 0001:0000a291       ___pctype_func             1000b291 f   libucrt:ctype.obj
 0001:0000a2b5       ___acrt_add_locale_ref     1000b2b5 f   libucrt:locale_refcounting.obj
 0001:0000a332       ___acrt_free_locale        1000b332 f   libucrt:locale_refcounting.obj
 0001:0000a47a       ___acrt_locale_add_lc_time_reference 1000b47a f   libucrt:locale_refcounting.obj
 0001:0000a4a3       ___acrt_locale_free_lc_time_if_unreferenced 1000b4a3 f   libucrt:locale_refcounting.obj
 0001:0000a4d4       ___acrt_locale_release_lc_time_reference 1000b4d4 f   libucrt:locale_refcounting.obj
 0001:0000a4fd       ___acrt_release_locale_ref 1000b4fd f   libucrt:locale_refcounting.obj
 0001:0000a57e       ___acrt_update_thread_locale_data 1000b57e f   libucrt:locale_refcounting.obj
 0001:0000a5ff       __updatetlocinfoEx_nolock  1000b5ff f   libucrt:locale_refcounting.obj
 0001:0000a64f       __query_new_mode           1000b64f f   libucrt:new_mode.obj
 0001:0000a6a0       _qsort                     1000b6a0 f   libucrt:qsort.obj
 0001:0000ab97       _strncpy_s                 1000bb97 f   libucrt:strncpy_s.obj
 0001:0000abb0       _strpbrk                   1000bbb0 f   libucrt:strpbrk.obj
 0001:0000abf0       __mbsdec                   1000bbf0 f   libucrt:mbsdec.obj
 0001:0000ac07       __mbsdec_l                 1000bc07 f   libucrt:mbsdec.obj
 0001:0000ac94       ___acrt_GetStringTypeA     1000bc94 f   libucrt:getstringtypea.obj
 0001:0000ad97       __freea_crt                1000bd97 f i libucrt:getstringtypea.obj
 0001:0000afa1       ___acrt_LCMapStringA       1000bfa1 f   libucrt:lcmapstringa.obj
 0001:0000aff9       __msize_base               1000bff9 f   libucrt:msize.obj
 0001:0000b02c       __realloc_base             1000c02c f   libucrt:realloc_base.obj
 0001:0000b0e5       ___acrt_DownlevelLocaleNameToLCID 1000c0e5 f   libucrt:lcidtoname_downlevel.obj
 0001:0000b111       ___acrt_lowio_create_handle_array 1000c111 f   libucrt:osfinfo.obj
 0001:0000b18c       ___acrt_lowio_destroy_handle_array 1000c18c f   libucrt:osfinfo.obj
 0001:0000b1c1       ___acrt_lowio_ensure_fh_exists 1000c1c1 f   libucrt:osfinfo.obj
 0001:0000b25f       ___acrt_lowio_lock_fh      1000c25f f   libucrt:osfinfo.obj
 0001:0000b282       ___acrt_lowio_unlock_fh    1000c282 f   libucrt:osfinfo.obj
 0001:0000b2a5       __free_osfhnd              1000c2a5 f   libucrt:osfinfo.obj
 0001:0000b336       __get_osfhandle            1000c336 f   libucrt:osfinfo.obj
 0001:0000b442       __commit                   1000c442 f   libucrt:commit.obj
 0001:0000bc38       __write                    1000cc38 f   libucrt:write.obj
 0001:0000bd2a       __write_nolock             1000cd2a f   libucrt:write.obj
 0001:0000bf0c       __fcloseall                1000cf0c f   libucrt:closeall.obj
 0001:0000bfb7       ___acrt_stdio_free_buffer_nolock 1000cfb7 f   libucrt:_freebuf.obj
 0001:0000bff7       __isatty                   1000cff7 f   libucrt:isatty.obj
 0001:0000c04d       __isleadbyte_l             1000d04d f i libucrt:_wctype.obj
 0001:0000c0b3       ?__mbrtowc_utf8@__crt_mbstring@@YAIPA_WPBDIPAU_Mbstatet@@@Z 1000d0b3 f   libucrt:mbrtowc.obj
 0001:0000c0f3       ?__mbsrtowcs_utf8@__crt_mbstring@@YAIPA_WPAPBDIPAU_Mbstatet@@@Z 1000d0f3 f   libucrt:mbrtowc.obj
 0001:0000c1ee       ?return_illegal_sequence@__crt_mbstring@@YAIPAU_Mbstatet@@@Z 1000d1ee f i libucrt:c32rtomb.obj
 0001:0000c20d       ___acrt_locale_free_monetary 1000d20d f   libucrt:initmon.obj
 0001:0000c30b       ___acrt_locale_free_numeric 1000d30b f   libucrt:initnum.obj
 0001:0000c3ac       ___acrt_locale_free_time   1000d3ac f   libucrt:inittime.obj
 0001:0000c490       ___strncnt                 1000d490 f   libucrt:strncnt.obj
 0001:0000c4ac       ___ascii_wcsnicmp          1000d4ac f   libucrt:wcsnicmp.obj
 0001:0000c4fb       __query_app_type           1000d4fb f   libucrt:report_runtime_error.obj
 0001:0000c57d       __lseeki64_nolock          1000d57d f   libucrt:lseek.obj
 0001:0000c598       __putwch_nolock            1000d598 f   libucrt:putwch.obj
 0001:0000c5ca       __fclose_nolock            1000d5ca f   libucrt:fclose.obj
 0001:0000c641       _fclose                    1000d641 f   libucrt:fclose.obj
 0001:0000c6c5       ?__mbrtoc32_utf8@__crt_mbstring@@YAIPA_UPBDIPAU_Mbstatet@@@Z 1000d6c5 f   libucrt:mbrtoc32.obj
 0001:0000c870       __CIlog10                  1000d870 f   libucrt:log10_impl.obj
 0001:0000c8ab       __CIlog10_default          1000d8ab f   libucrt:log10_impl.obj
 0001:0000c8bf       __log10_default            1000d8bf     libucrt:log10_impl.obj
 0001:0000c980       _ceil                      1000d980 f   libucrt:ceil_pentium4.obj
 0001:0000c9c0       __ceil_pentium4            1000d9c0 f   libucrt:ceil_pentium4.obj
 0001:0000caa0       ___ascii_strnicmp          1000daa0 f   libucrt:_strnicm.obj
 0001:0000cb20       ___dcrt_lowio_ensure_console_output_initialized 1000db20 f   libucrt:initcon.obj
 0001:0000cb3f       ___dcrt_terminate_console_output 1000db3f f   libucrt:initcon.obj
 0001:0000cb56       ___dcrt_write_console      1000db56 f   libucrt:initcon.obj
 0001:0000cc37       __close                    1000dc37 f   libucrt:close.obj
 0001:0000ccc4       __close_nolock             1000dcc4 f   libucrt:close.obj
 0001:0000cd60       ?__acrt_stdio_free_stream@@YAXV__crt_stdio_stream@@@Z 1000dd60 f   libucrt:stream.obj
 0001:0000cd9b       ___acrt_initialize_sse2    1000dd9b f   libucrt:mathfcns.obj
 0001:0000cdb0       __CIlog10_pentium4         1000ddb0 f   libucrt:log10_pentium4.obj
 0001:0000cdc8       __log10_pentium4           1000ddc8     libucrt:log10_pentium4.obj
 0001:0000d060       __fFEXP                    1000e060 f   libucrt:87tran.obj
 0001:0000d0b7       __rtinfpopse               1000e0b7     libucrt:87tran.obj
 0001:0000d0b9       __rtinfnpopse              1000e0b9     libucrt:87tran.obj
 0001:0000d0c9       __fFLN                     1000e0c9     libucrt:87tran.obj
 0001:0000d17e       __rtinfpop                 1000e17e     libucrt:87tran.obj
 0001:0000d180       __rtinfnpop                1000e180     libucrt:87tran.obj
 0001:0000d190       __rtforexpinf              1000e190 f   libucrt:87tran.obj
 0001:0000d19d       __ffexpm1                  1000e19d     libucrt:87tran.obj
 0001:0000d250       __trandisp1                1000e250 f   libucrt:87disp.obj
 0001:0000d2c5       __trandisp2                1000e2c5 f   libucrt:87disp.obj
 0001:0000d35f       __rttospopde               1000e35f     libucrt:87disp.obj
 0001:0000d364       __rttospop                 1000e364     libucrt:87disp.obj
 0001:0000d370       __rtnospop                 1000e370 f   libucrt:87disp.obj
 0001:0000d380       __rttosnpop                1000e380 f   libucrt:87disp.obj
 0001:0000d381       __rtnospopde               1000e381     libucrt:87disp.obj
 0001:0000d388       __rtzeropop                1000e388     libucrt:87disp.obj
 0001:0000d38a       __rtzeronpop               1000e38a     libucrt:87disp.obj
 0001:0000d390       __rtzerospop               1000e390 f   libucrt:87disp.obj
 0001:0000d39d       __rtonepop                 1000e39d     libucrt:87disp.obj
 0001:0000d3a0       __rtonenpop                1000e3a0 f   libucrt:87disp.obj
 0001:0000d3b0       __tosnan1                  1000e3b0 f   libucrt:87disp.obj
 0001:0000d3e0       __nosnan2                  1000e3e0 f   libucrt:87disp.obj
 0001:0000d3f0       __tosnan2                  1000e3f0 f   libucrt:87disp.obj
 0001:0000d420       __nan2                     1000e420 f   libucrt:87disp.obj
 0001:0000d460       __rtindfpop                1000e460 f   libucrt:87disp.obj
 0001:0000d462       __rtindfnpop               1000e462     libucrt:87disp.obj
 0001:0000d473       __rttosnpopde              1000e473     libucrt:87disp.obj
 0001:0000d480       __rtatan2inf               1000e480 f   libucrt:87disp.obj
 0001:0000d49d       __rtchsifneg               1000e49d     libucrt:87disp.obj
 0001:0000d4b0       __twoToTOS                 1000e4b0 f   libucrt:common.obj
 0001:0000d4c5       __load_CW                  1000e4c5 f   libucrt:common.obj
 0001:0000d4dc       __convertTOStoQNaN         1000e4dc f   libucrt:common.obj
 0001:0000d4f5       __fload_withFB             1000e4f5 f   libucrt:common.obj
 0001:0000d538       __checkTOS_withFB          1000e538 f   libucrt:common.obj
 0001:0000d54e       __fast_exit                1000e54e f   libucrt:common.obj
 0001:0000d55b       __math_exit                1000e55b f   libucrt:common.obj
 0001:0000d585       __check_overflow_exit      1000e585 f   libucrt:common.obj
 0001:0000d599       __check_range_exit         1000e599 f   libucrt:common.obj
 0001:0000d640       __startTwoArgErrorHandling 1000e640 f   libucrt:genexcep.obj
 0001:0000d657       __startOneArgErrorHandling 1000e657 f   libucrt:genexcep.obj
 0001:0000d693       ___libm_error_support      1000e693 f   libucrt:libm_error.obj
 0001:0000d887       __ceil_default             1000e887 f   libucrt:ceil.obj
 0001:0000d93c       __clrfp                    1000e93c f   libucrt:fpctrl.obj
 0001:0000d94d       __ctrlfp                   1000e94d f   libucrt:fpctrl.obj
 0001:0000d977       __set_statfp               1000e977 f   libucrt:fpctrl.obj
 0001:0000d9d0       __statfp                   1000e9d0 f   libucrt:fpctrl.obj
 0001:0000d9e0       __d_inttype                1000e9e0 f   libucrt:powhlp.obj
 0001:0000da48       __powhlp                   1000ea48 f   libucrt:powhlp.obj
 0001:0000db73       __87except                 1000eb73 f   libucrt:87except.obj
 0001:0000dc7d       __frnd                     1000ec7d f   libucrt:frnd.obj
 0001:0000dc91       __errcode                  1000ec91 f   libucrt:fpexcept.obj
 0001:0000dcc5       __except1                  1000ecc5 f   libucrt:fpexcept.obj
 0001:0000dd93       __handle_exc               1000ed93 f   libucrt:fpexcept.obj
 0001:0000df7e       __raise_exc                1000ef7e f   libucrt:fpexcept.obj
 0001:0000dfa1       __raise_exc_ex             1000efa1 f   libucrt:fpexcept.obj
 0001:0000e297       __set_errno_from_matherr   1000f297 f   libucrt:fpexcept.obj
 0001:0000e2c6       __umatherr                 1000f2c6 f   libucrt:fpexcept.obj
 0001:0000e366       __decomp                   1000f366 f   libucrt:util.obj
 0001:0000e438       __set_exp                  1000f438 f   libucrt:util.obj
 0001:0000e465       __sptype                   1000f465 f   libucrt:util.obj
 0001:0000e4c3       __fpclass                  1000f4c3 f   libucrt:ieeemisc.obj
 0001:0000e570       __FindPESection            1000f570 f   LIBCMT:pesect.obj
 0001:0000e5c0       __IsNonwritableInCurrentImage 1000f5c0 f   LIBCMT:pesect.obj
 0001:0000e680       __ValidateImageBase        1000f680 f   LIBCMT:pesect.obj
 0001:0000e6b3       __EH_prolog3_catch         1000f6b3 f   LIBCMT:ehprolg3.obj
 0001:0000e6f0       __alloca_probe_16          1000f6f0 f   LIBCMT:alloca16.obj
 0001:0000e706       __alloca_probe_8           1000f706     LIBCMT:alloca16.obj
 0001:0000e720       __alloca_probe             1000f720 f   LIBCMT:chkstk.obj
 0001:0000e720       __chkstk                   1000f720 f   LIBCMT:chkstk.obj
 0001:0000e750       __filter_x86_sse2_floating_point_exception 1000f750 f   LIBCMT:x86_exception_filter.obj
 0001:0000e750       __filter_x86_sse2_floating_point_exception_default 1000f750 f   LIBCMT:x86_exception_filter.obj
 0002:00000000       __imp__GetFullPathNameW@16 10010000     kernel32:KERNEL32.dll
 0002:00000004       __imp__lstrlenW@4          10010004     kernel32:KERNEL32.dll
 0002:00000008       __imp__WriteFile@20        10010008     kernel32:KERNEL32.dll
 0002:0000000c       __imp__lstrcpynW@12        1001000c     kernel32:KERNEL32.dll
 0002:00000010       __imp__ExpandEnvironmentStringsW@12 10010010     kernel32:KERNEL32.dll
 0002:00000014       __imp__CreateFileW@28      10010014     kernel32:KERNEL32.dll
 0002:00000018       __imp__GetFileAttributesW@4 10010018     kernel32:KERNEL32.dll
 0002:0000001c       __imp__lstrcatW@8          1001001c     kernel32:KERNEL32.dll
 0002:00000020       __imp__DeleteFileW@4       10010020     kernel32:KERNEL32.dll
 0002:00000024       __imp__CloseHandle@4       10010024     kernel32:KERNEL32.dll
 0002:00000028       __imp__lstrcpyW@8          10010028     kernel32:KERNEL32.dll
 0002:0000002c       __imp__CompareStringW@24   1001002c     kernel32:KERNEL32.dll
 0002:00000030       __imp__SetLastError@4      10010030     kernel32:KERNEL32.dll
 0002:00000034       __imp__EnterCriticalSection@4 10010034     kernel32:KERNEL32.dll
 0002:00000038       __imp__GetModuleFileNameW@12 10010038     kernel32:KERNEL32.dll
 0002:0000003c       __imp__LeaveCriticalSection@4 1001003c     kernel32:KERNEL32.dll
 0002:00000040       __imp__InitializeCriticalSection@4 10010040     kernel32:KERNEL32.dll
 0002:00000044       __imp__GetCurrentThread@0  10010044     kernel32:KERNEL32.dll
 0002:00000048       __imp__LoadLibraryW@4      10010048     kernel32:KERNEL32.dll
 0002:0000004c       __imp__GetProcAddress@8    1001004c     kernel32:KERNEL32.dll
 0002:00000050       __imp__DeleteCriticalSection@4 10010050     kernel32:KERNEL32.dll
 0002:00000054       __imp__LCMapStringW@24     10010054     kernel32:KERNEL32.dll
 0002:00000058       __imp__GetModuleHandleW@4  10010058     kernel32:KERNEL32.dll
 0002:0000005c       __imp__GetThreadTimes@20   1001005c     kernel32:KERNEL32.dll
 0002:00000060       __imp__VirtualQuery@12     10010060     kernel32:KERNEL32.dll
 0002:00000064       __imp__UnhandledExceptionFilter@4 10010064     kernel32:KERNEL32.dll
 0002:00000068       __imp__SetUnhandledExceptionFilter@4 10010068     kernel32:KERNEL32.dll
 0002:0000006c       __imp__GetCurrentProcess@0 1001006c     kernel32:KERNEL32.dll
 0002:00000070       __imp__TerminateProcess@8  10010070     kernel32:KERNEL32.dll
 0002:00000074       __imp__IsProcessorFeaturePresent@4 10010074     kernel32:KERNEL32.dll
 0002:00000078       __imp__IsDebuggerPresent@0 10010078     kernel32:KERNEL32.dll
 0002:0000007c       __imp__GetStartupInfoW@4   1001007c     kernel32:KERNEL32.dll
 0002:00000080       __imp__QueryPerformanceCounter@4 10010080     kernel32:KERNEL32.dll
 0002:00000084       __imp__GetCurrentProcessId@0 10010084     kernel32:KERNEL32.dll
 0002:00000088       __imp__GetCurrentThreadId@0 10010088     kernel32:KERNEL32.dll
 0002:0000008c       __imp__GetSystemTimeAsFileTime@4 1001008c     kernel32:KERNEL32.dll
 0002:00000090       __imp__RtlUnwind@16        10010090     kernel32:KERNEL32.dll
 0002:00000094       __imp__RaiseException@16   10010094     kernel32:KERNEL32.dll
 0002:00000098       __imp__GetLastError@0      10010098     kernel32:KERNEL32.dll
 0002:0000009c       __imp__InitializeCriticalSectionAndSpinCount@8 1001009c     kernel32:KERNEL32.dll
 0002:000000a0       __imp__TlsAlloc@0          100100a0     kernel32:KERNEL32.dll
 0002:000000a4       __imp__TlsGetValue@4       100100a4     kernel32:KERNEL32.dll
 0002:000000a8       __imp__TlsSetValue@8       100100a8     kernel32:KERNEL32.dll
 0002:000000ac       __imp__TlsFree@4           100100ac     kernel32:KERNEL32.dll
 0002:000000b0       __imp__FreeLibrary@4       100100b0     kernel32:KERNEL32.dll
 0002:000000b4       __imp__LoadLibraryExW@12   100100b4     kernel32:KERNEL32.dll
 0002:000000b8       __imp__ExitProcess@4       100100b8     kernel32:KERNEL32.dll
 0002:000000bc       __imp__HeapFree@12         100100bc     kernel32:KERNEL32.dll
 0002:000000c0       __imp__HeapAlloc@12        100100c0     kernel32:KERNEL32.dll
 0002:000000c4       __imp__FindClose@4         100100c4     kernel32:KERNEL32.dll
 0002:000000c8       __imp__FindFirstFileExW@24 100100c8     kernel32:KERNEL32.dll
 0002:000000cc       __imp__FindNextFileW@8     100100cc     kernel32:KERNEL32.dll
 0002:000000d0       __imp__IsValidCodePage@4   100100d0     kernel32:KERNEL32.dll
 0002:000000d4       __imp__GetACP@0            100100d4     kernel32:KERNEL32.dll
 0002:000000d8       __imp__GetOEMCP@0          100100d8     kernel32:KERNEL32.dll
 0002:000000dc       __imp__GetCPInfo@8         100100dc     kernel32:KERNEL32.dll
 0002:000000e0       __imp__GetCommandLineA@0   100100e0     kernel32:KERNEL32.dll
 0002:000000e4       __imp__GetCommandLineW@0   100100e4     kernel32:KERNEL32.dll
 0002:000000e8       __imp__MultiByteToWideChar@24 100100e8     kernel32:KERNEL32.dll
 0002:000000ec       __imp__WideCharToMultiByte@32 100100ec     kernel32:KERNEL32.dll
 0002:000000f0       __imp__GetEnvironmentStringsW@0 100100f0     kernel32:KERNEL32.dll
 0002:000000f4       __imp__FreeEnvironmentStringsW@4 100100f4     kernel32:KERNEL32.dll
 0002:000000f8       __imp__GetProcessHeap@0    100100f8     kernel32:KERNEL32.dll
 0002:000000fc       __imp__GetStdHandle@4      100100fc     kernel32:KERNEL32.dll
 0002:00000100       __imp__GetFileType@4       10010100     kernel32:KERNEL32.dll
 0002:00000104       __imp__GetStringTypeW@16   10010104     kernel32:KERNEL32.dll
 0002:00000108       __imp__HeapSize@12         10010108     kernel32:KERNEL32.dll
 0002:0000010c       __imp__HeapReAlloc@16      1001010c     kernel32:KERNEL32.dll
 0002:00000110       __imp__SetStdHandle@8      10010110     kernel32:KERNEL32.dll
 0002:00000114       __imp__FlushFileBuffers@4  10010114     kernel32:KERNEL32.dll
 0002:00000118       __imp__GetConsoleCP@0      10010118     kernel32:KERNEL32.dll
 0002:0000011c       __imp__GetConsoleMode@8    1001011c     kernel32:KERNEL32.dll
 0002:00000120       __imp__SetFilePointerEx@20 10010120     kernel32:KERNEL32.dll
 0002:00000124       __imp__WriteConsoleW@20    10010124     kernel32:KERNEL32.dll
 0002:00000128       \177KERNEL32_NULL_THUNK_DATA 10010128     kernel32:KERNEL32.dll
 0002:0000012c       __imp__UuidFromStringW@8   1001012c     rpcrt4:RPCRT4.dll
 0002:00000130       \177RPCRT4_NULL_THUNK_DATA 10010130     rpcrt4:RPCRT4.dll
 0002:00000134       ___guard_check_icall_fptr  10010134     LIBCMT:guard_support.obj
 0002:00000138       ___xc_a                    10010138     LIBCMT:initializers.obj
 0002:0000013c       ___xc_z                    1001013c     LIBCMT:initializers.obj
 0002:00000140       ___xi_a                    10010140     LIBCMT:initializers.obj
 0002:00000144       ___acrt_multibyte_initializer 10010144     libucrt:multibyte_initializer.obj
 0002:00000148       ___acrt_stdio_initializer  10010148     libucrt:stdio_initializer.obj
 0002:0000014c       ___acrt_tran_sse2_initializer 1001014c     libucrt:sse2_initializer.obj
 0002:00000150       ___xi_z                    10010150     LIBCMT:initializers.obj
 0002:00000154       ___xp_a                    10010154     LIBCMT:initializers.obj
 0002:00000158       ___acrt_locale_terminator  10010158     libucrt:locale_initializer.obj
 0002:0000015c       ___dcrt_console_output_terminator 1001015c     libucrt:console_output_initializer.obj
 0002:00000160       ___acrt_stdio_terminator   10010160     libucrt:stdio_initializer.obj
 0002:00000164       ___xp_z                    10010164     LIBCMT:initializers.obj
 0002:00000168       ___xt_a                    10010168     LIBCMT:initializers.obj
 0002:0000016c       ___xt_z                    1001016c     LIBCMT:initializers.obj
 0002:00000170       __imp__EncodePointer@4     10010170     vc_crt_fix.obj
 0002:00000174       __imp__DecodePointer@4     10010174     vc_crt_fix.obj
 0002:00000178       __imp__GetModuleHandleExW@12 10010178     vc_crt_fix.obj
 0002:0000017c       __imp__InitializeSListHead@4 1001017c     vc_crt_fix.obj
 0002:00000180       __imp__InterlockedFlushSList@4 10010180     vc_crt_fix.obj
 0002:00000184       __imp__InterlockedPopEntrySList@4 10010184     vc_crt_fix.obj
 0002:00000188       __imp__InterlockedPushEntrySList@8 10010188     vc_crt_fix.obj
 0002:0000018c       __imp__InterlockedPushListSListEx@16 1001018c     vc_crt_fix.obj
 0002:00000190       __imp__RtlFirstEntrySList@4 10010190     vc_crt_fix.obj
 0002:00000194       __imp__QueryDepthSList@4   10010194     vc_crt_fix.obj
 0002:00000198       __imp__GetNumaHighestNodeNumber@4 10010198     vc_crt_fix.obj
 0002:0000019c       __imp__GetLogicalProcessorInformation@8 1001019c     vc_crt_fix.obj
 0002:000001a0       __imp__SetThreadStackGuarantee@4 100101a0     vc_crt_fix.obj
 0002:000001a4       __imp__InitializeCriticalSectionEx@12 100101a4     vc_crt_fix.obj
 0002:000001a8       __imp__CompareStringEx@36  100101a8     vc_crt_fix.obj
 0002:000001ac       __imp__LCMapStringEx@36    100101ac     vc_crt_fix.obj
 0002:000001b4       ??_7exception@std@@6B@     100101b4     libcpmt:xthrow.obj
 0002:000001c0       ??_7bad_alloc@std@@6B@     100101c0     libcpmt:xthrow.obj
 0002:000001c8       ??_C@_0P@GHFPNOJB@bad?5allocation@ 100101c8     libcpmt:xthrow.obj
 0002:000001dc       ??_7logic_error@std@@6B@   100101dc     libcpmt:xthrow.obj
 0002:000001e8       ??_7length_error@std@@6B@  100101e8     libcpmt:xthrow.obj
 0002:000001fc       ??_7type_info@@6B@         100101fc     LIBCMT:std_type_info_static.obj
 0002:00000200       __pRawDllMain              10010200     LIBCMT:dll_dllmain.obj
 0002:00000200       __pDefaultRawDllMain       10010200     LIBCMT:dll_dllmain.obj
 0002:00000208       ??_7bad_array_new_length@std@@6B@ 10010208     LIBCMT:throw_bad_alloc.obj
 0002:00000210       __pDestructExceptionObject 10010210     libvcruntime:ehhelpers.obj
 0002:00000218       ??_7bad_exception@std@@6B@ 10010218     libvcruntime:frame.obj
 0002:00000220       ??_C@_0O@DPKOEFFH@bad?5exception@ 10010220     libvcruntime:frame.obj
 0002:000005b0       ??_C@_08EHJDFFNH@__based?$CI@ 100105b0     libvcruntime:undname.obj
 0002:000005bc       ??_C@_07KOLFKCDI@__cdecl@  100105bc     libvcruntime:undname.obj
 0002:000005c4       ??_C@_08GHMPAG@__pascal@   100105c4     libvcruntime:undname.obj
 0002:000005d0       ??_C@_09IFJBGAPI@__stdcall@ 100105d0     libvcruntime:undname.obj
 0002:000005dc       ??_C@_0L@NPHFGOKO@__thiscall@ 100105dc     libvcruntime:undname.obj
 0002:000005e8       ??_C@_0L@JMKHOMEK@__fastcall@ 100105e8     libvcruntime:undname.obj
 0002:000005f4       ??_C@_0N@BCKKPABJ@__vectorcall@ 100105f4     libvcruntime:undname.obj
 0002:00000604       ??_C@_09HIJEGCPM@__clrcall@ 10010604     libvcruntime:undname.obj
 0002:00000610       ??_C@_06GHPCKEAG@__eabi@   10010610     libvcruntime:undname.obj
 0002:00000618       ??_C@_09IOPIDJLG@__swift_1@ 10010618     libvcruntime:undname.obj
 0002:00000624       ??_C@_09KFNFGKHF@__swift_2@ 10010624     libvcruntime:undname.obj
 0002:00000630       ??_C@_07JOMMBBKO@__ptr64@  10010630     libvcruntime:undname.obj
 0002:00000638       ??_C@_0L@PILCLIHE@__restrict@ 10010638     libvcruntime:undname.obj
 0002:00000644       ??_C@_0M@GFIIJFMG@__unaligned@ 10010644     libvcruntime:undname.obj
 0002:00000650       ??_C@_09DHDLOLLB@restrict?$CI@ 10010650     libvcruntime:undname.obj
 0002:0000065a       ??_C@_00CNPNBAHC@@         1001065a     libvcruntime:undname.obj
 0002:0000065c       ??_C@_04NIHEBCM@?5new@     1001065c     libvcruntime:undname.obj
 0002:00000664       ??_C@_07FPCDHGMM@?5delete@ 10010664     libvcruntime:undname.obj
 0002:0000066c       ??_C@_01NEMOKFLO@?$DN@     1001066c     libvcruntime:undname.obj
 0002:00000670       ??_C@_02GPIOPFAK@?$DO?$DO@ 10010670     libvcruntime:undname.obj
 0002:00000674       ??_C@_02FODMEDOG@?$DM?$DM@ 10010674     libvcruntime:undname.obj
 0002:00000678       ??_C@_01DCLJPIOD@?$CB@     10010678     libvcruntime:undname.obj
 0002:0000067c       ??_C@_02EGOFBIJA@?$DN?$DN@ 1001067c     libvcruntime:undname.obj
 0002:00000680       ??_C@_02FDNJECIE@?$CB?$DN@ 10010680     libvcruntime:undname.obj
 0002:00000684       ??_C@_02GPECMEKF@?$FL?$FN@ 10010684     libvcruntime:undname.obj
 0002:00000688       ??_C@_08LHJFAFGD@operator@ 10010688     libvcruntime:undname.obj
 0002:00000694       ??_C@_02HBOOOICD@?9?$DO@   10010694     libvcruntime:undname.obj
 0002:00000698       ??_C@_01NBENCBCI@?$CK@     10010698     libvcruntime:undname.obj
 0002:0000069c       ??_C@_02ECNGHCIF@?$CL?$CL@ 1001069c     libvcruntime:undname.obj
 0002:000006a0       ??_C@_02BAABKJLB@?9?9@     100106a0     libvcruntime:undname.obj
 0002:000006a4       ??_C@_01JOAMLHOP@?9@       100106a4     libvcruntime:undname.obj
 0002:000006a8       ??_C@_01MIFGBAGJ@?$CL@     100106a8     libvcruntime:undname.obj
 0002:000006ac       ??_C@_01HNPIGOCE@?$CG@     100106ac     libvcruntime:undname.obj
 0002:000006b0       ??_C@_03MNHNFDLC@?9?$DO?$CK@ 100106b0     libvcruntime:undname.obj
 0002:000006b4       ??_C@_01KMDKNFGN@?1@       100106b4     libvcruntime:undname.obj
 0002:000006b8       ??_C@_01FGNFDNOH@?$CF@     100106b8     libvcruntime:undname.obj
 0002:000006bc       ??_C@_01MNNFJEPP@?$DM@     100106bc     libvcruntime:undname.obj
 0002:000006c0       ??_C@_02EHCHHCKH@?$DM?$DN@ 100106c0     libvcruntime:undname.obj
 0002:000006c4       ??_C@_01PPODPGHN@?$DO@     100106c4     libvcruntime:undname.obj
 0002:000006c8       ??_C@_02EEKDKGMJ@?$DO?$DN@ 100106c8     libvcruntime:undname.obj
 0002:000006cc       ??_C@_01IHBHIGKO@?0@       100106cc     libvcruntime:undname.obj
 0002:000006d0       ??_C@_02HCKGKOFO@?$CI?$CJ@ 100106d0     libvcruntime:undname.obj
 0002:000006d4       ??_C@_01PJKLJHI@?$HO@      100106d4     libvcruntime:undname.obj
 0002:000006d8       ??_C@_01JKBOJNNK@?$FO@     100106d8     libvcruntime:undname.obj
 0002:000006dc       ??_C@_01DNKMNLPK@?$HM@     100106dc     libvcruntime:undname.obj
 0002:000006e0       ??_C@_02PPKAJPJL@?$CG?$CG@ 100106e0     libvcruntime:undname.obj
 0002:000006e4       ??_C@_02NONPIBCD@?$HM?$HM@ 100106e4     libvcruntime:undname.obj
 0002:000006e8       ??_C@_02FPIMKNGF@?$CK?$DN@ 100106e8     libvcruntime:undname.obj
 0002:000006ec       ??_C@_02FOEOMHFC@?$CL?$DN@ 100106ec     libvcruntime:undname.obj
 0002:000006f0       ??_C@_02FKMDLLOA@?9?$DN@   100106f0     libvcruntime:undname.obj
 0002:000006f4       ??_C@_02FJEHGPIO@?1?$DN@   100106f4     libvcruntime:undname.obj
 0002:000006f8       ??_C@_02FENAOKFI@?$CF?$DN@ 100106f8     libvcruntime:undname.obj
 0002:000006fc       ??_C@_03IKFCCPFF@?$DO?$DO?$DN@ 100106fc     libvcruntime:undname.obj
 0002:00000700       ??_C@_03CDNPDDLA@?$DM?$DM?$DN@ 10010700     libvcruntime:undname.obj
 0002:00000704       ??_C@_02FGJGFEAB@?$CG?$DN@ 10010704     libvcruntime:undname.obj
 0002:00000708       ??_C@_02DHLNPPGH@?$HM?$DN@ 10010708     libvcruntime:undname.obj
 0002:0000070c       ??_C@_02MHEGNOJ@?$FO?$DN@  1001070c     libvcruntime:undname.obj
 0002:00000710       ??_C@_09IFPLHPGF@?$GAvftable?8@ 10010710     libvcruntime:undname.obj
 0002:0000071c       ??_C@_09BLBHBJP@?$GAvbtable?8@ 1001071c     libvcruntime:undname.obj
 0002:00000728       ??_C@_07FEEIOKP@?$GAvcall?8@ 10010728     libvcruntime:undname.obj
 0002:00000730       ??_C@_08LLFFHHDJ@?$GAtypeof?8@ 10010730     libvcruntime:undname.obj
 0002:0000073c       ??_C@_0BF@KDPPACIK@?$GAlocal?5static?5guard?8@ 1001073c     libvcruntime:undname.obj
 0002:00000754       ??_C@_08OBABFOLI@?$GAstring?8@ 10010754     libvcruntime:undname.obj
 0002:00000760       ??_C@_0BD@JDLKDPAB@?$GAvbase?5destructor?8@ 10010760     libvcruntime:undname.obj
 0002:00000774       ??_C@_0BN@DEGPLNFK@?$GAvector?5deleting?5destructor?8@ 10010774     libvcruntime:undname.obj
 0002:00000794       ??_C@_0BO@OBMKPJIG@?$GAdefault?5constructor?5closure?8@ 10010794     libvcruntime:undname.obj
 0002:000007b4       ??_C@_0BN@IMDCHIKM@?$GAscalar?5deleting?5destructor?8@ 100107b4     libvcruntime:undname.obj
 0002:000007d4       ??_C@_0BO@PFGOCPJJ@?$GAvector?5constructor?5iterator?8@ 100107d4     libvcruntime:undname.obj
 0002:000007f4       ??_C@_0BN@LFPFMEDL@?$GAvector?5destructor?5iterator?8@ 100107f4     libvcruntime:undname.obj
 0002:00000814       ??_C@_0CE@IKBNEHA@?$GAvector?5vbase?5constructor?5itera@ 10010814     libvcruntime:undname.obj
 0002:00000838       ??_C@_0BL@NILFHHPC@?$GAvirtual?5displacement?5map?8@ 10010838     libvcruntime:undname.obj
 0002:00000854       ??_C@_0CB@JONCMFFK@?$GAeh?5vector?5constructor?5iterator@ 10010854     libvcruntime:undname.obj
 0002:00000878       ??_C@_0CA@GCEOPDGL@?$GAeh?5vector?5destructor?5iterator?8@ 10010878     libvcruntime:undname.obj
 0002:00000898       ??_C@_0CH@OOJPLCPH@?$GAeh?5vector?5vbase?5constructor?5it@ 10010898     libvcruntime:undname.obj
 0002:000008c0       ??_C@_0BL@LLKPOHJI@?$GAcopy?5constructor?5closure?8@ 100108c0     libvcruntime:undname.obj
 0002:000008dc       ??_C@_0BA@KBCDOMBN@?$GAudt?5returning?8@ 100108dc     libvcruntime:undname.obj
 0002:000008ec       ??_C@_03KLGMFNMG@?$GAEH@   100108ec     libvcruntime:undname.obj
 0002:000008f0       ??_C@_05KHLCHHI@?$GARTTI@  100108f0     libvcruntime:undname.obj
 0002:000008f8       ??_C@_0BA@KKLDJDLB@?$GAlocal?5vftable?8@ 100108f8     libvcruntime:undname.obj
 0002:00000908       ??_C@_0CE@IIHCMGGL@?$GAlocal?5vftable?5constructor?5clos@ 10010908     libvcruntime:undname.obj
 0002:0000092c       ??_C@_06FHBGPFGH@?5new?$FL?$FN@ 1001092c     libvcruntime:undname.obj
 0002:00000934       ??_C@_09LBNFPBCA@?5delete?$FL?$FN@ 10010934     libvcruntime:undname.obj
 0002:00000940       ??_C@_0P@HJKNJFNN@?$GAomni?5callsig?8@ 10010940     libvcruntime:undname.obj
 0002:00000950       ??_C@_0BL@CNOONJFP@?$GAplacement?5delete?5closure?8@ 10010950     libvcruntime:undname.obj
 0002:0000096c       ??_C@_0BN@CKNJLHMB@?$GAplacement?5delete?$FL?$FN?5closure?8@ 1001096c     libvcruntime:undname.obj
 0002:0000098c       ??_C@_0CG@CFDHKGGD@?$GAmanaged?5vector?5constructor?5ite@ 1001098c     libvcruntime:undname.obj
 0002:000009b4       ??_C@_0CF@IMGKMJNO@?$GAmanaged?5vector?5destructor?5iter@ 100109b4     libvcruntime:undname.obj
 0002:000009dc       ??_C@_0CG@HLDDJMAG@?$GAeh?5vector?5copy?5constructor?5ite@ 100109dc     libvcruntime:undname.obj
 0002:00000a04       ??_C@_0CM@FCBBDIGB@?$GAeh?5vector?5vbase?5copy?5construct@ 10010a04     libvcruntime:undname.obj
 0002:00000a30       ??_C@_0BL@CLIPGLGB@?$GAdynamic?5initializer?5for?5?8@ 10010a30     libvcruntime:undname.obj
 0002:00000a4c       ??_C@_0CB@PDBIFEP@?$GAdynamic?5atexit?5destructor?5for?5@ 10010a4c     libvcruntime:undname.obj
 0002:00000a70       ??_C@_0CD@CGAJBKEJ@?$GAvector?5copy?5constructor?5iterat@ 10010a70     libvcruntime:undname.obj
 0002:00000a94       ??_C@_0CJ@GJELGAMM@?$GAvector?5vbase?5copy?5constructor?5@ 10010a94     libvcruntime:undname.obj
 0002:00000ac0       ??_C@_0CL@FGIJHLCE@?$GAmanaged?5vector?5copy?5constructo@ 10010ac0     libvcruntime:undname.obj
 0002:00000aec       ??_C@_0BM@PMGGMLDN@?$GAlocal?5static?5thread?5guard?8@ 10010aec     libvcruntime:undname.obj
 0002:00000b08       ??_C@_0N@BDNMDMOL@operator?5?$CC?$CC?5@ 10010b08     libvcruntime:undname.obj
 0002:00000b18       ??_C@_0BC@GGEBGALA@operator?5co_await@ 10010b18     libvcruntime:undname.obj
 0002:00000b2c       ??_C@_0M@GAAIMMOH@operator?$DM?$DN?$DO@ 10010b2c     libvcruntime:undname.obj
 0002:00000b38       ??_C@_0BC@DAFEJGAK@?5Type?5Descriptor?8@ 10010b38     libvcruntime:undname.obj
 0002:00000b4c       ??_C@_0BM@LDKODKLH@?5Base?5Class?5Descriptor?5at?5?$CI@ 10010b4c     libvcruntime:undname.obj
 0002:00000b68       ??_C@_0BD@LGICGFMM@?5Base?5Class?5Array?8@ 10010b68     libvcruntime:undname.obj
 0002:00000b7c       ??_C@_0BN@MECKDCOJ@?5Class?5Hierarchy?5Descriptor?8@ 10010b7c     libvcruntime:undname.obj
 0002:00000b9c       ??_C@_0BK@CFCOFLF@?5Complete?5Object?5Locator?8@ 10010b9c     libvcruntime:undname.obj
 0002:00000bb8       ??_C@_0BG@JNJLAMPM@?$GAanonymous?5namespace?8@ 10010bb8     libvcruntime:undname.obj
 0002:00000bdc       ??_C@_1DM@KHCHBNEB@?$AAa?$AAp?$AAi?$AA?9?$AAm?$AAs?$AA?9?$AAw?$AAi?$AAn?$AA?9?$AAc?$AAo?$AAr?$AAe@ 10010bdc     libvcruntime:winapi_downlevel.obj
 0002:00000c18       ??_C@_1DK@LPPGFMPP@?$AAa?$AAp?$AAi?$AA?9?$AAm?$AAs?$AA?9?$AAw?$AAi?$AAn?$AA?9?$AAc?$AAo?$AAr?$AAe@ 10010c18     libvcruntime:winapi_downlevel.obj
 0002:00000c54       ??_C@_1BC@GDMECMAK@?$AAk?$AAe?$AAr?$AAn?$AAe?$AAl?$AA3?$AA2@ 10010c54     libvcruntime:winapi_downlevel.obj
 0002:00000c68       ??_C@_1BA@PFFKHIOG@?$AAa?$AAp?$AAi?$AA?9?$AAm?$AAs?$AA?9@ 10010c68     libvcruntime:winapi_downlevel.obj
 0002:00000c80       ??_C@_08KNHFBNJ@FlsAlloc@  10010c80     libvcruntime:winapi_downlevel.obj
 0002:00000c94       ??_C@_07PEJMOBNF@FlsFree@  10010c94     libvcruntime:winapi_downlevel.obj
 0002:00000ca4       ??_C@_0M@GDNOONDI@FlsGetValue@ 10010ca4     libvcruntime:winapi_downlevel.obj
 0002:00000cb8       ??_C@_0M@JCPCPOEF@FlsSetValue@ 10010cb8     libvcruntime:winapi_downlevel.obj
 0002:00000cd0       ___acrt_exception_action_table 10010cd0     libucrt:exception_filter.obj
 0002:00000d60       ___acrt_signal_action_table_count 10010d60     libucrt:exception_filter.obj
 0002:00000d64       ___acrt_signal_action_first_fpe_index 10010d64     libucrt:exception_filter.obj
 0002:00000d68       ___acrt_signal_action_fpe_count 10010d68     libucrt:exception_filter.obj
 0002:00000d6c       ??_C@_1BI@BGOHAHKC@?$AAm?$AAs?$AAc?$AAo?$AAr?$AAe?$AAe?$AA?4?$AAd?$AAl?$AAl@ 10010d6c     libucrt:exit.obj
 0002:00000d84       ??_C@_0P@MIGLKIOC@CorExitProcess@ 10010d84     libucrt:exit.obj
 0002:00000f90       ??_C@_1M@HPNHIDJI@?$AAj?$AAa?$AA?9?$AAJ?$AAP@ 10010f90     libucrt:mbctype.obj
 0002:00000f9c       ??_C@_1M@BIBDDEMK@?$AAz?$AAh?$AA?9?$AAC?$AAN@ 10010f9c     libucrt:mbctype.obj
 0002:00000fa8       ??_C@_1M@JLOOOEGK@?$AAk?$AAo?$AA?9?$AAK?$AAR@ 10010fa8     libucrt:mbctype.obj
 0002:00000fb4       ??_C@_1M@CLNBBOPM@?$AAz?$AAh?$AA?9?$AAT?$AAW@ 10010fb4     libucrt:mbctype.obj
 0002:00001010       ??_C@_1EA@JGEFHKEI@?$AAa?$AAp?$AAi?$AA?9?$AAm?$AAs?$AA?9?$AAw?$AAi?$AAn?$AA?9?$AAc?$AAo?$AAr?$AAe@ 10011010     libucrt:winapi_thunks.obj
 0002:00001050       ??_C@_1DI@IJCEHOCB@?$AAa?$AAp?$AAi?$AA?9?$AAm?$AAs?$AA?9?$AAw?$AAi?$AAn?$AA?9?$AAc?$AAo?$AAr?$AAe@ 10011050     libucrt:winapi_thunks.obj
 0002:00001088       ??_C@_1EI@MPIAOHOC@?$AAa?$AAp?$AAi?$AA?9?$AAm?$AAs?$AA?9?$AAw?$AAi?$AAn?$AA?9?$AAc?$AAo?$AAr?$AAe@ 10011088     libucrt:winapi_thunks.obj
 0002:000010d0       ??_C@_1FK@FPHCKFIE@?$AAa?$AAp?$AAi?$AA?9?$AAm?$AAs?$AA?9?$AAw?$AAi?$AAn?$AA?9?$AAc?$AAo?$AAr?$AAe@ 100110d0     libucrt:winapi_thunks.obj
 0002:00001130       ??_C@_1EM@DILCGIIO@?$AAa?$AAp?$AAi?$AA?9?$AAm?$AAs?$AA?9?$AAw?$AAi?$AAn?$AA?9?$AAc?$AAo?$AAr?$AAe@ 10011130     libucrt:winapi_thunks.obj
 0002:0000117c       ??_C@_1DM@LNCGDDPN@?$AAa?$AAp?$AAi?$AA?9?$AAm?$AAs?$AA?9?$AAw?$AAi?$AAn?$AA?9?$AAc?$AAo?$AAr?$AAe@ 1001117c     libucrt:winapi_thunks.obj
 0002:000011b8       ??_C@_1DO@FPAPJEMD@?$AAa?$AAp?$AAi?$AA?9?$AAm?$AAs?$AA?9?$AAw?$AAi?$AAn?$AA?9?$AAc?$AAo?$AAr?$AAe@ 100111b8     libucrt:winapi_thunks.obj
 0002:000011f8       ??_C@_1DK@NDHNAHIO@?$AAa?$AAp?$AAi?$AA?9?$AAm?$AAs?$AA?9?$AAw?$AAi?$AAn?$AA?9?$AAc?$AAo?$AAr?$AAe@ 100111f8     libucrt:winapi_thunks.obj
 0002:00001234       ??_C@_1DM@KGHDGBCM@?$AAa?$AAp?$AAi?$AA?9?$AAm?$AAs?$AA?9?$AAw?$AAi?$AAn?$AA?9?$AAc?$AAo?$AAr?$AAe@ 10011234     libucrt:winapi_thunks.obj
 0002:00001270       ??_C@_1EO@IJIOEFOH@?$AAa?$AAp?$AAi?$AA?9?$AAm?$AAs?$AA?9?$AAw?$AAi?$AAn?$AA?9?$AAr?$AAt?$AAc?$AAo@ 10011270     libucrt:winapi_thunks.obj
 0002:000012c0       ??_C@_1FG@HHGEKANL@?$AAa?$AAp?$AAi?$AA?9?$AAm?$AAs?$AA?9?$AAw?$AAi?$AAn?$AA?9?$AAs?$AAe?$AAc?$AAu@ 100112c0     libucrt:winapi_thunks.obj
 0002:00001318       ??_C@_1EG@DBIOJECG@?$AAe?$AAx?$AAt?$AA?9?$AAm?$AAs?$AA?9?$AAw?$AAi?$AAn?$AA?9?$AAn?$AAt?$AAu?$AAs@ 10011318     libucrt:winapi_thunks.obj
 0002:00001360       ??_C@_1EO@FIHMJCLF@?$AAe?$AAx?$AAt?$AA?9?$AAm?$AAs?$AA?9?$AAw?$AAi?$AAn?$AA?9?$AAn?$AAt?$AAu?$AAs@ 10011360     libucrt:winapi_thunks.obj
 0002:000013b0       ??_C@_1BC@DNHGCMLG@?$AAa?$AAd?$AAv?$AAa?$AAp?$AAi?$AA3?$AA2@ 100113b0     libucrt:winapi_thunks.obj
 0002:000013c4       ??_C@_1M@OAIMIKLP@?$AAn?$AAt?$AAd?$AAl?$AAl@ 100113c4     libucrt:winapi_thunks.obj
 0002:000013d0       ??_C@_1EG@DPGNFKGC@?$AAa?$AAp?$AAi?$AA?9?$AAm?$AAs?$AA?9?$AAw?$AAi?$AAn?$AA?9?$AAa?$AAp?$AAp?$AAm@ 100113d0     libucrt:winapi_thunks.obj
 0002:00001418       ??_C@_1O@BCCLBEOE@?$AAu?$AAs?$AAe?$AAr?$AA3?$AA2@ 10011418     libucrt:winapi_thunks.obj
 0002:00001428       ??_C@_1BA@IAIFMGEF@?$AAe?$AAx?$AAt?$AA?9?$AAm?$AAs?$AA?9@ 10011428     libucrt:winapi_thunks.obj
 0002:0000143c       ??_C@_0BA@FHFNEAED@AreFileApisANSI@ 1001143c     libucrt:winapi_thunks.obj
 0002:0000147c       ??_C@_0O@KKBNKAPF@LCMapStringEx@ 1001147c     libucrt:winapi_thunks.obj
 0002:00001494       ??_C@_0BB@HBDEELFH@LocaleNameToLCID@ 10011494     libucrt:winapi_thunks.obj
 0002:000014ac       ??_C@_0CF@OJOFEIGO@AppPolicyGetProcessTerminationM@ 100114ac     libucrt:winapi_thunks.obj
 0002:000014d8       ___lc_time_c               100114d8     libucrt:nlsdata.obj
 0002:0000163c       ??_C@_03KOEHGMDN@Sun@      1001163c     libucrt:nlsdata.obj
 0002:00001640       ??_C@_03PDAGKDH@Mon@       10011640     libucrt:nlsdata.obj
 0002:00001644       ??_C@_03NAGEINEP@Tue@      10011644     libucrt:nlsdata.obj
 0002:00001648       ??_C@_03MHOMLAJA@Wed@      10011648     libucrt:nlsdata.obj
 0002:0000164c       ??_C@_03IOFIKPDN@Thu@      1001164c     libucrt:nlsdata.obj
 0002:00001650       ??_C@_03IDIOELNC@Fri@      10011650     libucrt:nlsdata.obj
 0002:00001654       ??_C@_03FEFJNEK@Sat@       10011654     libucrt:nlsdata.obj
 0002:00001658       ??_C@_06OOPIFAJ@Sunday@    10011658     libucrt:nlsdata.obj
 0002:00001660       ??_C@_06JLEDEDGH@Monday@   10011660     libucrt:nlsdata.obj
 0002:00001668       ??_C@_07BAAGCFCM@Tuesday@  10011668     libucrt:nlsdata.obj
 0002:00001670       ??_C@_09DLIGFAKA@Wednesday@ 10011670     libucrt:nlsdata.obj
 0002:0000167c       ??_C@_08HACCIKIA@Thursday@ 1001167c     libucrt:nlsdata.obj
 0002:00001688       ??_C@_06JECMNKMI@Friday@   10011688     libucrt:nlsdata.obj
 0002:00001690       ??_C@_08INBOOONO@Saturday@ 10011690     libucrt:nlsdata.obj
 0002:0000169c       ??_C@_03JIHJHPIE@Jan@      1001169c     libucrt:nlsdata.obj
 0002:000016a0       ??_C@_03HJBDCHOM@Feb@      100116a0     libucrt:nlsdata.obj
 0002:000016a4       ??_C@_03ODNJBKGA@Mar@      100116a4     libucrt:nlsdata.obj
 0002:000016a8       ??_C@_03LEOLGMJP@Apr@      100116a8     libucrt:nlsdata.obj
 0002:000016ac       ??_C@_03CNMDKL@May@        100116ac     libucrt:nlsdata.obj
 0002:000016b0       ??_C@_03IDFGHECI@Jun@      100116b0     libucrt:nlsdata.obj
 0002:000016b4       ??_C@_03LBGABGKK@Jul@      100116b4     libucrt:nlsdata.obj
 0002:000016b8       ??_C@_03IFJFEIGA@Aug@      100116b8     libucrt:nlsdata.obj
 0002:000016bc       ??_C@_03GGCAPAJC@Sep@      100116bc     libucrt:nlsdata.obj
 0002:000016c0       ??_C@_03BMAOKBAD@Oct@      100116c0     libucrt:nlsdata.obj
 0002:000016c4       ??_C@_03JPJOFNIA@Nov@      100116c4     libucrt:nlsdata.obj
 0002:000016c8       ??_C@_03MKABNOCG@Dec@      100116c8     libucrt:nlsdata.obj
 0002:000016cc       ??_C@_07CGJPFGJA@January@  100116cc     libucrt:nlsdata.obj
 0002:000016d4       ??_C@_08GNJGEPFN@February@ 100116d4     libucrt:nlsdata.obj
 0002:000016e0       ??_C@_05HPCKOFNC@March@    100116e0     libucrt:nlsdata.obj
 0002:000016e8       ??_C@_05DMJDNLEJ@April@    100116e8     libucrt:nlsdata.obj
 0002:000016f0       ??_C@_04CNLMGBGM@June@     100116f0     libucrt:nlsdata.obj
 0002:000016f8       ??_C@_04MIEPOIFP@July@     100116f8     libucrt:nlsdata.obj
 0002:00001700       ??_C@_06LBBHFDDG@August@   10011700     libucrt:nlsdata.obj
 0002:00001708       ??_C@_09BHHEALKD@September@ 10011708     libucrt:nlsdata.obj
 0002:00001714       ??_C@_07JJNFCEND@October@  10011714     libucrt:nlsdata.obj
 0002:0000171c       ??_C@_08HCHEGEOA@November@ 1001171c     libucrt:nlsdata.obj
 0002:00001728       ??_C@_08EDHMEBNP@December@ 10011728     libucrt:nlsdata.obj
 0002:00001734       ??_C@_02DEDBPAFC@AM@       10011734     libucrt:nlsdata.obj
 0002:00001738       ??_C@_02CJNFDJBF@PM@       10011738     libucrt:nlsdata.obj
 0002:0000173c       ??_C@_08BPBNCDIB@MM?1dd?1yy@ 1001173c     libucrt:nlsdata.obj
 0002:00001748       ??_C@_0BE@CKGJFCPC@dddd?0?5MMMM?5dd?0?5yyyy@ 10011748     libucrt:nlsdata.obj
 0002:0000175c       ??_C@_08JCCMCCIL@HH?3mm?3ss@ 1001175c     libucrt:nlsdata.obj
 0002:00001768       ??_C@_17MBGCMIPB@?$AAS?$AAu?$AAn@ 10011768     libucrt:nlsdata.obj
 0002:00001770       ??_C@_17KBOMKBF@?$AAM?$AAo?$AAn@ 10011770     libucrt:nlsdata.obj
 0002:00001778       ??_C@_17BMKGEGOJ@?$AAT?$AAu?$AAe@ 10011778     libucrt:nlsdata.obj
 0002:00001780       ??_C@_17CJEDCEPE@?$AAW?$AAe?$AAd@ 10011780     libucrt:nlsdata.obj
 0002:00001788       ??_C@_17PDPHAADD@?$AAT?$AAh?$AAu@ 10011788     libucrt:nlsdata.obj
 0002:00001790       ??_C@_17HFOLPPLP@?$AAF?$AAr?$AAi@ 10011790     libucrt:nlsdata.obj
 0002:00001798       ??_C@_17GGIBDPIH@?$AAS?$AAa?$AAt@ 10011798     libucrt:nlsdata.obj
 0002:000017a0       ??_C@_1O@IHNHDHPB@?$AAS?$AAu?$AAn?$AAd?$AAa?$AAy@ 100117a0     libucrt:nlsdata.obj
 0002:000017b0       ??_C@_1O@MMNBFLIA@?$AAM?$AAo?$AAn?$AAd?$AAa?$AAy@ 100117b0     libucrt:nlsdata.obj
 0002:000017c0       ??_C@_1BA@ENFBFFEK@?$AAT?$AAu?$AAe?$AAs?$AAd?$AAa?$AAy@ 100117c0     libucrt:nlsdata.obj
 0002:000017d0       ??_C@_1BE@EBOGMDOH@?$AAW?$AAe?$AAd?$AAn?$AAe?$AAs?$AAd?$AAa?$AAy@ 100117d0     libucrt:nlsdata.obj
 0002:000017e4       ??_C@_1BC@HHMNLIHE@?$AAT?$AAh?$AAu?$AAr?$AAs?$AAd?$AAa?$AAy@ 100117e4     libucrt:nlsdata.obj
 0002:000017f8       ??_C@_1O@PDICJHAG@?$AAF?$AAr?$AAi?$AAd?$AAa?$AAy@ 100117f8     libucrt:nlsdata.obj
 0002:00001808       ??_C@_1BC@ENMNNPAJ@?$AAS?$AAa?$AAt?$AAu?$AAr?$AAd?$AAa?$AAy@ 10011808     libucrt:nlsdata.obj
 0002:0000181c       ??_C@_17DKNBKCHM@?$AAJ?$AAa?$AAn@ 1001181c     libucrt:nlsdata.obj
 0002:00001824       ??_C@_17LMDJEKJN@?$AAF?$AAe?$AAb@ 10011824     libucrt:nlsdata.obj
 0002:0000182c       ??_C@_17CKNLEDEC@?$AAM?$AAa?$AAr@ 1001182c     libucrt:nlsdata.obj
 0002:00001834       ??_C@_17LFPOIHDD@?$AAA?$AAp?$AAr@ 10011834     libucrt:nlsdata.obj
 0002:0000183c       ??_C@_17PNNKMEED@?$AAM?$AAa?$AAy@ 1001183c     libucrt:nlsdata.obj
 0002:00001844       ??_C@_17KCJGOCPB@?$AAJ?$AAu?$AAn@ 10011844     libucrt:nlsdata.obj
 0002:0000184c       ??_C@_17IJPCKHK@?$AAJ?$AAu?$AAl@ 1001184c     libucrt:nlsdata.obj
 0002:00001854       ??_C@_17ICPELBCN@?$AAA?$AAu?$AAg@ 10011854     libucrt:nlsdata.obj
 0002:0000185c       ??_C@_17HCHCOKMG@?$AAS?$AAe?$AAp@ 1001185c     libucrt:nlsdata.obj
 0002:00001864       ??_C@_17FNLKOI@?$AAO?$AAc?$AAt@ 10011864     libucrt:nlsdata.obj
 0002:0000186c       ??_C@_17BBDMLCIG@?$AAN?$AAo?$AAv@ 1001186c     libucrt:nlsdata.obj
 0002:00001874       ??_C@_17EGKACKIF@?$AAD?$AAe?$AAc@ 10011874     libucrt:nlsdata.obj
 0002:0000187c       ??_C@_1BA@EFMEIEBA@?$AAJ?$AAa?$AAn?$AAu?$AAa?$AAr?$AAy@ 1001187c     libucrt:nlsdata.obj
 0002:0000188c       ??_C@_1BC@JGDDFFAM@?$AAF?$AAe?$AAb?$AAr?$AAu?$AAa?$AAr?$AAy@ 1001188c     libucrt:nlsdata.obj
 0002:000018a0       ??_C@_1M@IKEENEDF@?$AAM?$AAa?$AAr?$AAc?$AAh@ 100118a0     libucrt:nlsdata.obj
 0002:000018ac       ??_C@_1M@GJNLMHFD@?$AAA?$AAp?$AAr?$AAi?$AAl@ 100118ac     libucrt:nlsdata.obj
 0002:000018b8       ??_C@_19EPFLPGAP@?$AAJ?$AAu?$AAn?$AAe@ 100118b8     libucrt:nlsdata.obj
 0002:000018c4       ??_C@_19BIFMLPCD@?$AAJ?$AAu?$AAl?$AAy@ 100118c4     libucrt:nlsdata.obj
 0002:000018d0       ??_C@_1O@PAHLKOAC@?$AAA?$AAu?$AAg?$AAu?$AAs?$AAt@ 100118d0     libucrt:nlsdata.obj
 0002:000018e0       ??_C@_1BE@DKAAMBJL@?$AAS?$AAe?$AAp?$AAt?$AAe?$AAm?$AAb?$AAe?$AAr@ 100118e0     libucrt:nlsdata.obj
 0002:000018f4       ??_C@_1BA@EPANDLNG@?$AAO?$AAc?$AAt?$AAo?$AAb?$AAe?$AAr@ 100118f4     libucrt:nlsdata.obj
 0002:00001904       ??_C@_1BC@BGLIFPF@?$AAN?$AAo?$AAv?$AAe?$AAm?$AAb?$AAe?$AAr@ 10011904     libucrt:nlsdata.obj
 0002:00001918       ??_C@_1BC@FEMKIFH@?$AAD?$AAe?$AAc?$AAe?$AAm?$AAb?$AAe?$AAr@ 10011918     libucrt:nlsdata.obj
 0002:0000192c       ??_C@_15ODEHAHHF@?$AAA?$AAM@ 1001192c     libucrt:nlsdata.obj
 0002:00001934       ??_C@_15CLMNNGEL@?$AAP?$AAM@ 10011934     libucrt:nlsdata.obj
 0002:0000193c       ??_C@_1BC@IEBCMHCM@?$AAM?$AAM?$AA?1?$AAd?$AAd?$AA?1?$AAy?$AAy@ 1001193c     libucrt:nlsdata.obj
 0002:00001950       ??_C@_1CI@KNAKOEBC@?$AAd?$AAd?$AAd?$AAd?$AA?0?$AA?5?$AAM?$AAM?$AAM?$AAM?$AA?5?$AAd?$AAd?$AA?0?$AA?5@ 10011950     libucrt:nlsdata.obj
 0002:00001978       ??_C@_1BC@GDGBMEMK@?$AAH?$AAH?$AA?3?$AAm?$AAm?$AA?3?$AAs?$AAs@ 10011978     libucrt:nlsdata.obj
 0002:0000198c       ??_C@_1M@BMHNFIME@?$AAe?$AAn?$AA?9?$AAU?$AAS@ 1001198c     libucrt:nlsdata.obj
 0002:00001998       ___newctype                10011998     libucrt:ctype.obj
 0002:00001c98       ___newclmap                10011c98     libucrt:ctype.obj
 0002:00001e18       ___newcumap                10011e18     libucrt:ctype.obj
 0002:000026b8       ??_C@_15EMKDOKLE@?$AAa?$AAr@ 100126b8     libucrt:lcidtoname_downlevel.obj
 0002:000026c0       ??_C@_15KNPADPLH@?$AAb?$AAg@ 100126c0     libucrt:lcidtoname_downlevel.obj
 0002:000026c8       ??_C@_15EDMHLDMO@?$AAc?$AAa@ 100126c8     libucrt:lcidtoname_downlevel.obj
 0002:000026d0       ??_C@_1O@BPEAJADD@?$AAz?$AAh?$AA?9?$AAC?$AAH?$AAS@ 100126d0     libucrt:lcidtoname_downlevel.obj
 0002:000026e0       ??_C@_15LJNHCMNK@?$AAc?$AAs@ 100126e0     libucrt:lcidtoname_downlevel.obj
 0002:000026e8       ??_C@_15FOMCIDHG@?$AAd?$AAa@ 100126e8     libucrt:lcidtoname_downlevel.obj
 0002:000026f0       ??_C@_15NBKABECB@?$AAd?$AAe@ 100126f0     libucrt:lcidtoname_downlevel.obj
 0002:000026f8       ??_C@_15GHPEIIAO@?$AAe?$AAl@ 100126f8     libucrt:lcidtoname_downlevel.obj
 0002:00002700       ??_C@_15MNPNEAIF@?$AAe?$AAn@ 10012700     libucrt:lcidtoname_downlevel.obj
 0002:00002708       ??_C@_15GPIOMPMH@?$AAe?$AAs@ 10012708     libucrt:lcidtoname_downlevel.obj
 0002:00002710       ??_C@_15NGLOAKJC@?$AAf?$AAi@ 10012710     libucrt:lcidtoname_downlevel.obj
 0002:00002718       ??_C@_15FBKGNKAM@?$AAf?$AAr@ 10012718     libucrt:lcidtoname_downlevel.obj
 0002:00002720       ??_C@_15KGGCNEFK@?$AAh?$AAe@ 10012720     libucrt:lcidtoname_downlevel.obj
 0002:00002728       ??_C@_15PGHLIDMF@?$AAh?$AAu@ 10012728     libucrt:lcidtoname_downlevel.obj
 0002:00002730       ??_C@_15BIEMAPLM@?$AAi?$AAs@ 10012730     libucrt:lcidtoname_downlevel.obj
 0002:00002738       ??_C@_15IFJLDHAF@?$AAi?$AAt@ 10012738     libucrt:lcidtoname_downlevel.obj
 0002:00002740       ??_C@_15GEMIOCAG@?$AAj?$AAa@ 10012740     libucrt:lcidtoname_downlevel.obj
 0002:00002748       ??_C@_15EPELEGJA@?$AAk?$AAo@ 10012748     libucrt:lcidtoname_downlevel.obj
 0002:00002750       ??_C@_15NDDHIMN@?$AAn?$AAl@ 10012750     libucrt:lcidtoname_downlevel.obj
 0002:00002758       ??_C@_15BPIGNHCD@?$AAn?$AAo@ 10012758     libucrt:lcidtoname_downlevel.obj
 0002:00002760       ??_C@_15DEOPBLCG@?$AAp?$AAl@ 10012760     libucrt:lcidtoname_downlevel.obj
 0002:00002768       ??_C@_15KBECGEFG@?$AAp?$AAt@ 10012768     libucrt:lcidtoname_downlevel.obj
 0002:00002770       ??_C@_15GLJCBFMD@?$AAr?$AAo@ 10012770     libucrt:lcidtoname_downlevel.obj
 0002:00002778       ??_C@_15FEDGKCDI@?$AAr?$AAu@ 10012778     libucrt:lcidtoname_downlevel.obj
 0002:00002780       ??_C@_15GLKMLLHM@?$AAh?$AAr@ 10012780     libucrt:lcidtoname_downlevel.obj
 0002:00002788       ??_C@_15CPKMFBDB@?$AAs?$AAk@ 10012788     libucrt:lcidtoname_downlevel.obj
 0002:00002790       ??_C@_15BAAIOGMK@?$AAs?$AAq@ 10012790     libucrt:lcidtoname_downlevel.obj
 0002:00002798       ??_C@_15INNPNOHD@?$AAs?$AAv@ 10012798     libucrt:lcidtoname_downlevel.obj
 0002:000027a0       ??_C@_15CABMMOGH@?$AAt?$AAh@ 100127a0     libucrt:lcidtoname_downlevel.obj
 0002:000027a8       ??_C@_15BPLIHJJM@?$AAt?$AAr@ 100127a8     libucrt:lcidtoname_downlevel.obj
 0002:000027b0       ??_C@_15NEOEKKDJ@?$AAu?$AAr@ 100127b0     libucrt:lcidtoname_downlevel.obj
 0002:000027b8       ??_C@_15NFICGAJK@?$AAi?$AAd@ 100127b8     libucrt:lcidtoname_downlevel.obj
 0002:000027c0       ??_C@_15PJPFLCCM@?$AAu?$AAk@ 100127c0     libucrt:lcidtoname_downlevel.obj
 0002:000027c8       ??_C@_15HPJPHDM@?$AAb?$AAe@ 100127c8     libucrt:lcidtoname_downlevel.obj
 0002:000027d0       ??_C@_15LCHLGJII@?$AAs?$AAl@ 100127d0     libucrt:lcidtoname_downlevel.obj
 0002:000027d8       ??_C@_15PCFJPHHO@?$AAe?$AAt@ 100127d8     libucrt:lcidtoname_downlevel.obj
 0002:000027e0       ??_C@_15HPFPGODN@?$AAl?$AAv@ 100127e0     libucrt:lcidtoname_downlevel.obj
 0002:000027e8       ??_C@_15NFFGKGLG@?$AAl?$AAt@ 100127e8     libucrt:lcidtoname_downlevel.obj
 0002:000027f0       ??_C@_15BDAKCCHN@?$AAf?$AAa@ 100127f0     libucrt:lcidtoname_downlevel.obj
 0002:000027f8       ??_C@_15NFGIAIAJ@?$AAv?$AAi@ 100127f8     libucrt:lcidtoname_downlevel.obj
 0002:00002800       ??_C@_15LMKNDMHN@?$AAh?$AAy@ 10012800     libucrt:lcidtoname_downlevel.obj
 0002:00002808       ??_C@_15IJBHMCFL@?$AAa?$AAz@ 10012808     libucrt:lcidtoname_downlevel.obj
 0002:00002810       ??_C@_15EKOFJABL@?$AAe?$AAu@ 10012810     libucrt:lcidtoname_downlevel.obj
 0002:00002818       ??_C@_15BGHADCNK@?$AAm?$AAk@ 10012818     libucrt:lcidtoname_downlevel.obj
 0002:00002820       ??_C@_15JDNICKHM@?$AAa?$AAf@ 10012820     libucrt:lcidtoname_downlevel.obj
 0002:00002828       ??_C@_15KPJEDBKD@?$AAk?$AAa@ 10012828     libucrt:lcidtoname_downlevel.obj
 0002:00002830       ??_C@_15PDNFFFEO@?$AAf?$AAo@ 10012830     libucrt:lcidtoname_downlevel.obj
 0002:00002838       ??_C@_15OMLEGLOC@?$AAh?$AAi@ 10012838     libucrt:lcidtoname_downlevel.obj
 0002:00002840       ??_C@_15IDNNENKK@?$AAm?$AAs@ 10012840     libucrt:lcidtoname_downlevel.obj
 0002:00002848       ??_C@_15MACJNBMH@?$AAk?$AAk@ 10012848     libucrt:lcidtoname_downlevel.obj
 0002:00002850       ??_C@_15DKDJEOND@?$AAk?$AAy@ 10012850     libucrt:lcidtoname_downlevel.obj
 0002:00002858       ??_C@_15DFGDLJBG@?$AAs?$AAw@ 10012858     libucrt:lcidtoname_downlevel.obj
 0002:00002860       ??_C@_15BBFAICNG@?$AAu?$AAz@ 10012860     libucrt:lcidtoname_downlevel.obj
 0002:00002868       ??_C@_15DKNDCGEA@?$AAt?$AAt@ 10012868     libucrt:lcidtoname_downlevel.obj
 0002:00002870       ??_C@_15MGIFMDPL@?$AAp?$AAa@ 10012870     libucrt:lcidtoname_downlevel.obj
 0002:00002878       ??_C@_15HCNDBBA@?$AAg?$AAu@ 10012878     libucrt:lcidtoname_downlevel.obj
 0002:00002880       ??_C@_15FNBEIBON@?$AAt?$AAa@ 10012880     libucrt:lcidtoname_downlevel.obj
 0002:00002888       ??_C@_15NCHGBGLK@?$AAt?$AAe@ 10012888     libucrt:lcidtoname_downlevel.obj
 0002:00002890       ??_C@_15PHPHCBPF@?$AAk?$AAn@ 10012890     libucrt:lcidtoname_downlevel.obj
 0002:00002898       ??_C@_15DLGBCKMP@?$AAm?$AAr@ 10012898     libucrt:lcidtoname_downlevel.obj
 0002:000028a0       ??_C@_15EABBLBFF@?$AAs?$AAa@ 100128a0     libucrt:lcidtoname_downlevel.obj
 0002:000028a8       ??_C@_15CBKOMCOI@?$AAm?$AAn@ 100128a8     libucrt:lcidtoname_downlevel.obj
 0002:000028b0       ??_C@_15CKDMCJAF@?$AAg?$AAl@ 100128b0     libucrt:lcidtoname_downlevel.obj
 0002:000028b8       ??_C@_17CNJFBPG@?$AAk?$AAo?$AAk@ 100128b8     libucrt:lcidtoname_downlevel.obj
 0002:000028c0       ??_C@_17FFBJICPL@?$AAs?$AAy?$AAr@ 100128c0     libucrt:lcidtoname_downlevel.obj
 0002:000028c8       ??_C@_17KPNDCPAF@?$AAd?$AAi?$AAv@ 100128c8     libucrt:lcidtoname_downlevel.obj
 0002:000028d0       ??_C@_1M@OKAHONE@?$AAa?$AAr?$AA?9?$AAS?$AAA@ 100128d0     libucrt:lcidtoname_downlevel.obj
 0002:000028dc       ??_C@_1M@FFFIGIGK@?$AAb?$AAg?$AA?9?$AAB?$AAG@ 100128dc     libucrt:lcidtoname_downlevel.obj
 0002:000028e8       ??_C@_1M@BJNKEDC@?$AAc?$AAa?$AA?9?$AAE?$AAS@ 100128e8     libucrt:lcidtoname_downlevel.obj
 0002:000028f4       ??_C@_1M@IJJHFJHA@?$AAc?$AAs?$AA?9?$AAC?$AAZ@ 100128f4     libucrt:lcidtoname_downlevel.obj
 0002:00002900       ??_C@_1M@CLPEOBGI@?$AAd?$AAa?$AA?9?$AAD?$AAK@ 10012900     libucrt:lcidtoname_downlevel.obj
 0002:0000290c       ??_C@_1M@MCMADGCB@?$AAd?$AAe?$AA?9?$AAD?$AAE@ 1001290c     libucrt:lcidtoname_downlevel.obj
 0002:00002918       ??_C@_1M@OOCKEMAM@?$AAe?$AAl?$AA?9?$AAG?$AAR@ 10012918     libucrt:lcidtoname_downlevel.obj
 0002:00002924       ??_C@_1M@DDNJFGID@?$AAf?$AAi?$AA?9?$AAF?$AAI@ 10012924     libucrt:lcidtoname_downlevel.obj
 0002:00002930       ??_C@_1M@GLIPPMAC@?$AAf?$AAr?$AA?9?$AAF?$AAR@ 10012930     libucrt:lcidtoname_downlevel.obj
 0002:0000293c       ??_C@_1M@GFMCHPE@?$AAh?$AAe?$AA?9?$AAI?$AAL@ 1001293c     libucrt:lcidtoname_downlevel.obj
 0002:00002948       ??_C@_1M@MHLPGNKM@?$AAh?$AAu?$AA?9?$AAH?$AAU@ 10012948     libucrt:lcidtoname_downlevel.obj
 0002:00002954       ??_C@_1M@LPDDNNPN@?$AAi?$AAs?$AA?9?$AAI?$AAS@ 10012954     libucrt:lcidtoname_downlevel.obj
 0002:00002960       ??_C@_1M@MADIPODN@?$AAi?$AAt?$AA?9?$AAI?$AAT@ 10012960     libucrt:lcidtoname_downlevel.obj
 0002:0000296c       ??_C@_1M@IHBJJGG@?$AAn?$AAl?$AA?9?$AAN?$AAL@ 1001296c     libucrt:lcidtoname_downlevel.obj
 0002:00002978       ??_C@_1M@EANAGDL@?$AAn?$AAb?$AA?9?$AAN?$AAO@ 10012978     libucrt:lcidtoname_downlevel.obj
 0002:00002984       ??_C@_1M@NEIEMEGP@?$AAp?$AAl?$AA?9?$AAP?$AAL@ 10012984     libucrt:lcidtoname_downlevel.obj
 0002:00002990       ??_C@_1M@BOCFIGEP@?$AAp?$AAt?$AA?9?$AAB?$AAR@ 10012990     libucrt:lcidtoname_downlevel.obj
 0002:0000299c       ??_C@_1M@IMPFOPBG@?$AAr?$AAo?$AA?9?$AAR?$AAO@ 1001299c     libucrt:lcidtoname_downlevel.obj
 0002:000029a8       ??_C@_1M@IDNNEJMM@?$AAr?$AAu?$AA?9?$AAR?$AAU@ 100129a8     libucrt:lcidtoname_downlevel.obj
 0002:000029b4       ??_C@_1M@LILEEOGM@?$AAh?$AAr?$AA?9?$AAH?$AAR@ 100129b4     libucrt:lcidtoname_downlevel.obj
 0002:000029c0       ??_C@_1M@FKIFEHPB@?$AAs?$AAk?$AA?9?$AAS?$AAK@ 100129c0     libucrt:lcidtoname_downlevel.obj
 0002:000029cc       ??_C@_1M@LJMAMNPJ@?$AAs?$AAq?$AA?9?$AAA?$AAL@ 100129cc     libucrt:lcidtoname_downlevel.obj
 0002:000029d8       ??_C@_1M@GIAKDKJK@?$AAs?$AAv?$AA?9?$AAS?$AAE@ 100129d8     libucrt:lcidtoname_downlevel.obj
 0002:000029e4       ??_C@_1M@MKJKIKCL@?$AAt?$AAh?$AA?9?$AAT?$AAH@ 100129e4     libucrt:lcidtoname_downlevel.obj
 0002:000029f0       ??_C@_1M@MFLCCMPB@?$AAt?$AAr?$AA?9?$AAT?$AAR@ 100129f0     libucrt:lcidtoname_downlevel.obj
 0002:000029fc       ??_C@_1M@OIJHDKJN@?$AAu?$AAr?$AA?9?$AAP?$AAK@ 100129fc     libucrt:lcidtoname_downlevel.obj
 0002:00002a08       ??_C@_1M@LHIPCIEK@?$AAi?$AAd?$AA?9?$AAI?$AAD@ 10012a08     libucrt:lcidtoname_downlevel.obj
 0002:00002a14       ??_C@_1M@MFMOBGI@?$AAu?$AAk?$AA?9?$AAU?$AAA@ 10012a14     libucrt:lcidtoname_downlevel.obj
 0002:00002a20       ??_C@_1M@OBGLJIPL@?$AAb?$AAe?$AA?9?$AAB?$AAY@ 10012a20     libucrt:lcidtoname_downlevel.obj
 0002:00002a2c       ??_C@_1M@BCFAJEAD@?$AAs?$AAl?$AA?9?$AAS?$AAI@ 10012a2c     libucrt:lcidtoname_downlevel.obj
 0002:00002a38       ??_C@_1M@FKFFEDDN@?$AAe?$AAt?$AA?9?$AAE?$AAE@ 10012a38     libucrt:lcidtoname_downlevel.obj
 0002:00002a44       ??_C@_1M@KGKKAACI@?$AAl?$AAv?$AA?9?$AAL?$AAV@ 10012a44     libucrt:lcidtoname_downlevel.obj
 0002:00002a50       ??_C@_1M@IFGBIJO@?$AAl?$AAt?$AA?9?$AAL?$AAT@ 10012a50     libucrt:lcidtoname_downlevel.obj
 0002:00002a5c       ??_C@_1M@FGEAHEDM@?$AAf?$AAa?$AA?9?$AAI?$AAR@ 10012a5c     libucrt:lcidtoname_downlevel.obj
 0002:00002a68       ??_C@_1M@KBMAIBFN@?$AAv?$AAi?$AA?9?$AAV?$AAN@ 10012a68     libucrt:lcidtoname_downlevel.obj
 0002:00002a74       ??_C@_1M@GPCBKDJK@?$AAh?$AAy?$AA?9?$AAA?$AAM@ 10012a74     libucrt:lcidtoname_downlevel.obj
 0002:00002a80       ??_C@_1BG@BECMDDJB@?$AAa?$AAz?$AA?9?$AAA?$AAZ?$AA?9?$AAL?$AAa?$AAt?$AAn@ 10012a80     libucrt:lcidtoname_downlevel.obj
 0002:00002a98       ??_C@_1M@MAOFCAEA@?$AAe?$AAu?$AA?9?$AAE?$AAS@ 10012a98     libucrt:lcidtoname_downlevel.obj
 0002:00002aa4       ??_C@_1M@IGHABKPI@?$AAm?$AAk?$AA?9?$AAM?$AAK@ 10012aa4     libucrt:lcidtoname_downlevel.obj
 0002:00002ab0       ??_C@_1M@IAIGNEJG@?$AAt?$AAn?$AA?9?$AAZ?$AAA@ 10012ab0     libucrt:lcidtoname_downlevel.obj
 0002:00002abc       ??_C@_1M@IIJCOJFA@?$AAx?$AAh?$AA?9?$AAZ?$AAA@ 10012abc     libucrt:lcidtoname_downlevel.obj
 0002:00002ac8       ??_C@_1M@LGPJHNJH@?$AAz?$AAu?$AA?9?$AAZ?$AAA@ 10012ac8     libucrt:lcidtoname_downlevel.obj
 0002:00002ad4       ??_C@_1M@HOKAOIO@?$AAa?$AAf?$AA?9?$AAZ?$AAA@ 10012ad4     libucrt:lcidtoname_downlevel.obj
 0002:00002ae0       ??_C@_1M@DPCLHLIE@?$AAk?$AAa?$AA?9?$AAG?$AAE@ 10012ae0     libucrt:lcidtoname_downlevel.obj
 0002:00002aec       ??_C@_1M@BLKMHJBI@?$AAf?$AAo?$AA?9?$AAF?$AAO@ 10012aec     libucrt:lcidtoname_downlevel.obj
 0002:00002af8       ??_C@_1M@LGGJAPPB@?$AAh?$AAi?$AA?9?$AAI?$AAN@ 10012af8     libucrt:lcidtoname_downlevel.obj
 0002:00002b04       ??_C@_1M@FIKPIHFE@?$AAm?$AAt?$AA?9?$AAM?$AAT@ 10012b04     libucrt:lcidtoname_downlevel.obj
 0002:00002b10       ??_C@_1M@HEGGPBFA@?$AAs?$AAe?$AA?9?$AAN?$AAO@ 10012b10     libucrt:lcidtoname_downlevel.obj
 0002:00002b1c       ??_C@_1M@EIBJEEPA@?$AAm?$AAs?$AA?9?$AAM?$AAY@ 10012b1c     libucrt:lcidtoname_downlevel.obj
 0002:00002b28       ??_C@_1M@FHLBGMPP@?$AAk?$AAk?$AA?9?$AAK?$AAZ@ 10012b28     libucrt:lcidtoname_downlevel.obj
 0002:00002b34       ??_C@_1M@NGJJLCGI@?$AAk?$AAy?$AA?9?$AAK?$AAG@ 10012b34     libucrt:lcidtoname_downlevel.obj
 0002:00002b40       ??_C@_1M@GIENNBFC@?$AAs?$AAw?$AA?9?$AAK?$AAE@ 10012b40     libucrt:lcidtoname_downlevel.obj
 0002:00002b4c       ??_C@_1BG@NDGMJIMJ@?$AAu?$AAz?$AA?9?$AAU?$AAZ?$AA?9?$AAL?$AAa?$AAt?$AAn@ 10012b4c     libucrt:lcidtoname_downlevel.obj
 0002:00002b64       ??_C@_1M@IDCCIHBC@?$AAt?$AAt?$AA?9?$AAR?$AAU@ 10012b64     libucrt:lcidtoname_downlevel.obj
 0002:00002b70       ??_C@_1M@LOICPMOJ@?$AAb?$AAn?$AA?9?$AAI?$AAN@ 10012b70     libucrt:lcidtoname_downlevel.obj
 0002:00002b7c       ??_C@_1M@KPKKNEAH@?$AAp?$AAa?$AA?9?$AAI?$AAN@ 10012b7c     libucrt:lcidtoname_downlevel.obj
 0002:00002b88       ??_C@_1M@PJGPPBOG@?$AAg?$AAu?$AA?9?$AAI?$AAN@ 10012b88     libucrt:lcidtoname_downlevel.obj
 0002:00002b94       ??_C@_1M@KMKMOPHI@?$AAt?$AAa?$AA?9?$AAI?$AAN@ 10012b94     libucrt:lcidtoname_downlevel.obj
 0002:00002ba0       ??_C@_1M@KFEHEPAC@?$AAt?$AAe?$AA?9?$AAI?$AAN@ 10012ba0     libucrt:lcidtoname_downlevel.obj
 0002:00002bac       ??_C@_1M@CDCLMGHI@?$AAk?$AAn?$AA?9?$AAI?$AAN@ 10012bac     libucrt:lcidtoname_downlevel.obj
 0002:00002bb8       ??_C@_1M@MIODLDKF@?$AAm?$AAl?$AA?9?$AAI?$AAN@ 10012bb8     libucrt:lcidtoname_downlevel.obj
 0002:00002bc4       ??_C@_1M@PBIEACPO@?$AAm?$AAr?$AA?9?$AAI?$AAN@ 10012bc4     libucrt:lcidtoname_downlevel.obj
 0002:00002bd0       ??_C@_1M@NIDEAGPH@?$AAs?$AAa?$AA?9?$AAI?$AAN@ 10012bd0     libucrt:lcidtoname_downlevel.obj
 0002:00002bdc       ??_C@_1M@FHIHCBIO@?$AAm?$AAn?$AA?9?$AAM?$AAN@ 10012bdc     libucrt:lcidtoname_downlevel.obj
 0002:00002be8       ??_C@_1M@JAIJPENP@?$AAc?$AAy?$AA?9?$AAG?$AAB@ 10012be8     libucrt:lcidtoname_downlevel.obj
 0002:00002bf4       ??_C@_1M@PHGFBEPN@?$AAg?$AAl?$AA?9?$AAE?$AAS@ 10012bf4     libucrt:lcidtoname_downlevel.obj
 0002:00002c00       ??_C@_1O@KPIPDNCP@?$AAk?$AAo?$AAk?$AA?9?$AAI?$AAN@ 10012c00     libucrt:lcidtoname_downlevel.obj
 0002:00002c10       ??_C@_1O@KNHJLDJA@?$AAs?$AAy?$AAr?$AA?9?$AAS?$AAY@ 10012c10     libucrt:lcidtoname_downlevel.obj
 0002:00002c20       ??_C@_1O@MKEKBLAH@?$AAd?$AAi?$AAv?$AA?9?$AAM?$AAV@ 10012c20     libucrt:lcidtoname_downlevel.obj
 0002:00002c30       ??_C@_1O@OHDCKDDF@?$AAq?$AAu?$AAz?$AA?9?$AAB?$AAO@ 10012c30     libucrt:lcidtoname_downlevel.obj
 0002:00002c40       ??_C@_1M@LEPJNLFD@?$AAn?$AAs?$AA?9?$AAZ?$AAA@ 10012c40     libucrt:lcidtoname_downlevel.obj
 0002:00002c4c       ??_C@_1M@OMLEIIJB@?$AAm?$AAi?$AA?9?$AAN?$AAZ@ 10012c4c     libucrt:lcidtoname_downlevel.obj
 0002:00002c58       ??_C@_1M@PMPEAILG@?$AAa?$AAr?$AA?9?$AAI?$AAQ@ 10012c58     libucrt:lcidtoname_downlevel.obj
 0002:00002c64       ??_C@_1M@CNKPNOEE@?$AAd?$AAe?$AA?9?$AAC?$AAH@ 10012c64     libucrt:lcidtoname_downlevel.obj
 0002:00002c70       ??_C@_1M@LKMGMLKO@?$AAe?$AAn?$AA?9?$AAG?$AAB@ 10012c70     libucrt:lcidtoname_downlevel.obj
 0002:00002c7c       ??_C@_1M@PGKJFFGL@?$AAe?$AAs?$AA?9?$AAM?$AAX@ 10012c7c     libucrt:lcidtoname_downlevel.obj
 0002:00002c88       ??_C@_1M@DNNANBDC@?$AAf?$AAr?$AA?9?$AAB?$AAE@ 10012c88     libucrt:lcidtoname_downlevel.obj
 0002:00002c94       ??_C@_1M@HLGMDFHM@?$AAi?$AAt?$AA?9?$AAC?$AAH@ 10012c94     libucrt:lcidtoname_downlevel.obj
 0002:00002ca0       ??_C@_1M@CLLBGJH@?$AAn?$AAl?$AA?9?$AAB?$AAE@ 10012ca0     libucrt:lcidtoname_downlevel.obj
 0002:00002cac       ??_C@_1M@BODBOGLF@?$AAn?$AAn?$AA?9?$AAN?$AAO@ 10012cac     libucrt:lcidtoname_downlevel.obj
 0002:00002cb8       ??_C@_1M@HFFAHKAD@?$AAp?$AAt?$AA?9?$AAP?$AAT@ 10012cb8     libucrt:lcidtoname_downlevel.obj
 0002:00002cc4       ??_C@_1BG@LNOAKHIE@?$AAs?$AAr?$AA?9?$AAS?$AAP?$AA?9?$AAL?$AAa?$AAt?$AAn@ 10012cc4     libucrt:lcidtoname_downlevel.obj
 0002:00002cdc       ??_C@_1M@HBMHBGAK@?$AAs?$AAv?$AA?9?$AAF?$AAI@ 10012cdc     libucrt:lcidtoname_downlevel.obj
 0002:00002ce8       ??_C@_1BG@DGCJGJBE@?$AAa?$AAz?$AA?9?$AAA?$AAZ?$AA?9?$AAC?$AAy?$AAr?$AAl@ 10012ce8     libucrt:lcidtoname_downlevel.obj
 0002:00002d00       ??_C@_1M@KEJDAAHB@?$AAs?$AAe?$AA?9?$AAS?$AAE@ 10012d00     libucrt:lcidtoname_downlevel.obj
 0002:00002d0c       ??_C@_1M@HEIBJJAD@?$AAm?$AAs?$AA?9?$AAB?$AAN@ 10012d0c     libucrt:lcidtoname_downlevel.obj
 0002:00002d18       ??_C@_1BG@PBGJMCEM@?$AAu?$AAz?$AA?9?$AAU?$AAZ?$AA?9?$AAC?$AAy?$AAr?$AAl@ 10012d18     libucrt:lcidtoname_downlevel.obj
 0002:00002d30       ??_C@_1O@LAOBCMDF@?$AAq?$AAu?$AAz?$AA?9?$AAE?$AAC@ 10012d30     libucrt:lcidtoname_downlevel.obj
 0002:00002d40       ??_C@_1M@POEEMAIO@?$AAa?$AAr?$AA?9?$AAE?$AAG@ 10012d40     libucrt:lcidtoname_downlevel.obj
 0002:00002d4c       ??_C@_1M@EFAKDEDL@?$AAz?$AAh?$AA?9?$AAH?$AAK@ 10012d4c     libucrt:lcidtoname_downlevel.obj
 0002:00002d58       ??_C@_1M@HKKIJHGI@?$AAd?$AAe?$AA?9?$AAA?$AAT@ 10012d58     libucrt:lcidtoname_downlevel.obj
 0002:00002d64       ??_C@_1M@KBFBEHJF@?$AAe?$AAn?$AA?9?$AAA?$AAU@ 10012d64     libucrt:lcidtoname_downlevel.obj
 0002:00002d70       ??_C@_1M@MNPLFAAH@?$AAe?$AAs?$AA?9?$AAE?$AAS@ 10012d70     libucrt:lcidtoname_downlevel.obj
 0002:00002d7c       ??_C@_1M@HJOOJFMA@?$AAf?$AAr?$AA?9?$AAC?$AAA@ 10012d7c     libucrt:lcidtoname_downlevel.obj
 0002:00002d88       ??_C@_1BG@JPOFPNAB@?$AAs?$AAr?$AA?9?$AAS?$AAP?$AA?9?$AAC?$AAy?$AAr?$AAl@ 10012d88     libucrt:lcidtoname_downlevel.obj
 0002:00002da0       ??_C@_1M@LNFOCMOB@?$AAs?$AAe?$AA?9?$AAF?$AAI@ 10012da0     libucrt:lcidtoname_downlevel.obj
 0002:00002dac       ??_C@_1O@MGJBOAMB@?$AAq?$AAu?$AAz?$AA?9?$AAP?$AAE@ 10012dac     libucrt:lcidtoname_downlevel.obj
 0002:00002dbc       ??_C@_1M@GJINLBOK@?$AAa?$AAr?$AA?9?$AAL?$AAY@ 10012dbc     libucrt:lcidtoname_downlevel.obj
 0002:00002dc8       ??_C@_1M@GGMNHJNL@?$AAz?$AAh?$AA?9?$AAS?$AAG@ 10012dc8     libucrt:lcidtoname_downlevel.obj
 0002:00002dd4       ??_C@_1M@HOIKODND@?$AAd?$AAe?$AA?9?$AAL?$AAU@ 10012dd4     libucrt:lcidtoname_downlevel.obj
 0002:00002de0       ??_C@_1M@DDOCCGFG@?$AAe?$AAn?$AA?9?$AAC?$AAA@ 10012de0     libucrt:lcidtoname_downlevel.obj
 0002:00002dec       ??_C@_1M@BNOEMJLF@?$AAe?$AAs?$AA?9?$AAG?$AAT@ 10012dec     libucrt:lcidtoname_downlevel.obj
 0002:00002df8       ??_C@_1M@EOGNKEK@?$AAf?$AAr?$AA?9?$AAC?$AAH@ 10012df8     libucrt:lcidtoname_downlevel.obj
 0002:00002e04       ??_C@_1M@FLIDJFHL@?$AAh?$AAr?$AA?9?$AAB?$AAA@ 10012e04     libucrt:lcidtoname_downlevel.obj
 0002:00002e10       ??_C@_1O@FMCELNAJ@?$AAs?$AAm?$AAj?$AA?9?$AAN?$AAO@ 10012e10     libucrt:lcidtoname_downlevel.obj
 0002:00002e20       ??_C@_1M@JHGLJMGJ@?$AAa?$AAr?$AA?9?$AAD?$AAZ@ 10012e20     libucrt:lcidtoname_downlevel.obj
 0002:00002e2c       ??_C@_1M@JKKFDCNP@?$AAz?$AAh?$AA?9?$AAM?$AAO@ 10012e2c     libucrt:lcidtoname_downlevel.obj
 0002:00002e38       ??_C@_1M@GEEFALPE@?$AAd?$AAe?$AA?9?$AAL?$AAI@ 10012e38     libucrt:lcidtoname_downlevel.obj
 0002:00002e44       ??_C@_1M@IGEOFBG@?$AAe?$AAn?$AA?9?$AAN?$AAZ@ 10012e44     libucrt:lcidtoname_downlevel.obj
 0002:00002e50       ??_C@_1M@KDBONEHP@?$AAe?$AAs?$AA?9?$AAC?$AAR@ 10012e50     libucrt:lcidtoname_downlevel.obj
 0002:00002e5c       ??_C@_1M@FHMDOHNN@?$AAf?$AAr?$AA?9?$AAL?$AAU@ 10012e5c     libucrt:lcidtoname_downlevel.obj
 0002:00002e68       ??_C@_1BG@NFKKMAFG@?$AAb?$AAs?$AA?9?$AAB?$AAA?$AA?9?$AAL?$AAa?$AAt?$AAn@ 10012e68     libucrt:lcidtoname_downlevel.obj
 0002:00002e80       ??_C@_1O@IMNBEMCI@?$AAs?$AAm?$AAj?$AA?9?$AAS?$AAE@ 10012e80     libucrt:lcidtoname_downlevel.obj
 0002:00002e90       ??_C@_1M@DHHMBNDP@?$AAa?$AAr?$AA?9?$AAM?$AAA@ 10012e90     libucrt:lcidtoname_downlevel.obj
 0002:00002e9c       ??_C@_1M@BNBLJCGH@?$AAe?$AAn?$AA?9?$AAI?$AAE@ 10012e9c     libucrt:lcidtoname_downlevel.obj
 0002:00002ea8       ??_C@_1M@GEPAFMDL@?$AAe?$AAs?$AA?9?$AAP?$AAA@ 10012ea8     libucrt:lcidtoname_downlevel.obj
 0002:00002eb4       ??_C@_1M@OJONDMDL@?$AAf?$AAr?$AA?9?$AAM?$AAC@ 10012eb4     libucrt:lcidtoname_downlevel.obj
 0002:00002ec0       ??_C@_1BG@OBCNFJB@?$AAs?$AAr?$AA?9?$AAB?$AAA?$AA?9?$AAL?$AAa?$AAt?$AAn@ 10012ec0     libucrt:lcidtoname_downlevel.obj
 0002:00002ed8       ??_C@_1O@KEMEEGPO@?$AAs?$AAm?$AAa?$AA?9?$AAN?$AAO@ 10012ed8     libucrt:lcidtoname_downlevel.obj
 0002:00002ee8       ??_C@_1M@ELMGFODK@?$AAa?$AAr?$AA?9?$AAT?$AAN@ 10012ee8     libucrt:lcidtoname_downlevel.obj
 0002:00002ef4       ??_C@_1M@BHDLHFAF@?$AAe?$AAn?$AA?9?$AAZ?$AAA@ 10012ef4     libucrt:lcidtoname_downlevel.obj
 0002:00002f00       ??_C@_1M@BMGIGLIF@?$AAe?$AAs?$AA?9?$AAD?$AAO@ 10012f00     libucrt:lcidtoname_downlevel.obj
 0002:00002f0c       ??_C@_1BG@CMBHIPBE@?$AAs?$AAr?$AA?9?$AAB?$AAA?$AA?9?$AAC?$AAy?$AAr?$AAl@ 10012f0c     libucrt:lcidtoname_downlevel.obj
 0002:00002f24       ??_C@_1O@HEDBLHNP@?$AAs?$AAm?$AAa?$AA?9?$AAS?$AAE@ 10012f24     libucrt:lcidtoname_downlevel.obj
 0002:00002f34       ??_C@_1M@DAGCADIM@?$AAa?$AAr?$AA?9?$AAO?$AAM@ 10012f34     libucrt:lcidtoname_downlevel.obj
 0002:00002f40       ??_C@_1M@FODLMICG@?$AAe?$AAn?$AA?9?$AAJ?$AAM@ 10012f40     libucrt:lcidtoname_downlevel.obj
 0002:00002f4c       ??_C@_1M@DNMLCIHB@?$AAe?$AAs?$AA?9?$AAV?$AAE@ 10012f4c     libucrt:lcidtoname_downlevel.obj
 0002:00002f58       ??_C@_1O@EOKHMKJK@?$AAs?$AAm?$AAs?$AA?9?$AAF?$AAI@ 10012f58     libucrt:lcidtoname_downlevel.obj
 0002:00002f68       ??_C@_1M@CAFJMKOF@?$AAa?$AAr?$AA?9?$AAY?$AAE@ 10012f68     libucrt:lcidtoname_downlevel.obj
 0002:00002f74       ??_C@_1M@CBFHIJLI@?$AAe?$AAn?$AA?9?$AAC?$AAB@ 10012f74     libucrt:lcidtoname_downlevel.obj
 0002:00002f80       ??_C@_1M@BGNFLDN@?$AAe?$AAs?$AA?9?$AAC?$AAO@ 10012f80     libucrt:lcidtoname_downlevel.obj
 0002:00002f8c       ??_C@_1O@JMPHMAMC@?$AAs?$AAm?$AAn?$AA?9?$AAF?$AAI@ 10012f8c     libucrt:lcidtoname_downlevel.obj
 0002:00002f9c       ??_C@_1M@JLANABKE@?$AAa?$AAr?$AA?9?$AAS?$AAY@ 10012f9c     libucrt:lcidtoname_downlevel.obj
 0002:00002fa8       ??_C@_1M@HPKGCFGN@?$AAe?$AAn?$AA?9?$AAB?$AAZ@ 10012fa8     libucrt:lcidtoname_downlevel.obj
 0002:00002fb4       ??_C@_1M@OLJCMLGM@?$AAe?$AAs?$AA?9?$AAP?$AAE@ 10012fb4     libucrt:lcidtoname_downlevel.obj
 0002:00002fc0       ??_C@_1M@MKKGFKLE@?$AAa?$AAr?$AA?9?$AAJ?$AAO@ 10012fc0     libucrt:lcidtoname_downlevel.obj
 0002:00002fcc       ??_C@_1M@EKPGLDNI@?$AAe?$AAn?$AA?9?$AAT?$AAT@ 10012fcc     libucrt:lcidtoname_downlevel.obj
 0002:00002fd8       ??_C@_1M@OONGHFHE@?$AAe?$AAs?$AA?9?$AAA?$AAR@ 10012fd8     libucrt:lcidtoname_downlevel.obj
 0002:00002fe4       ??_C@_1M@OOJFGBHE@?$AAa?$AAr?$AA?9?$AAL?$AAB@ 10012fe4     libucrt:lcidtoname_downlevel.obj
 0002:00002ff0       ??_C@_1M@GCEJHNEG@?$AAe?$AAn?$AA?9?$AAZ?$AAW@ 10012ff0     libucrt:lcidtoname_downlevel.obj
 0002:00002ffc       ??_C@_1M@JNOCAHJI@?$AAe?$AAs?$AA?9?$AAE?$AAC@ 10012ffc     libucrt:lcidtoname_downlevel.obj
 0002:00003008       ??_C@_1M@JEFHPGGB@?$AAa?$AAr?$AA?9?$AAK?$AAW@ 10013008     libucrt:lcidtoname_downlevel.obj
 0002:00003014       ??_C@_1M@MLKIBJOJ@?$AAe?$AAn?$AA?9?$AAP?$AAH@ 10013014     libucrt:lcidtoname_downlevel.obj
 0002:00003020       ??_C@_1M@BDNIPEND@?$AAe?$AAs?$AA?9?$AAC?$AAL@ 10013020     libucrt:lcidtoname_downlevel.obj
 0002:0000302c       ??_C@_1M@MPNMEKBD@?$AAa?$AAr?$AA?9?$AAA?$AAE@ 1001302c     libucrt:lcidtoname_downlevel.obj
 0002:00003038       ??_C@_1M@KBJALCPI@?$AAe?$AAs?$AA?9?$AAU?$AAY@ 10013038     libucrt:lcidtoname_downlevel.obj
 0002:00003044       ??_C@_1M@LLCCOAGA@?$AAa?$AAr?$AA?9?$AAB?$AAH@ 10013044     libucrt:lcidtoname_downlevel.obj
 0002:00003050       ??_C@_1M@PBFNCDEL@?$AAe?$AAs?$AA?9?$AAP?$AAY@ 10013050     libucrt:lcidtoname_downlevel.obj
 0002:0000305c       ??_C@_1M@EDGINPNP@?$AAa?$AAr?$AA?9?$AAQ?$AAA@ 1001305c     libucrt:lcidtoname_downlevel.obj
 0002:00003068       ??_C@_1M@MKDBIIJI@?$AAe?$AAs?$AA?9?$AAB?$AAO@ 10013068     libucrt:lcidtoname_downlevel.obj
 0002:00003074       ??_C@_1M@CPKKEBLD@?$AAe?$AAs?$AA?9?$AAS?$AAV@ 10013074     libucrt:lcidtoname_downlevel.obj
 0002:00003080       ??_C@_1M@NDBGMMJL@?$AAe?$AAs?$AA?9?$AAH?$AAN@ 10013080     libucrt:lcidtoname_downlevel.obj
 0002:0000308c       ??_C@_1M@JIJIBHDP@?$AAe?$AAs?$AA?9?$AAN?$AAI@ 1001308c     libucrt:lcidtoname_downlevel.obj
 0002:00003098       ??_C@_1M@CGFMKEEK@?$AAe?$AAs?$AA?9?$AAP?$AAR@ 10013098     libucrt:lcidtoname_downlevel.obj
 0002:000030a4       ??_C@_1O@ICJHKIIK@?$AAz?$AAh?$AA?9?$AAC?$AAH?$AAT@ 100130a4     libucrt:lcidtoname_downlevel.obj
 0002:000030b4       ??_C@_15CLNEJCE@?$AAs?$AAr@ 100130b4     libucrt:lcidtoname_downlevel.obj
 0002:000037e0       ??_C@_1M@KAHEKEIG@?$AAa?$AAf?$AA?9?$AAz?$AAa@ 100137e0     libucrt:lcidtoname_downlevel.obj
 0002:000037ec       ??_C@_1M@GIECOABL@?$AAa?$AAr?$AA?9?$AAa?$AAe@ 100137ec     libucrt:lcidtoname_downlevel.obj
 0002:000037f8       ??_C@_1M@BMLMEKGI@?$AAa?$AAr?$AA?9?$AAb?$AAh@ 100137f8     libucrt:lcidtoname_downlevel.obj
 0002:00003804       ??_C@_1M@DAPFDGGB@?$AAa?$AAr?$AA?9?$AAd?$AAz@ 10013804     libucrt:lcidtoname_downlevel.obj
 0002:00003810       ??_C@_1M@FJNKGKIG@?$AAa?$AAr?$AA?9?$AAe?$AAg@ 10013810     libucrt:lcidtoname_downlevel.obj
 0002:0000381c       ??_C@_1M@FLGKKCLO@?$AAa?$AAr?$AA?9?$AAi?$AAq@ 1001381c     libucrt:lcidtoname_downlevel.obj
 0002:00003828       ??_C@_1M@GNDIPALM@?$AAa?$AAr?$AA?9?$AAj?$AAo@ 10013828     libucrt:lcidtoname_downlevel.obj
 0002:00003834       ??_C@_1M@DDMJFMGJ@?$AAa?$AAr?$AA?9?$AAk?$AAw@ 10013834     libucrt:lcidtoname_downlevel.obj
 0002:00003840       ??_C@_1M@EJALMLHM@?$AAa?$AAr?$AA?9?$AAl?$AAb@ 10013840     libucrt:lcidtoname_downlevel.obj
 0002:0000384c       ??_C@_1M@MOBDBLOC@?$AAa?$AAr?$AA?9?$AAl?$AAy@ 1001384c     libucrt:lcidtoname_downlevel.obj
 0002:00003858       ??_C@_1M@JAOCLHDH@?$AAa?$AAr?$AA?9?$AAm?$AAa@ 10013858     libucrt:lcidtoname_downlevel.obj
 0002:00003864       ??_C@_1M@JHPMKJIE@?$AAa?$AAr?$AA?9?$AAo?$AAm@ 10013864     libucrt:lcidtoname_downlevel.obj
 0002:00003870       ??_C@_1M@OEPGHFNH@?$AAa?$AAr?$AA?9?$AAq?$AAa@ 10013870     libucrt:lcidtoname_downlevel.obj
 0002:0000387c       ??_C@_1M@KJDONENM@?$AAa?$AAr?$AA?9?$AAs?$AAa@ 1001387c     libucrt:lcidtoname_downlevel.obj
 0002:00003888       ??_C@_1M@DMJDKLKM@?$AAa?$AAr?$AA?9?$AAs?$AAy@ 10013888     libucrt:lcidtoname_downlevel.obj
 0002:00003894       ??_C@_1M@OMFIPEDC@?$AAa?$AAr?$AA?9?$AAt?$AAn@ 10013894     libucrt:lcidtoname_downlevel.obj
 0002:000038a0       ??_C@_1M@IHMHGAON@?$AAa?$AAr?$AA?9?$AAy?$AAe@ 100138a0     libucrt:lcidtoname_downlevel.obj
 0002:000038ac       ??_C@_1BG@KDCPGJGB@?$AAa?$AAz?$AA?9?$AAa?$AAz?$AA?9?$AAc?$AAy?$AAr?$AAl@ 100138ac     libucrt:lcidtoname_downlevel.obj
 0002:000038c4       ??_C@_1BG@IBCKDDOE@?$AAa?$AAz?$AA?9?$AAa?$AAz?$AA?9?$AAl?$AAa?$AAt?$AAn@ 100138c4     libucrt:lcidtoname_downlevel.obj
 0002:000038dc       ??_C@_1M@EGPFDCPD@?$AAb?$AAe?$AA?9?$AAb?$AAy@ 100138dc     libucrt:lcidtoname_downlevel.obj
 0002:000038e8       ??_C@_1M@PCMGMCGC@?$AAb?$AAg?$AA?9?$AAb?$AAg@ 100138e8     libucrt:lcidtoname_downlevel.obj
 0002:000038f4       ??_C@_1M@BJBMFGOB@?$AAb?$AAn?$AA?9?$AAi?$AAn@ 100138f4     libucrt:lcidtoname_downlevel.obj
 0002:00003900       ??_C@_1BG@EAKMMACD@?$AAb?$AAs?$AA?9?$AAb?$AAa?$AA?9?$AAl?$AAa?$AAt?$AAn@ 10013900     libucrt:lcidtoname_downlevel.obj
 0002:00003918       ??_C@_1M@KGADAODK@?$AAc?$AAa?$AA?9?$AAe?$AAs@ 10013918     libucrt:lcidtoname_downlevel.obj
 0002:00003924       ??_C@_1M@COAJPDHI@?$AAc?$AAs?$AA?9?$AAc?$AAz@ 10013924     libucrt:lcidtoname_downlevel.obj
 0002:00003930       ??_C@_1M@DHBHFONH@?$AAc?$AAy?$AA?9?$AAg?$AAb@ 10013930     libucrt:lcidtoname_downlevel.obj
 0002:0000393c       ??_C@_1M@IMGKELGA@?$AAd?$AAa?$AA?9?$AAd?$AAk@ 1001393c     libucrt:lcidtoname_downlevel.obj
 0002:00003948       ??_C@_1M@NNDGDNGA@?$AAd?$AAe?$AA?9?$AAa?$AAt@ 10013948     libucrt:lcidtoname_downlevel.obj
 0002:00003954       ??_C@_1M@IKDBHEEM@?$AAd?$AAe?$AA?9?$AAc?$AAh@ 10013954     libucrt:lcidtoname_downlevel.obj
 0002:00003960       ??_C@_1M@GFFOJMCJ@?$AAd?$AAe?$AA?9?$AAd?$AAe@ 10013960     libucrt:lcidtoname_downlevel.obj
 0002:0000396c       ??_C@_1M@MDNLKBPM@?$AAd?$AAe?$AA?9?$AAl?$AAi@ 1001396c     libucrt:lcidtoname_downlevel.obj
 0002:00003978       ??_C@_1M@NJBEEJNL@?$AAd?$AAe?$AA?9?$AAl?$AAu@ 10013978     libucrt:lcidtoname_downlevel.obj
 0002:00003984       ??_C@_1O@GNNELBAP@?$AAd?$AAi?$AAv?$AA?9?$AAm?$AAv@ 10013984     libucrt:lcidtoname_downlevel.obj
 0002:00003994       ??_C@_1M@EJLEOGAE@?$AAe?$AAl?$AA?9?$AAg?$AAr@ 10013994     libucrt:lcidtoname_downlevel.obj
 0002:000039a0       ??_C@_1M@GMPONJN@?$AAe?$AAn?$AA?9?$AAa?$AAu@ 100139a0     libucrt:lcidtoname_downlevel.obj
 0002:000039ac       ??_C@_1M@NIDIIPGF@?$AAe?$AAn?$AA?9?$AAb?$AAz@ 100139ac     libucrt:lcidtoname_downlevel.obj
 0002:000039b8       ??_C@_1M@JEHMIMFO@?$AAe?$AAn?$AA?9?$AAc?$AAa@ 100139b8     libucrt:lcidtoname_downlevel.obj
 0002:000039c4       ??_C@_1M@IGMJCDLA@?$AAe?$AAn?$AA?9?$AAc?$AAb@ 100139c4     libucrt:lcidtoname_downlevel.obj
 0002:000039d0       ??_C@_1M@BNFIGBKG@?$AAe?$AAn?$AA?9?$AAg?$AAb@ 100139d0     libucrt:lcidtoname_downlevel.obj
 0002:000039dc       ??_C@_1M@LKIFDIGP@?$AAe?$AAn?$AA?9?$AAi?$AAe@ 100139dc     libucrt:lcidtoname_downlevel.obj
 0002:000039e8       ??_C@_1M@PJKFGCCO@?$AAe?$AAn?$AA?9?$AAj?$AAm@ 100139e8     libucrt:lcidtoname_downlevel.obj
 0002:000039f4       ??_C@_1M@KPPKEPBO@?$AAe?$AAn?$AA?9?$AAn?$AAz@ 100139f4     libucrt:lcidtoname_downlevel.obj
 0002:00003a00       ??_C@_1M@GMDGLDOB@?$AAe?$AAn?$AA?9?$AAp?$AAh@ 10013a00     libucrt:lcidtoname_downlevel.obj
 0002:00003a0c       ??_C@_1M@ONGIBJNA@?$AAe?$AAn?$AA?9?$AAt?$AAt@ 10013a0c     libucrt:lcidtoname_downlevel.obj
 0002:00003a18       ??_C@_1M@LLODPCMM@?$AAe?$AAn?$AA?9?$AAu?$AAs@ 10013a18     libucrt:lcidtoname_downlevel.obj
 0002:00003a24       ??_C@_1M@LAKFNPAN@?$AAe?$AAn?$AA?9?$AAz?$AAa@ 10013a24     libucrt:lcidtoname_downlevel.obj
 0002:00003a30       ??_C@_1M@MFNHNHEO@?$AAe?$AAn?$AA?9?$AAz?$AAw@ 10013a30     libucrt:lcidtoname_downlevel.obj
 0002:00003a3c       ??_C@_1M@EJEINPHM@?$AAe?$AAs?$AA?9?$AAa?$AAr@ 10013a3c     libucrt:lcidtoname_downlevel.obj
 0002:00003a48       ??_C@_1M@GNKPCCJA@?$AAe?$AAs?$AA?9?$AAb?$AAo@ 10013a48     libucrt:lcidtoname_downlevel.obj
 0002:00003a54       ??_C@_1M@LEEGFONL@?$AAe?$AAs?$AA?9?$AAc?$AAl@ 10013a54     libucrt:lcidtoname_downlevel.obj
 0002:00003a60       ??_C@_1M@KGPDPBDF@?$AAe?$AAs?$AA?9?$AAc?$AAo@ 10013a60     libucrt:lcidtoname_downlevel.obj
 0002:00003a6c       ??_C@_1M@EIAHOHH@?$AAe?$AAs?$AA?9?$AAc?$AAr@ 10013a6c     libucrt:lcidtoname_downlevel.obj
 0002:00003a78       ??_C@_1M@LLPGMBIN@?$AAe?$AAs?$AA?9?$AAd?$AAo@ 10013a78     libucrt:lcidtoname_downlevel.obj
 0002:00003a84       ??_C@_1M@DKHMKNJA@?$AAe?$AAs?$AA?9?$AAe?$AAc@ 10013a84     libucrt:lcidtoname_downlevel.obj
 0002:00003a90       ??_C@_1M@GKGFPKAP@?$AAe?$AAs?$AA?9?$AAe?$AAs@ 10013a90     libucrt:lcidtoname_downlevel.obj
 0002:00003a9c       ??_C@_1M@LKHKGDLN@?$AAe?$AAs?$AA?9?$AAg?$AAt@ 10013a9c     libucrt:lcidtoname_downlevel.obj
 0002:00003aa8       ??_C@_1M@HEIIGGJD@?$AAe?$AAs?$AA?9?$AAh?$AAn@ 10013aa8     libucrt:lcidtoname_downlevel.obj
 0002:00003ab4       ??_C@_1M@FBDHPPGD@?$AAe?$AAs?$AA?9?$AAm?$AAx@ 10013ab4     libucrt:lcidtoname_downlevel.obj
 0002:00003ac0       ??_C@_1M@DPAGLNDH@?$AAe?$AAs?$AA?9?$AAn?$AAi@ 10013ac0     libucrt:lcidtoname_downlevel.obj
 0002:00003acc       ??_C@_1M@MDGOPGDD@?$AAe?$AAs?$AA?9?$AAp?$AAa@ 10013acc     libucrt:lcidtoname_downlevel.obj
 0002:00003ad8       ??_C@_1M@EMAMGBGE@?$AAe?$AAs?$AA?9?$AAp?$AAe@ 10013ad8     libucrt:lcidtoname_downlevel.obj
 0002:00003ae4       ??_C@_1M@IBMCAOEC@?$AAe?$AAs?$AA?9?$AAp?$AAr@ 10013ae4     libucrt:lcidtoname_downlevel.obj
 0002:00003af0       ??_C@_1M@FGMDIJED@?$AAe?$AAs?$AA?9?$AAp?$AAy@ 10013af0     libucrt:lcidtoname_downlevel.obj
 0002:00003afc       ??_C@_1M@IIDEOLLL@?$AAe?$AAs?$AA?9?$AAs?$AAv@ 10013afc     libucrt:lcidtoname_downlevel.obj
 0002:00003b08       ??_C@_1M@GAOBIPA@?$AAe?$AAs?$AA?9?$AAu?$AAy@ 10013b08     libucrt:lcidtoname_downlevel.obj
 0002:00003b14       ??_C@_1M@JKFFICHJ@?$AAe?$AAs?$AA?9?$AAv?$AAe@ 10013b14     libucrt:lcidtoname_downlevel.obj
 0002:00003b20       ??_C@_1M@PNMLOJDF@?$AAe?$AAt?$AA?9?$AAe?$AAe@ 10013b20     libucrt:lcidtoname_downlevel.obj
 0002:00003b2c       ??_C@_1M@GHHLIKEI@?$AAe?$AAu?$AA?9?$AAe?$AAs@ 10013b2c     libucrt:lcidtoname_downlevel.obj
 0002:00003b38       ??_C@_1M@PBNONODE@?$AAf?$AAa?$AA?9?$AAi?$AAr@ 10013b38     libucrt:lcidtoname_downlevel.obj
 0002:00003b44       ??_C@_1M@JEEHPMIL@?$AAf?$AAi?$AA?9?$AAf?$AAi@ 10013b44     libucrt:lcidtoname_downlevel.obj
 0002:00003b50       ??_C@_1M@LMDCNDBA@?$AAf?$AAo?$AA?9?$AAf?$AAo@ 10013b50     libucrt:lcidtoname_downlevel.obj
 0002:00003b5c       ??_C@_1M@JKEOHLDK@?$AAf?$AAr?$AA?9?$AAb?$AAe@ 10013b5c     libucrt:lcidtoname_downlevel.obj
 0002:00003b68       ??_C@_1M@NOHADPMI@?$AAf?$AAr?$AA?9?$AAc?$AAa@ 10013b68     libucrt:lcidtoname_downlevel.obj
 0002:00003b74       ??_C@_1M@KDHIHAEC@?$AAf?$AAr?$AA?9?$AAc?$AAh@ 10013b74     libucrt:lcidtoname_downlevel.obj
 0002:00003b80       ??_C@_1M@MMBBFGAK@?$AAf?$AAr?$AA?9?$AAf?$AAr@ 10013b80     libucrt:lcidtoname_downlevel.obj
 0002:00003b8c       ??_C@_1M@PAFNENNF@?$AAf?$AAr?$AA?9?$AAl?$AAu@ 10013b8c     libucrt:lcidtoname_downlevel.obj
 0002:00003b98       ??_C@_1M@EOHDJGDD@?$AAf?$AAr?$AA?9?$AAm?$AAc@ 10013b98     libucrt:lcidtoname_downlevel.obj
 0002:00003ba4       ??_C@_1M@FAPLLOPF@?$AAg?$AAl?$AA?9?$AAe?$AAs@ 10013ba4     libucrt:lcidtoname_downlevel.obj
 0002:00003bb0       ??_C@_1M@FOPBFLOO@?$AAg?$AAu?$AA?9?$AAi?$AAn@ 10013bb0     libucrt:lcidtoname_downlevel.obj
 0002:00003bbc       ??_C@_1M@KBMCINPM@?$AAh?$AAe?$AA?9?$AAi?$AAl@ 10013bbc     libucrt:lcidtoname_downlevel.obj
 0002:00003bc8       ??_C@_1M@BBPHKFPJ@?$AAh?$AAi?$AA?9?$AAi?$AAn@ 10013bc8     libucrt:lcidtoname_downlevel.obj
 0002:00003bd4       ??_C@_1M@PMBNDPHD@?$AAh?$AAr?$AA?9?$AAb?$AAa@ 10013bd4     libucrt:lcidtoname_downlevel.obj
 0002:00003be0       ??_C@_1M@BPCKOEGE@?$AAh?$AAr?$AA?9?$AAh?$AAr@ 10013be0     libucrt:lcidtoname_downlevel.obj
 0002:00003bec       ??_C@_1M@GACBMHKE@?$AAh?$AAu?$AA?9?$AAh?$AAu@ 10013bec     libucrt:lcidtoname_downlevel.obj
 0002:00003bf8       ??_C@_1M@MILPAJJC@?$AAh?$AAy?$AA?9?$AAa?$AAm@ 10013bf8     libucrt:lcidtoname_downlevel.obj
 0002:00003c04       ??_C@_1M@BABBICEC@?$AAi?$AAd?$AA?9?$AAi?$AAd@ 10013c04     libucrt:lcidtoname_downlevel.obj
 0002:00003c10       ??_C@_1M@BIKNHHPF@?$AAi?$AAs?$AA?9?$AAi?$AAs@ 10013c10     libucrt:lcidtoname_downlevel.obj
 0002:00003c1c       ??_C@_1M@NMPCJPHE@?$AAi?$AAt?$AA?9?$AAc?$AAh@ 10013c1c     libucrt:lcidtoname_downlevel.obj
 0002:00003c28       ??_C@_1M@GHKGFEDF@?$AAi?$AAt?$AA?9?$AAi?$AAt@ 10013c28     libucrt:lcidtoname_downlevel.obj
 0002:00003c34       ??_C@_1M@NIEJCJJA@?$AAj?$AAa?$AA?9?$AAj?$AAp@ 10013c34     libucrt:lcidtoname_downlevel.obj
 0002:00003c40       ??_C@_1M@JILFNBIM@?$AAk?$AAa?$AA?9?$AAg?$AAe@ 10013c40     libucrt:lcidtoname_downlevel.obj
 0002:00003c4c       ??_C@_1M@PACPMGPH@?$AAk?$AAk?$AA?9?$AAk?$AAz@ 10013c4c     libucrt:lcidtoname_downlevel.obj
 0002:00003c58       ??_C@_1M@IELFGMHA@?$AAk?$AAn?$AA?9?$AAi?$AAn@ 10013c58     libucrt:lcidtoname_downlevel.obj
 0002:00003c64       ??_C@_1O@IBBJHCH@?$AAk?$AAo?$AAk?$AA?9?$AAi?$AAn@ 10013c64     libucrt:lcidtoname_downlevel.obj
 0002:00003c74       ??_C@_1M@DMHAEOGC@?$AAk?$AAo?$AA?9?$AAk?$AAr@ 10013c74     libucrt:lcidtoname_downlevel.obj
 0002:00003c80       ??_C@_1M@HBAHBIGA@?$AAk?$AAy?$AA?9?$AAk?$AAg@ 10013c80     libucrt:lcidtoname_downlevel.obj
 0002:00003c8c       ??_C@_1M@KPMILCJG@?$AAl?$AAt?$AA?9?$AAl?$AAt@ 10013c8c     libucrt:lcidtoname_downlevel.obj
 0002:00003c98       ??_C@_1M@BDEKKCA@?$AAl?$AAv?$AA?9?$AAl?$AAv@ 10013c98     libucrt:lcidtoname_downlevel.obj
 0002:00003ca4       ??_C@_1M@ELCKCCJJ@?$AAm?$AAi?$AA?9?$AAn?$AAz@ 10013ca4     libucrt:lcidtoname_downlevel.obj
 0002:00003cb0       ??_C@_1M@CBOOLAPA@?$AAm?$AAk?$AA?9?$AAm?$AAk@ 10013cb0     libucrt:lcidtoname_downlevel.obj
 0002:00003cbc       ??_C@_1M@GPHNBJKN@?$AAm?$AAl?$AA?9?$AAi?$AAn@ 10013cbc     libucrt:lcidtoname_downlevel.obj
 0002:00003cc8       ??_C@_1M@PABJILIG@?$AAm?$AAn?$AA?9?$AAm?$AAn@ 10013cc8     libucrt:lcidtoname_downlevel.obj
 0002:00003cd4       ??_C@_1M@FGBKKIPG@?$AAm?$AAr?$AA?9?$AAi?$AAn@ 10013cd4     libucrt:lcidtoname_downlevel.obj
 0002:00003ce0       ??_C@_1M@NDBPDDAL@?$AAm?$AAs?$AA?9?$AAb?$AAn@ 10013ce0     libucrt:lcidtoname_downlevel.obj
 0002:00003cec       ??_C@_1M@OPIHOOPI@?$AAm?$AAs?$AA?9?$AAm?$AAy@ 10013cec     libucrt:lcidtoname_downlevel.obj
 0002:00003cf8       ??_C@_1M@PPDBCNFM@?$AAm?$AAt?$AA?9?$AAm?$AAt@ 10013cf8     libucrt:lcidtoname_downlevel.obj
 0002:00003d04       ??_C@_1M@KDJDKMDD@?$AAn?$AAb?$AA?9?$AAn?$AAo@ 10013d04     libucrt:lcidtoname_downlevel.obj
 0002:00003d10       ??_C@_1M@KFCFLMJP@?$AAn?$AAl?$AA?9?$AAb?$AAe@ 10013d10     libucrt:lcidtoname_downlevel.obj
 0002:00003d1c       ??_C@_1M@KPOPDDGO@?$AAn?$AAl?$AA?9?$AAn?$AAl@ 10013d1c     libucrt:lcidtoname_downlevel.obj
 0002:00003d28       ??_C@_1M@LJKPEMLN@?$AAn?$AAn?$AA?9?$AAn?$AAo@ 10013d28     libucrt:lcidtoname_downlevel.obj
 0002:00003d34       ??_C@_1M@BDGHHBFL@?$AAn?$AAs?$AA?9?$AAz?$AAa@ 10013d34     libucrt:lcidtoname_downlevel.obj
 0002:00003d40       ??_C@_1M@IDEHOAP@?$AAp?$AAa?$AA?9?$AAi?$AAn@ 10013d40     libucrt:lcidtoname_downlevel.obj
 0002:00003d4c       ??_C@_1M@HDBKGOGH@?$AAp?$AAl?$AA?9?$AAp?$AAl@ 10013d4c     libucrt:lcidtoname_downlevel.obj
 0002:00003d58       ??_C@_1M@LJLLCMEH@?$AAp?$AAt?$AA?9?$AAb?$AAr@ 10013d58     libucrt:lcidtoname_downlevel.obj
 0002:00003d64       ??_C@_1M@NCMONAAL@?$AAp?$AAt?$AA?9?$AAp?$AAt@ 10013d64     libucrt:lcidtoname_downlevel.obj
 0002:00003d70       ??_C@_1O@EAKMAJDN@?$AAq?$AAu?$AAz?$AA?9?$AAb?$AAo@ 10013d70     libucrt:lcidtoname_downlevel.obj
 0002:00003d80       ??_C@_1O@BHHPIGDN@?$AAq?$AAu?$AAz?$AA?9?$AAe?$AAc@ 10013d80     libucrt:lcidtoname_downlevel.obj
 0002:00003d90       ??_C@_1O@GBAPEKMJ@?$AAq?$AAu?$AAz?$AA?9?$AAp?$AAe@ 10013d90     libucrt:lcidtoname_downlevel.obj
 0002:00003da0       ??_C@_1M@CLGLEFBO@?$AAr?$AAo?$AA?9?$AAr?$AAo@ 10013da0     libucrt:lcidtoname_downlevel.obj
 0002:00003dac       ??_C@_1M@CEEDODME@?$AAr?$AAu?$AA?9?$AAr?$AAu@ 10013dac     libucrt:lcidtoname_downlevel.obj
 0002:00003db8       ??_C@_1M@HPKKKMPP@?$AAs?$AAa?$AA?9?$AAi?$AAn@ 10013db8     libucrt:lcidtoname_downlevel.obj
 0002:00003dc4       ??_C@_1M@BKMAIGOJ@?$AAs?$AAe?$AA?9?$AAf?$AAi@ 10013dc4     libucrt:lcidtoname_downlevel.obj
 0002:00003dd0       ??_C@_1M@NDPIFLFI@?$AAs?$AAe?$AA?9?$AAn?$AAo@ 10013dd0     libucrt:lcidtoname_downlevel.obj
 0002:00003ddc       ??_C@_1M@DANKKHJ@?$AAs?$AAe?$AA?9?$AAs?$AAe@ 10013ddc     libucrt:lcidtoname_downlevel.obj
 0002:00003de8       ??_C@_1M@PNBLONPJ@?$AAs?$AAk?$AA?9?$AAs?$AAk@ 10013de8     libucrt:lcidtoname_downlevel.obj
 0002:00003df4       ??_C@_1M@LFMODOAL@?$AAs?$AAl?$AA?9?$AAs?$AAi@ 10013df4     libucrt:lcidtoname_downlevel.obj
 0002:00003e00       ??_C@_1O@DFKOMPG@?$AAs?$AAm?$AAa?$AA?9?$AAn?$AAo@ 10013e00     libucrt:lcidtoname_downlevel.obj
 0002:00003e10       ??_C@_1O@NDKPBNNH@?$AAs?$AAm?$AAa?$AA?9?$AAs?$AAe@ 10013e10     libucrt:lcidtoname_downlevel.obj
 0002:00003e20       ??_C@_1O@PLLKBHAB@?$AAs?$AAm?$AAj?$AA?9?$AAn?$AAo@ 10013e20     libucrt:lcidtoname_downlevel.obj
 0002:00003e30       ??_C@_1O@CLEPOGCA@?$AAs?$AAm?$AAj?$AA?9?$AAs?$AAe@ 10013e30     libucrt:lcidtoname_downlevel.obj
 0002:00003e40       ??_C@_1O@DLGJGKMK@?$AAs?$AAm?$AAn?$AA?9?$AAf?$AAi@ 10013e40     libucrt:lcidtoname_downlevel.obj
 0002:00003e50       ??_C@_1O@OJDJGAJC@?$AAs?$AAm?$AAs?$AA?9?$AAf?$AAi@ 10013e50     libucrt:lcidtoname_downlevel.obj
 0002:00003e60       ??_C@_1M@BOFOGHPB@?$AAs?$AAq?$AA?9?$AAa?$AAl@ 10013e60     libucrt:lcidtoname_downlevel.obj
 0002:00003e6c       ??_C@_1BG@LJBBIPGB@?$AAs?$AAr?$AA?9?$AAb?$AAa?$AA?9?$AAc?$AAy?$AAr?$AAl@ 10013e6c     libucrt:lcidtoname_downlevel.obj
 0002:00003e84       ??_C@_1BG@JLBENFOE@?$AAs?$AAr?$AA?9?$AAb?$AAa?$AA?9?$AAl?$AAa?$AAt?$AAn@ 10013e84     libucrt:lcidtoname_downlevel.obj
 0002:00003e9c       ??_C@_1BG@KODPNHE@?$AAs?$AAr?$AA?9?$AAs?$AAp?$AA?9?$AAc?$AAy?$AAr?$AAl@ 10013e9c     libucrt:lcidtoname_downlevel.obj
 0002:00003eb4       ??_C@_1BG@CIOGKHPB@?$AAs?$AAr?$AA?9?$AAs?$AAp?$AA?9?$AAl?$AAa?$AAt?$AAn@ 10013eb4     libucrt:lcidtoname_downlevel.obj
 0002:00003ecc       ??_C@_1M@NGFJLMAC@?$AAs?$AAv?$AA?9?$AAf?$AAi@ 10013ecc     libucrt:lcidtoname_downlevel.obj
 0002:00003ed8       ??_C@_1M@MPJEJAJC@?$AAs?$AAv?$AA?9?$AAs?$AAe@ 10013ed8     libucrt:lcidtoname_downlevel.obj
 0002:00003ee4       ??_C@_1M@MPNDHLFK@?$AAs?$AAw?$AA?9?$AAk?$AAe@ 10013ee4     libucrt:lcidtoname_downlevel.obj
 0002:00003ef0       ??_C@_1O@KOHBJJI@?$AAs?$AAy?$AAr?$AA?9?$AAs?$AAy@ 10013ef0     libucrt:lcidtoname_downlevel.obj
 0002:00003f00       ??_C@_1M@LDCEFHA@?$AAt?$AAa?$AA?9?$AAi?$AAn@ 10013f00     libucrt:lcidtoname_downlevel.obj
 0002:00003f0c       ??_C@_1M@CNJOFAK@?$AAt?$AAe?$AA?9?$AAi?$AAn@ 10013f0c     libucrt:lcidtoname_downlevel.obj
 0002:00003f18       ??_C@_1M@GNAECACD@?$AAt?$AAh?$AA?9?$AAt?$AAh@ 10013f18     libucrt:lcidtoname_downlevel.obj
 0002:00003f24       ??_C@_1M@CHBIHOJO@?$AAt?$AAn?$AA?9?$AAz?$AAa@ 10013f24     libucrt:lcidtoname_downlevel.obj
 0002:00003f30       ??_C@_1M@GCCMIGPJ@?$AAt?$AAr?$AA?9?$AAt?$AAr@ 10013f30     libucrt:lcidtoname_downlevel.obj
 0002:00003f3c       ??_C@_1M@CELMCNBK@?$AAt?$AAt?$AA?9?$AAr?$AAu@ 10013f3c     libucrt:lcidtoname_downlevel.obj
 0002:00003f48       ??_C@_1M@KLMCELGA@?$AAu?$AAk?$AA?9?$AAu?$AAa@ 10013f48     libucrt:lcidtoname_downlevel.obj
 0002:00003f54       ??_C@_1M@EPAJJAJF@?$AAu?$AAr?$AA?9?$AAp?$AAk@ 10013f54     libucrt:lcidtoname_downlevel.obj
 0002:00003f60       ??_C@_1BG@GEGPMCDJ@?$AAu?$AAz?$AA?9?$AAu?$AAz?$AA?9?$AAc?$AAy?$AAr?$AAl@ 10013f60     libucrt:lcidtoname_downlevel.obj
 0002:00003f78       ??_C@_1BG@EGGKJILM@?$AAu?$AAz?$AA?9?$AAu?$AAz?$AA?9?$AAl?$AAa?$AAt?$AAn@ 10013f78     libucrt:lcidtoname_downlevel.obj
 0002:00003f90       ??_C@_1M@GFOCLFF@?$AAv?$AAi?$AA?9?$AAv?$AAn@ 10013f90     libucrt:lcidtoname_downlevel.obj
 0002:00003f9c       ??_C@_1M@CPAMEDFI@?$AAx?$AAh?$AA?9?$AAz?$AAa@ 10013f9c     libucrt:lcidtoname_downlevel.obj
 0002:00003fa8       ??_C@_1O@EBKIFIGN@?$AAz?$AAh?$AA?9?$AAc?$AAh?$AAs@ 10013fa8     libucrt:lcidtoname_downlevel.obj
 0002:00003fb8       ??_C@_1O@NMHPGANE@?$AAz?$AAh?$AA?9?$AAc?$AAh?$AAt@ 10013fb8     libucrt:lcidtoname_downlevel.obj
 0002:00003fc8       ??_C@_1M@LPINJOMC@?$AAz?$AAh?$AA?9?$AAc?$AAn@ 10013fc8     libucrt:lcidtoname_downlevel.obj
 0002:00003fd4       ??_C@_1M@OCJEJODD@?$AAz?$AAh?$AA?9?$AAh?$AAk@ 10013fd4     libucrt:lcidtoname_downlevel.obj
 0002:00003fe0       ??_C@_1M@DNDLJINH@?$AAz?$AAh?$AA?9?$AAm?$AAo@ 10013fe0     libucrt:lcidtoname_downlevel.obj
 0002:00003fec       ??_C@_1M@MBFDNDND@?$AAz?$AAh?$AA?9?$AAs?$AAg@ 10013fec     libucrt:lcidtoname_downlevel.obj
 0002:00003ff8       ??_C@_1M@IMEPLEPE@?$AAz?$AAh?$AA?9?$AAt?$AAw@ 10013ff8     libucrt:lcidtoname_downlevel.obj
 0002:00004004       ??_C@_1M@BBGHNHJP@?$AAz?$AAu?$AA?9?$AAz?$AAa@ 10014004     libucrt:lcidtoname_downlevel.obj
 0002:00004068       ??_C@_1BA@BALFACEM@?$AAC?$AAO?$AAN?$AAO?$AAU?$AAT?$AA$@ 10014068     libucrt:initcon.obj
 0002:00004180       __infinity                 10014180     libucrt:87tran.obj
 0002:0000418a       __minfinity                1001418a     libucrt:87tran.obj
 0002:00004194       __logemax                  10014194     libucrt:87tran.obj
 0002:000041ba       __OP_EXPjmptab             100141ba     libucrt:87tran.obj
 0002:000041e0       __indefinite               100141e0     libucrt:87disp.obj
 0002:000041ea       __piby2                    100141ea     libucrt:87disp.obj
 0002:000041f4       __piby4                    100141f4     libucrt:87disp.obj
 0002:00004228       __DEFAULT_CW_in_mem        10014228     libucrt:common.obj
 0002:0000422a       __pi_by_2_to_61            1001422a     libucrt:common.obj
 0002:00004264       ??_C@_03MGHMBJCF@log@      10014264     libucrt:libm_error.obj
 0002:00004268       ??_C@_05HGHHAHAP@log10@    10014268     libucrt:libm_error.obj
 0002:00004270       ??_C@_03KHJOGHMM@exp@      10014270     libucrt:libm_error.obj
 0002:00004274       ??_C@_03JGHBODFD@pow@      10014274     libucrt:libm_error.obj
 0002:00004278       ??_C@_04FIHNOPOL@asin@     10014278     libucrt:libm_error.obj
 0002:00004280       ??_C@_04PDIFKINK@acos@     10014280     libucrt:libm_error.obj
 0002:00004288       ??_C@_04EIAKFFMI@sqrt@     10014288     libucrt:libm_error.obj
 0002:00004290       __real@3ff0000000000000    10014290     libucrt:libm_error.obj
 0002:000042b0       ___acrt_log10_table_t      100142b0     libucrt:log10_tables.obj
 0002:000046c0       ___acrt_log10_table_cb     100146c0     libucrt:log10_tables.obj
 0002:00004ad0       __real@3fe0000000000000    10014ad0     libucrt:powhlp.obj
 0002:00004bc0       ??_C@_04COOMCNPB@sinh@     10014bc0     libucrt:fpexcept.obj
 0002:00004bc8       ??_C@_04HPJJNFIM@cosh@     10014bc8     libucrt:fpexcept.obj
 0002:00004bd0       ??_C@_04FJHINJAO@tanh@     10014bd0     libucrt:fpexcept.obj
 0002:00004bd8       ??_C@_04MLLJIGOK@atan@     10014bd8     libucrt:fpexcept.obj
 0002:00004be0       ??_C@_05KNGEOGJB@atan2@    10014be0     libucrt:fpexcept.obj
 0002:00004be8       ??_C@_03BLEJJJBH@sin@      10014be8     libucrt:fpexcept.obj
 0002:00004bec       ??_C@_03LALBNOCG@cos@      10014bec     libucrt:fpexcept.obj
 0002:00004bf0       ??_C@_03IIINPABG@tan@      10014bf0     libucrt:fpexcept.obj
 0002:00004bf4       ??_C@_04GFPJNGEK@ceil@     10014bf4     libucrt:fpexcept.obj
 0002:00004bfc       ??_C@_05PBJFFIGL@floor@    10014bfc     libucrt:fpexcept.obj
 0002:00004c04       ??_C@_04ODHECPBC@fabs@     10014c04     libucrt:fpexcept.obj
 0002:00004c0c       ??_C@_04EHEDPDJG@modf@     10014c0c     libucrt:fpexcept.obj
 0002:00004c14       ??_C@_05CEJMAHNP@ldexp@    10014c14     libucrt:fpexcept.obj
 0002:00004c1c       ??_C@_05KBKMEMPO@_cabs@    10014c1c     libucrt:fpexcept.obj
 0002:00004c24       ??_C@_06MEIMCGCF@_hypot@   10014c24     libucrt:fpexcept.obj
 0002:00004c2c       ??_C@_04KEPJIHGP@fmod@     10014c2c     libucrt:fpexcept.obj
 0002:00004c34       ??_C@_05GKKHEGJL@frexp@    10014c34     libucrt:fpexcept.obj
 0002:00004c3c       ??_C@_03MJLDFKDL@_y0@      10014c3c     libucrt:fpexcept.obj
 0002:00004c40       ??_C@_03NAKIGLHK@_y1@      10014c40     libucrt:fpexcept.obj
 0002:00004c44       ??_C@_03ONILCKOB@_yn@      10014c44     libucrt:fpexcept.obj
 0002:00004c48       ??_C@_05JGDBENOH@_logb@    10014c48     libucrt:fpexcept.obj
 0002:00004c50       ??_C@_0L@KDOEJCKC@_nextafter@ 10014c50     libucrt:fpexcept.obj
 0002:00004c60       __d_inf                    10014c60     libucrt:util.obj
 0002:00004c68       __d_max                    10014c68     libucrt:util.obj
 0002:00004c70       __d_mzero                  10014c70     libucrt:util.obj
 0002:00004c8c       ??_C@_0BC@EOODALEL@Unknown?5exception@ 10014c8c     HlfViewer.obj
 0002:00004ca0       ??_C@_0BF@KINCDENJ@bad?5array?5new?5length@ 10014ca0     HlfViewer.obj
 0002:00004cb8       ??_C@_0BA@JFNIOLAK@string?5too?5long@ 10014cb8     HlfViewer.obj
 0002:00004cc8       ??_C@_11LOCGONAA@@         10014cc8     HlfViewer.obj
 0002:00004ccc       ??_C@_1BE@KLINDABO@?$AAH?$AAl?$AAf?$AAV?$AAi?$AAe?$AAw?$AAe?$AAr@ 10014ccc     HlfViewer.obj
 0002:00004ce0       ??_C@_1EA@CONHECGE@?$AAH?$AAl?$AAf?$AA?9?$AAf?$AAi?$AAl?$AAe?$AA?5?$AAV?$AAi?$AAe?$AAw?$AAe?$AAr@ 10014ce0     HlfViewer.obj
 0002:00004d20       ??_C@_1DE@BGKMIKPD@?$AAE?$AAu?$AAg?$AAe?$AAn?$AAe?$AA?5?$AAR?$AAo?$AAs?$AAh?$AAa?$AAl?$AA?5?$AA?$CG@ 10014d20     HlfViewer.obj
 0002:00004d54       ??_C@_13FPGAJAPJ@?$AA?2@   10014d54     HlfViewer.obj
 0002:00004d58       ??_C@_1BE@BAOBMOBE@?$AA?$CF?$AAF?$AAA?$AAR?$AAH?$AAO?$AAM?$AAE?$AA?$CF@ 10014d58     HlfViewer.obj
 0002:00004d6c       ??_C@_17MEJHPLBO@?$AAc?$AAm?$AAd@ 10014d6c     HlfViewer.obj
 0002:00004d74       ??_C@_17KGEADEDI@?$AAH?$AAL?$AAF@ 10014d74     HlfViewer.obj
 0002:00004d7c       ??_C@_19CPJEHIBK@?$AA?4?$AAh?$AAl?$AAf@ 10014d7c     HlfViewer.obj
 0002:00004d88       ??_C@_15JNBOKNOG@?$AA?$AN?$AA?6@ 10014d88     HlfViewer.obj
 0002:00004d90       ??_C@_1BG@IOFJDEI@?$AA?4?$AAL?$AAa?$AAn?$AAg?$AAu?$AAa?$AAg?$AAe?$AA?$DN@ 10014d90     HlfViewer.obj
 0002:00004da8       ??_C@_1O@BJPKKLLM@?$AAC?$AAo?$AAn?$AAf?$AAi?$AAg@ 10014da8     HlfViewer.obj
 0002:00004db8       ??_C@_15NPKLCIOJ@?$AAF?$AA1@ 10014db8     HlfViewer.obj
 0002:00004dc0       ??_C@_1CG@GFFDAIMK@?$AAP?$AAr?$AAo?$AAc?$AAe?$AAs?$AAs?$AAE?$AAd?$AAi?$AAt?$AAo?$AAr?$AAI?$AAn@ 10014dc0     HlfViewer.obj
 0002:00004de8       ??_C@_1M@PALMNGCF@?$AAS?$AAt?$AAy?$AAl?$AAe@ 10014de8     HlfViewer.obj
 0002:00004df4       ??_C@_1BE@IHEBLNLC@?$AAE?$AAd?$AAi?$AAt?$AAo?$AAr?$AAK?$AAe?$AAy@ 10014df4     HlfViewer.obj
 0002:00004e08       ??_C@_1BM@GGPBEDKL@?$AAC?$AAh?$AAe?$AAc?$AAk?$AAM?$AAa?$AAs?$AAk?$AAF?$AAi?$AAl?$AAe@ 10014e08     HlfViewer.obj
 0002:00004e24       ??_C@_1BC@KGOLMJNA@?$AAM?$AAa?$AAs?$AAk?$AAF?$AAi?$AAl?$AAe@ 10014e24     HlfViewer.obj
 0002:00004e38       ??_C@_1M@EFMNOFJK@?$AA?$CK?$AA?4?$AAh?$AAl?$AAf@ 10014e38     HlfViewer.obj
 0002:00004e44       _MenuGuid                  10014e44     HlfViewer.obj
 0002:00004e54       _MainGuid                  10014e54     HlfViewer.obj
 0002:00004e68       ??_7PluginCheckBoxBinding@@6B@ 10014e68     HlfViewer.obj
 0002:00004e88       ??_7PluginEditFieldBinding@@6B@ 10014e88     HlfViewer.obj
 0002:00004e90       _DialogGuid                10014e90     HlfViewer.obj
 0002:00004ea4       ??_7PluginRadioButtonBinding@@6B@ 10014ea4     HlfViewer.obj
 0002:00004eac       ??_C@_0O@NLDKAIKN@EncodePointer@ 10014eac     vc_crt_fix_impl.obj
 0002:00004ebc       ??_C@_0O@KBPMFGHI@DecodePointer@ 10014ebc     vc_crt_fix_impl.obj
 0002:00004ecc       ??_C@_0BD@GIGEJCNH@GetModuleHandleExW@ 10014ecc     vc_crt_fix_impl.obj
 0002:00004ee0       ??_C@_0BE@NBEJPEJA@InitializeSListHead@ 10014ee0     vc_crt_fix_impl.obj
 0002:00004ef4       ??_C@_0BG@PLLPFLHB@InterlockedFlushSList@ 10014ef4     vc_crt_fix_impl.obj
 0002:00004f0c       ??_C@_0BJ@PNEEKDOK@InterlockedPopEntrySList@ 10014f0c     vc_crt_fix_impl.obj
 0002:00004f28       ??_C@_0BK@JFGGAIOA@InterlockedPushEntrySList@ 10014f28     vc_crt_fix_impl.obj
 0002:00004f44       ??_C@_0BL@FOECAEGO@InterlockedPushListSListEx@ 10014f44     vc_crt_fix_impl.obj
 0002:00004f60       ??_C@_0BD@FHMMIGCI@RtlFirstEntrySList@ 10014f60     vc_crt_fix_impl.obj
 0002:00004f74       ??_C@_0BA@FGPHPMJB@QueryDepthSList@ 10014f74     vc_crt_fix_impl.obj
 0002:00004f84       ??_C@_0BJ@NLNFLAMA@GetNumaHighestNodeNumber@ 10014f84     vc_crt_fix_impl.obj
 0002:00004fa0       ??_C@_0BP@KHGALBC@GetLogicalProcessorInformation@ 10014fa0     vc_crt_fix_impl.obj
 0002:00004fc0       ??_C@_0BI@BKLFFAPO@SetThreadStackGuarantee@ 10014fc0     vc_crt_fix_impl.obj
 0002:00004fd8       ??_C@_0BM@HCFOFFN@InitializeCriticalSectionEx@ 10014fd8     vc_crt_fix_impl.obj
 0002:00004ff4       ??_C@_0BA@IHGNDAEB@CompareStringEx@ 10014ff4     vc_crt_fix_impl.obj
 0002:00005078       __load_config_used         10015078     LIBCMT:loadcfg.obj
 0002:00005140       ??_R4logic_error@std@@6B@  10015140     libcpmt:xthrow.obj
 0002:00005154       ??_R3logic_error@std@@8    10015154     libcpmt:xthrow.obj
 0002:00005164       ??_R2logic_error@std@@8    10015164     libcpmt:xthrow.obj
 0002:00005170       ??_R1A@?0A@EA@logic_error@std@@8 10015170     libcpmt:xthrow.obj
 0002:0000518c       ??_R4length_error@std@@6B@ 1001518c     libcpmt:xthrow.obj
 0002:000051a0       ??_R3length_error@std@@8   100151a0     libcpmt:xthrow.obj
 0002:000051b0       ??_R2length_error@std@@8   100151b0     libcpmt:xthrow.obj
 0002:000051c0       ??_R1A@?0A@EA@length_error@std@@8 100151c0     libcpmt:xthrow.obj
 0002:000051dc       ??_R4type_info@@6B@        100151dc     LIBCMT:std_type_info_static.obj
 0002:000051f0       ??_R3type_info@@8          100151f0     LIBCMT:std_type_info_static.obj
 0002:00005200       ??_R2type_info@@8          10015200     LIBCMT:std_type_info_static.obj
 0002:00005208       ??_R1A@?0A@EA@type_info@@8 10015208     LIBCMT:std_type_info_static.obj
 0002:00005224       ??_R4bad_exception@std@@6B@ 10015224     libvcruntime:frame.obj
 0002:00005238       ??_R3bad_exception@std@@8  10015238     libvcruntime:frame.obj
 0002:00005248       ??_R2bad_exception@std@@8  10015248     libvcruntime:frame.obj
 0002:00005254       ??_R1A@?0A@EA@bad_exception@std@@8 10015254     libvcruntime:frame.obj
 0002:00005270       ??_R4exception@std@@6B@    10015270     HlfViewer.obj
 0002:00005284       ??_R2bad_array_new_length@std@@8 10015284     HlfViewer.obj
 0002:00005294       ??_R2PluginEditFieldBinding@@8 10015294     HlfViewer.obj
 0002:000052a0       ??_R3DialogAPIBinding@@8   100152a0     HlfViewer.obj
 0002:000052b0       ??_R1A@?0A@EA@PluginCheckBoxBinding@@8 100152b0     HlfViewer.obj
 0002:000052cc       ??_R2bad_alloc@std@@8      100152cc     HlfViewer.obj
 0002:000052d8       ??_R1A@?0A@EA@exception@std@@8 100152d8     HlfViewer.obj
 0002:000052f4       ??_R2PluginRadioButtonBinding@@8 100152f4     HlfViewer.obj
 0002:00005300       ??_R1A@?0A@EA@bad_alloc@std@@8 10015300     HlfViewer.obj
 0002:0000531c       ??_R3PluginRadioButtonBinding@@8 1001531c     HlfViewer.obj
 0002:0000532c       ??_R2exception@std@@8      1001532c     HlfViewer.obj
 0002:00005334       ??_R4PluginRadioButtonBinding@@6B@ 10015334     HlfViewer.obj
 0002:00005348       ??_R3PluginCheckBoxBinding@@8 10015348     HlfViewer.obj
 0002:00005358       ??_R2DialogAPIBinding@@8   10015358     HlfViewer.obj
 0002:00005360       ??_R3exception@std@@8      10015360     HlfViewer.obj
 0002:00005370       ??_R4PluginEditFieldBinding@@6B@ 10015370     HlfViewer.obj
 0002:00005384       ??_R4bad_alloc@std@@6B@    10015384     HlfViewer.obj
 0002:00005398       ??_R4PluginCheckBoxBinding@@6B@ 10015398     HlfViewer.obj
 0002:000053ac       ??_R1A@?0A@EA@PluginRadioButtonBinding@@8 100153ac     HlfViewer.obj
 0002:000053c8       ??_R3bad_array_new_length@std@@8 100153c8     HlfViewer.obj
 0002:000053d8       ??_R3bad_alloc@std@@8      100153d8     HlfViewer.obj
 0002:000053e8       ??_R4bad_array_new_length@std@@6B@ 100153e8     HlfViewer.obj
 0002:000053fc       ??_R3PluginEditFieldBinding@@8 100153fc     HlfViewer.obj
 0002:0000540c       ??_R1A@?0A@EA@bad_array_new_length@std@@8 1001540c     HlfViewer.obj
 0002:00005428       ??_R1A@?0A@EA@PluginEditFieldBinding@@8 10015428     HlfViewer.obj
 0002:00005444       ??_R2PluginCheckBoxBinding@@8 10015444     HlfViewer.obj
 0002:00005450       ??_R1A@?0A@EA@DialogAPIBinding@@8 10015450     HlfViewer.obj
 0002:0000546c       ___safe_se_handler_table   1001546c     <linker-defined>
 0002:0000548c       ___volatile_metadata       1001548c     <linker-defined>
 0002:000057d0       ___rtc_iaa                 100157d0     LIBCMT:initsect.obj
 0002:000057d4       ___rtc_izz                 100157d4     LIBCMT:initsect.obj
 0002:000057d8       ___rtc_taa                 100157d8     LIBCMT:initsect.obj
 0002:000057dc       ___rtc_tzz                 100157dc     LIBCMT:initsect.obj
 0002:0000586c       __TI2?AVbad_alloc@std@@    1001586c     libcpmt:xthrow.obj
 0002:0000587c       __CTA2?AVbad_alloc@std@@   1001587c     libcpmt:xthrow.obj
 0002:00005888       __CT??_R0?AVlogic_error@std@@@8??0logic_error@std@@QAE@ABV01@@Z12 10015888     libcpmt:xthrow.obj
 0002:000058a4       __TI3?AVlength_error@std@@ 100158a4     libcpmt:xthrow.obj
 0002:000058b4       __CTA3?AVlength_error@std@@ 100158b4     libcpmt:xthrow.obj
 0002:000058c4       __CT??_R0?AVlength_error@std@@@8??0length_error@std@@QAE@ABV01@@Z12 100158c4     libcpmt:xthrow.obj
 0002:00005a6c       __TI2?AVbad_exception@std@@ 10015a6c     libvcruntime:frame.obj
 0002:00005a7c       __CTA2?AVbad_exception@std@@ 10015a7c     libvcruntime:frame.obj
 0002:00005a88       __CT??_R0?AVbad_exception@std@@@8??0bad_exception@std@@QAE@ABV01@@Z12 10015a88     libvcruntime:frame.obj
 0002:00005de4       __CTA3?AVbad_array_new_length@std@@ 10015de4     HlfViewer.obj
 0002:00005df4       __CT??_R0?AVbad_alloc@std@@@8??0bad_alloc@std@@QAE@ABV01@@Z12 10015df4     HlfViewer.obj
 0002:00005e10       __CT??_R0?AVexception@std@@@8??0exception@std@@QAE@ABV01@@Z12 10015e10     HlfViewer.obj
 0002:00005e2c       __TI3?AVbad_array_new_length@std@@ 10015e2c     HlfViewer.obj
 0002:00005e3c       __CT??_R0?AVbad_array_new_length@std@@@8??0bad_array_new_length@std@@QAE@ABV01@@Z12 10015e3c     HlfViewer.obj
 0002:00005f28       __IMPORT_DESCRIPTOR_KERNEL32 10015f28     kernel32:KERNEL32.dll
 0002:00005f3c       __IMPORT_DESCRIPTOR_RPCRT4 10015f3c     rpcrt4:RPCRT4.dll
 0002:00005f50       __NULL_IMPORT_DESCRIPTOR   10015f50     kernel32:KERNEL32.dll
 0003:00000000       ___scrt_native_dllmain_reason 10017000     LIBCMT:utility.obj
 0003:00000004       ___security_cookie_complement 10017004     LIBCMT:gs_cookie.obj
 0003:00000008       ___security_cookie         10017008     LIBCMT:gs_cookie.obj
 0003:0000000c       ___isa_enabled             1001700c     LIBCMT:cpu_disp.obj
 0003:00000020       __NLG_Destination          10017020     libvcruntime:exsup.obj
 0003:00000030       ___abort_behavior          10017030     libucrt:abort.obj
 0003:00000050       ___acrt_initial_multibyte_data 10017050     libucrt:mbctype.obj
 0003:00000570       ___acrt_initial_locale_data 10017570     libucrt:nlsdata.obj
 0003:00000628       ___acrt_initial_locale_pointers 10017628     libucrt:nlsdata.obj
 0003:00000630       ___acrt_wide_c_locale_string 10017630     libucrt:nlsdata.obj
 0003:00000638       __iob                      10017638     libucrt:_file.obj
 0003:000006e0       ___globallocalestatus      100176e0     libucrt:glstatus.obj
 0003:000006e8       ___acrt_lconv_c            100176e8     libucrt:localeconv.obj
 0003:00000738       ___acrt_lconv_static_decimal 10017738     libucrt:localeconv.obj
 0003:0000073c       ___acrt_lconv_static_W_decimal 1001773c     libucrt:localeconv.obj
 0003:00000740       __lookuptrailbytes         10017740     libucrt:read.obj
 0003:00000850       __fltused                  10017850     LIBCMT:fltused.obj
 0003:00000860       ??_R0?AVlogic_error@std@@@8 10017860     libcpmt:xthrow.obj
 0003:00000880       ??_R0?AVlength_error@std@@@8 10017880     libcpmt:xthrow.obj
 0003:000008a0       ??_R0?AVbad_exception@std@@@8 100178a0     libvcruntime:frame.obj
 0003:000008c0       ??_R0?AVbad_alloc@std@@@8  100178c0     HlfViewer.obj
 0003:000008dc       ??_R0?AVexception@std@@@8  100178dc     HlfViewer.obj
 0003:000008f8       ??_R0?AVbad_array_new_length@std@@@8 100178f8     HlfViewer.obj
 0003:00000920       ??_R0?AVtype_info@@@8      10017920     LIBCMT:std_type_info_static.obj
 0003:00000938       ??_R0?AVPluginEditFieldBinding@@@8 10017938     HlfViewer.obj
 0003:00000960       ??_R0?AVPluginRadioButtonBinding@@@8 10017960     HlfViewer.obj
 0003:00000988       ??_R0?AVDialogAPIBinding@@@8 10017988     HlfViewer.obj
 0003:000009a8       ??_R0?AVPluginCheckBoxBinding@@@8 100179a8     HlfViewer.obj
 0003:00000cec       ___scrt_current_native_startup_state 10017cec     LIBCMT:utility.obj
 0003:00000cf0       ___scrt_native_startup_lock 10017cf0     LIBCMT:utility.obj
 0003:00000d14       ___isa_available           10017d14     LIBCMT:cpu_disp.obj
 0003:00000d18       ___favor                   10017d18     LIBCMT:cpu_disp.obj
 0003:00000d1c       ___scrt_debugger_hook_flag 10017d1c     LIBCMT:utility_desktop.obj
 0003:00000d20       ___castguard_check_failure_os_handled_fptr 10017d20     LIBCMT:guard_support.obj
 0003:00000d28       ?__type_info_root_node@@3U__type_info_node@@A 10017d28     LIBCMT:tncleanup.obj
 0003:00000d30       ?_OptionsStorage@?1??__local_stdio_printf_options@@9@4_KA 10017d30     LIBCMT:default_local_stdio_options.obj
 0003:00000d38       ?_OptionsStorage@?1??__local_stdio_scanf_options@@9@4_KA 10017d38     LIBCMT:default_local_stdio_options.obj
 0003:00000d40       ?__WinRTOutOfMemoryExceptionCallback@@3P6GPAXXZA 10017d40     libvcruntime:ehhelpers.obj
 0003:00000d6c       ___pPurecall               10017d6c     libvcruntime:purevirt_data.obj
 0003:00000d8c       ?pArgList@UnDecorator@@0PAVReplicator@@A 10017d8c     libvcruntime:undname.obj
 0003:00000d90       ?pZNameList@UnDecorator@@0PAVReplicator@@A 10017d90     libvcruntime:undname.obj
 0003:00000d94       ?pTemplateArgList@UnDecorator@@0PAVReplicator@@A 10017d94     libvcruntime:undname.obj
 0003:00000d98       ?gName@UnDecorator@@0PBDB  10017d98     libvcruntime:undname.obj
 0003:00000d9c       ?name@UnDecorator@@0PBDB   10017d9c     libvcruntime:undname.obj
 0003:00000da0       ?disableFlags@UnDecorator@@0KA 10017da0     libvcruntime:undname.obj
 0003:00000da4       ?fExplicitTemplateParams@UnDecorator@@0_NA 10017da4     libvcruntime:undname.obj
 0003:00000da5       ?fGetTemplateArgumentList@UnDecorator@@0_NA 10017da5     libvcruntime:undname.obj
 0003:00000da8       ?m_pGetParameter@UnDecorator@@0P6APADJ@ZA 10017da8     libvcruntime:undname.obj
 0003:00000dac       ?m_CHPENameOffset@UnDecorator@@0KA 10017dac     libvcruntime:undname.obj
 0003:00000db0       ?m_recursionLevel@UnDecorator@@0KA 10017db0     libvcruntime:undname.obj
 0003:00000df8       ?c_exit_complete@?1???R<lambda_6e4b09c48022b2350581041d5f6b0c4c>@@QBE@XZ@4_NA 10017df8     libucrt:exit.obj
 0003:00000f08       __environ_table            10017f08     libucrt:environment_initialization.obj
 0003:00000f0c       __wenviron_table           10017f0c     libucrt:environment_initialization.obj
 0003:00000f10       ___dcrt_initial_wide_environment 10017f10     libucrt:environment_initialization.obj
 0003:00000f14       ___dcrt_initial_narrow_environment 10017f14     libucrt:environment_initialization.obj
 0003:00000f18       ___acrt_atexit_table       10017f18     libucrt:onexit.obj
 0003:00000f24       ___acrt_at_quick_exit_table 10017f24     libucrt:onexit.obj
 0003:00001084       __mbctype                  10018084     libucrt:mbctype.obj
 0003:00001088       __mbcasemap                10018088     libucrt:mbctype.obj
 0003:0000108c       ___acrt_current_multibyte_data 1001808c     libucrt:mbctype.obj
 0003:00001098       __pgmptr                   10018098     libucrt:argv_data.obj
 0003:0000109c       ___argc                    1001809c     libucrt:argv_data.obj
 0003:000010a0       ___argv                    100180a0     libucrt:argv_data.obj
 0003:000010a4       ___wargv                   100180a4     libucrt:argv_data.obj
 0003:000010a8       __acmdln                   100180a8     libucrt:argv_data.obj
 0003:000010ac       __wcmdln                   100180ac     libucrt:argv_data.obj
 0003:00001188       ___acrt_heap               10018188     libucrt:heap_handle.obj
 0003:00001190       ___pioinfo                 10018190     libucrt:ioinit.obj
 0003:00001390       __nhandle                  10018390     libucrt:ioinit.obj
 0003:000013a8       ___acrt_current_locale_data 100183a8     libucrt:nlsdata.obj
 0003:000013ac       __nstream                  100183ac     libucrt:_file.obj
 0003:000013b0       ___piob                    100183b0     libucrt:_file.obj
 0003:000013b4       ___acrt_stdout_buffer      100183b4     libucrt:_sftbuf.obj
 0003:000013b8       ___acrt_stderr_buffer      100183b8     libucrt:_sftbuf.obj
 0003:000013c4       ___acrt_locale_changed_data 100183c4     libucrt:wsetlocale.obj
 0003:000013cc       ___acrt_lconv_static_null  100183cc     libucrt:localeconv.obj
 0003:000013d0       ___acrt_lconv_static_W_null 100183d0     libucrt:localeconv.obj
 0003:000013e0       ___fastflag                100183e0     libucrt:fp_flags.obj
 0003:000022c8       ___dyn_tls_init_callback   100192c8     <common>
 0003:000022cc       ___scrt_ucrt_dll_is_in_use 100192cc     <common>
 0003:000022d0       __pmatherr                 100192d0     <common>
 0003:000022d4       ___use_sse2_mathfcns       100192d4     <common>

 entry point at        0001:0000394d

 Static symbols

 0000:fffe3000       .debug$S                   10000000     HlfViewer.exp
 0000:fffe3000       .debug$S                   10000000     kernel32:KERNEL32.dll
 0000:fffe3000       .debug$S                   10000000     kernel32:KERNEL32.dll
 0000:fffe3000       .debug$S                   10000000     kernel32:KERNEL32.dll
 0000:fffe3000       .debug$S                   10000000     kernel32:KERNEL32.dll
 0000:fffe3000       .debug$S                   10000000     kernel32:KERNEL32.dll
 0000:fffe3000       .debug$S                   10000000     kernel32:KERNEL32.dll
 0000:fffe3000       .debug$S                   10000000     kernel32:KERNEL32.dll
 0000:fffe3000       .debug$S                   10000000     kernel32:KERNEL32.dll
 0000:fffe3000       .debug$S                   10000000     kernel32:KERNEL32.dll
 0000:fffe3000       .debug$S                   10000000     kernel32:KERNEL32.dll
 0000:fffe3000       .debug$S                   10000000     kernel32:KERNEL32.dll
 0000:fffe3000       .debug$S                   10000000     kernel32:KERNEL32.dll
 0000:fffe3000       .debug$S                   10000000     kernel32:KERNEL32.dll
 0000:fffe3000       .debug$S                   10000000     kernel32:KERNEL32.dll
 0000:fffe3000       .debug$S                   10000000     kernel32:KERNEL32.dll
 0000:fffe3000       .debug$S                   10000000     kernel32:KERNEL32.dll
 0000:fffe3000       .debug$S                   10000000     kernel32:KERNEL32.dll
 0000:fffe3000       .debug$S                   10000000     kernel32:KERNEL32.dll
 0000:fffe3000       .debug$S                   10000000     kernel32:KERNEL32.dll
 0000:fffe3000       .debug$S                   10000000     kernel32:KERNEL32.dll
 0000:fffe3000       .debug$S                   10000000     kernel32:KERNEL32.dll
 0000:fffe3000       .debug$S                   10000000     kernel32:KERNEL32.dll
 0000:fffe3000       .debug$S                   10000000     kernel32:KERNEL32.dll
 0000:fffe3000       .debug$S                   10000000     kernel32:KERNEL32.dll
 0000:fffe3000       .debug$S                   10000000     kernel32:KERNEL32.dll
 0000:fffe3000       .debug$S                   10000000     kernel32:KERNEL32.dll
 0000:fffe3000       .debug$S                   10000000     kernel32:KERNEL32.dll
 0000:fffe3000       .debug$S                   10000000     kernel32:KERNEL32.dll
 0000:fffe3000       .debug$S                   10000000     kernel32:KERNEL32.dll
 0000:fffe3000       .debug$S                   10000000     kernel32:KERNEL32.dll
 0000:fffe3000       .debug$S                   10000000     kernel32:KERNEL32.dll
 0000:fffe3000       .debug$S                   10000000     kernel32:KERNEL32.dll
 0000:fffe3000       .debug$S                   10000000     kernel32:KERNEL32.dll
 0000:fffe3000       .debug$S                   10000000     kernel32:KERNEL32.dll
 0000:fffe3000       .debug$S                   10000000     kernel32:KERNEL32.dll
 0000:fffe3000       .debug$S                   10000000     kernel32:KERNEL32.dll
 0000:fffe3000       .debug$S                   10000000     kernel32:KERNEL32.dll
 0000:fffe3000       .debug$S                   10000000     kernel32:KERNEL32.dll
 0000:fffe3000       .debug$S                   10000000     kernel32:KERNEL32.dll
 0000:fffe3000       .debug$S                   10000000     kernel32:KERNEL32.dll
 0000:fffe3000       .debug$S                   10000000     kernel32:KERNEL32.dll
 0000:fffe3000       .debug$S                   10000000     kernel32:KERNEL32.dll
 0000:fffe3000       .debug$S                   10000000     kernel32:KERNEL32.dll
 0000:fffe3000       .debug$S                   10000000     kernel32:KERNEL32.dll
 0000:fffe3000       .debug$S                   10000000     kernel32:KERNEL32.dll
 0000:fffe3000       .debug$S                   10000000     kernel32:KERNEL32.dll
 0000:fffe3000       .debug$S                   10000000     kernel32:KERNEL32.dll
 0000:fffe3000       .debug$S                   10000000     kernel32:KERNEL32.dll
 0000:fffe3000       .debug$S                   10000000     kernel32:KERNEL32.dll
 0000:fffe3000       .debug$S                   10000000     kernel32:KERNEL32.dll
 0000:fffe3000       .debug$S                   10000000     kernel32:KERNEL32.dll
 0000:fffe3000       .debug$S                   10000000     kernel32:KERNEL32.dll
 0000:fffe3000       .debug$S                   10000000     kernel32:KERNEL32.dll
 0000:fffe3000       .debug$S                   10000000     kernel32:KERNEL32.dll
 0000:fffe3000       .debug$S                   10000000     kernel32:KERNEL32.dll
 0000:fffe3000       .debug$S                   10000000     kernel32:KERNEL32.dll
 0000:fffe3000       .debug$S                   10000000     kernel32:KERNEL32.dll
 0000:fffe3000       .debug$S                   10000000     kernel32:KERNEL32.dll
 0000:fffe3000       .debug$S                   10000000     kernel32:KERNEL32.dll
 0000:fffe3000       .debug$S                   10000000     kernel32:KERNEL32.dll
 0000:fffe3000       .debug$S                   10000000     kernel32:KERNEL32.dll
 0000:fffe3000       .debug$S                   10000000     kernel32:KERNEL32.dll
 0000:fffe3000       .debug$S                   10000000     kernel32:KERNEL32.dll
 0000:fffe3000       .debug$S                   10000000     kernel32:KERNEL32.dll
 0000:fffe3000       .debug$S                   10000000     kernel32:KERNEL32.dll
 0000:fffe3000       .debug$S                   10000000     kernel32:KERNEL32.dll
 0000:fffe3000       .debug$S                   10000000     kernel32:KERNEL32.dll
 0000:fffe3000       .debug$S                   10000000     kernel32:KERNEL32.dll
 0000:fffe3000       .debug$S                   10000000     kernel32:KERNEL32.dll
 0000:fffe3000       .debug$S                   10000000     kernel32:KERNEL32.dll
 0000:fffe3000       .debug$S                   10000000     kernel32:KERNEL32.dll
 0000:fffe3000       .debug$S                   10000000     kernel32:KERNEL32.dll
 0000:fffe3000       .debug$S                   10000000     kernel32:KERNEL32.dll
 0000:fffe3000       .debug$S                   10000000     kernel32:KERNEL32.dll
 0000:fffe3000       .debug$S                   10000000     kernel32:KERNEL32.dll
 0000:fffe3000       .debug$S                   10000000     kernel32:KERNEL32.dll
 0000:fffe3000       .debug$S                   10000000     kernel32:KERNEL32.dll
 0000:fffe3000       .debug$S                   10000000     kernel32:KERNEL32.dll
 0000:fffe3000       .debug$S                   10000000     kernel32:KERNEL32.dll
 0000:fffe3000       .debug$S                   10000000     kernel32:KERNEL32.dll
 0000:fffe3000       .debug$S                   10000000     kernel32:KERNEL32.dll
 0000:fffe3000       .debug$S                   10000000     kernel32:KERNEL32.dll
 0000:fffe3000       .debug$S                   10000000     kernel32:KERNEL32.dll
 0000:fffe3000       .debug$S                   10000000     kernel32:KERNEL32.dll
 0000:fffe3000       .debug$S                   10000000     kernel32:KERNEL32.dll
 0000:fffe3000       .debug$S                   10000000     kernel32:KERNEL32.dll
 0000:fffe3000       .debug$S                   10000000     rpcrt4:RPCRT4.dll
 0001:0000062c       $LN40                      1000162c     HlfViewer.obj
 0001:0000063c       $LN39                      1000163c     HlfViewer.obj
 0001:00000874       $LN61                      10001874     HlfViewer.obj
 0001:00000884       $LN60                      10001884     HlfViewer.obj
 0001:00000b34       $LN51                      10001b34     HlfViewer.obj
 0001:00000b44       $LN50                      10001b44     HlfViewer.obj
 0001:00000d90       $LN76                      10001d90     HlfViewer.obj
 0001:00000da0       $LN75                      10001da0     HlfViewer.obj
 0001:00000ed0       ?CheckExtension@@YA_NPB_W@Z 10001ed0 f   HlfViewer.obj
 0001:00001e80       ?frsuserfunc@@YGHPBUPluginPanelItem@@PB_WPAX@Z 10002e80 f   HlfViewer.obj
 0001:000023c0       $LN112                     100033c0     HlfViewer.obj
 0001:000023d0       $LN111                     100033d0     HlfViewer.obj
 0001:00002780       ?DecodePointer@implementation@?1??DecodePointerWrapper@@YGPAXPAX@Z@SGPAX0@Z 10003780 f   vc_crt_fix_impl.obj
 0001:00002780       ?EncodePointer@implementation@?1??EncodePointerWrapper@@YGPAXPAX@Z@SGPAX0@Z 10003780 f   vc_crt_fix_impl.obj
 0001:00002890       ?GetModuleHandleExW@implementation@?1??GetModuleHandleExWWrapper@@YGHKPB_WPAPAUHINSTANCE__@@@Z@SGHK01@Z 10003890 f   vc_crt_fix_impl.obj
 0001:00002960       ?InitializeSListHead@implementation@slist@@YGXPAT_SLIST_HEADER@@@Z 10003960 f   vc_crt_fix_impl.obj
 0001:00002a20       ?InterlockedFlushSList@implementation@slist@@YGPAU_SINGLE_LIST_ENTRY@@PAT_SLIST_HEADER@@@Z 10003a20 f   vc_crt_fix_impl.obj
 0001:00002a50       ?InterlockedPopEntrySList@implementation@slist@@YGPAU_SINGLE_LIST_ENTRY@@PAT_SLIST_HEADER@@@Z 10003a50 f   vc_crt_fix_impl.obj
 0001:00002aa0       ?InterlockedPushEntrySList@implementation@slist@@YGPAU_SINGLE_LIST_ENTRY@@PAT_SLIST_HEADER@@PAU3@@Z 10003aa0 f   vc_crt_fix_impl.obj
 0001:00002ae0       ?InterlockedPushListSListEx@implementation@slist@@YGPAU_SINGLE_LIST_ENTRY@@PAT_SLIST_HEADER@@PAU3@1K@Z 10003ae0 f   vc_crt_fix_impl.obj
 0001:00002b20       ?RtlFirstEntrySList@implementation@slist@@YGPAU_SINGLE_LIST_ENTRY@@PAT_SLIST_HEADER@@@Z 10003b20 f   vc_crt_fix_impl.obj
 0001:00002b50       ?QueryDepthSList@implementation@slist@@YGGPAT_SLIST_HEADER@@@Z 10003b50 f   vc_crt_fix_impl.obj
 0001:00002e00       ?GetNumaHighestNodeNumber@implementation@?1??GetNumaHighestNodeNumberWrapper@@YGHPAK@Z@SGH0@Z 10003e00 f   vc_crt_fix_impl.obj
 0001:00002e70       ?GetLogicalProcessorInformation@implementation@?1??GetLogicalProcessorInformationWrapper@@YGHPAU_SYSTEM_LOGICAL_PROCESSOR_INFORMATION@@PAK@Z@SGH01@Z 10003e70 f   vc_crt_fix_impl.obj
 0001:00002ed0       ?SetThreadStackGuarantee@implementation@?1??SetThreadStackGuaranteeWrapper@@YGHPAK@Z@SGH0@Z 10003ed0 f   vc_crt_fix_impl.obj
 0001:00002f30       ?InitializeCriticalSectionEx@implementation@?1??InitializeCriticalSectionExWrapper@@YGHPAU_RTL_CRITICAL_SECTION@@KK@Z@SGH0KK@Z 10003f30 f   vc_crt_fix_impl.obj
 0001:00002fb0       ?CompareStringEx@implementation@?1??CompareStringExWrapper@@YGHPB_WK0H0HPAU_nlsversioninfo@@PAXJ@Z@SGH0K0H0H12J@Z 10003fb0 f   vc_crt_fix_impl.obj
 0001:00003030       ?CompareStringEx@implementation@?1??LCMapStringExWrapper@@YGHPB_WK0HPA_WHPAU_nlsversioninfo@@PAXJ@Z@SGH0K0H1H23J@Z 10004030 f   vc_crt_fix_impl.obj
 0001:000032f3       ?find_pe_section@@YAPAU_IMAGE_SECTION_HEADER@@QAEI@Z 100042f3 f   LIBCMT:utility.obj
 0001:0000360d       ?dllmain_crt_dispatch@@YGHQAUHINSTANCE__@@KQAX@Z 1000460d f   LIBCMT:dll_dllmain.obj
 0001:00003660       ?dllmain_crt_process_attach@@YAHQAUHINSTANCE__@@QAX@Z 10004660 f   LIBCMT:dll_dllmain.obj
 0001:00003767       ?dllmain_crt_process_detach@@YAH_N@Z 10004767 f   LIBCMT:dll_dllmain.obj
 0001:00003817       ?dllmain_dispatch@@YAHQAUHINSTANCE__@@KQAX@Z 10004817 f   LIBCMT:dll_dllmain.obj
 0001:00003922       ?dllmain_raw@@YGHQAUHINSTANCE__@@KQAX@Z 10004922 f   LIBCMT:dll_dllmain.obj
 0001:00003ca0       $$000000                   10004ca0     LIBCMT:sehprolg4.obj
 0001:00003ce8       ___get_entropy             10004ce8 f   LIBCMT:gs_support.obj
 0001:000043d2       ?_FilterSetCurrentException@@YAKPAU_EXCEPTION_POINTERS@@E@Z 100053d2 f   libvcruntime:ehhelpers.obj
 0001:00004590       _ValidateLocalCookies      10005590 f   libvcruntime:chandler4.obj
 0001:00004730       $$000000                   10005730     libvcruntime:memset.obj
 0001:00004775       XMMMov                     10005775     libvcruntime:memset.obj
 0001:000047b0       LargeRangeBytes            100057b0     libvcruntime:memset.obj
 0001:000047ed       XmmMovSmall                100057ed     libvcruntime:memset.obj
 0001:00004800       XmmSmallLoop               10005800     libvcruntime:memset.obj
 0001:00004805       MidRangeBytes              10005805     libvcruntime:memset.obj
 0001:00004821       XMMTrailingBytes           10005821     libvcruntime:memset.obj
 0001:00004835       SmallMov                   10005835     libvcruntime:memset.obj
 0001:0000483d       ByteLoop                   1000583d     libvcruntime:memset.obj
 0001:0000484b       DwordTest                  1000584b     libvcruntime:memset.obj
 0001:0000485b       QwordTest                  1000585b     libvcruntime:memset.obj
 0001:00004870       QwordLoop                  10005870     libvcruntime:memset.obj
 0001:00004883       toend                      10005883     libvcruntime:memset.obj
 0001:00004a29       ??$BuildCatchObjectHelperInternal@V__FrameHandler3@@@@YAHPAUEHExceptionRecord@@PAXPBU_s_HandlerType@@PBU_s_CatchableType@@@Z 10005a29 f   libvcruntime:frame.obj
 0001:00004b67       ??$BuildCatchObjectInternal@V__FrameHandler3@@@@YAXPAUEHExceptionRecord@@PAXPBU_s_HandlerType@@PBU_s_CatchableType@@@Z 10005b67 f   libvcruntime:frame.obj
 0001:00004c00       ??$CatchIt@V__FrameHandler3@@@@YAXPAUEHExceptionRecord@@PAUEHRegistrationNode@@PAU_CONTEXT@@PAXPBU_s_FuncInfo@@PBU_s_HandlerType@@PBU_s_CatchableType@@PBU_s_TryBlockMapEntry@@H1EE@Z 10005c00 f   libvcruntime:frame.obj
 0001:00004c80       ??$FindHandler@V__FrameHandler3@@@@YAXPAUEHExceptionRecord@@PAUEHRegistrationNode@@PAU_CONTEXT@@PAXPBU_s_FuncInfo@@EH1@Z 10005c80 f   libvcruntime:frame.obj
 0001:0000502a       ??$FindHandlerForForeignException@V__FrameHandler3@@@@YAXPAUEHExceptionRecord@@PAUEHRegistrationNode@@PAU_CONTEXT@@PAXPBU_s_FuncInfo@@HH1@Z 1000602a f   libvcruntime:frame.obj
 0001:00005342       ?CallCatchBlock@@YAPAXPAUEHExceptionRecord@@PAUEHRegistrationNode@@PAU_CONTEXT@@PBU_s_FuncInfo@@PAXHK@Z 10006342 f   libvcruntime:frame.obj
 0001:00005506       ?CallUnexpected@@YAXPBU_s_ESTypeList@@@Z 10006506 f   libvcruntime:frame.obj
 0001:00005526       __catch$?CallUnexpected@@YAXPBU_s_ESTypeList@@@Z$0 10006526 f   libvcruntime:frame.obj
 0001:00005545       ?ExFilterRethrow@@YAHPAU_EXCEPTION_POINTERS@@@Z 10006545 f   libvcruntime:frame.obj
 0001:0000568f       ?IsInExceptionSpec@@YAEPAUEHExceptionRecord@@PBU_s_ESTypeList@@@Z 1000668f f   libvcruntime:frame.obj
 0001:00005760       $$000000                   10006760     libvcruntime:lowhelpr.obj
 0001:0000579f       _NLG_Continue              1000679f     libvcruntime:lowhelpr.obj
 0001:00005850       $$000000                   10006850     libvcruntime:exsup4.obj
 0001:00005882       _lu_top                    10006882     libvcruntime:exsup4.obj
 0001:000058e1       _lu_done                   100068e1     libvcruntime:exsup4.obj
 0001:000058f0       $$000000                   100068f0     libvcruntime:exsup4.obj
 0001:000058f0       __unwind_handler4          100068f0 f   libvcruntime:exsup4.obj
 0001:00005940       $$000000                   10006940     libvcruntime:exsup4.obj
 0001:00005960       $$000000                   10006960     libvcruntime:exsup4.obj
 0001:00005980       $$000000                   10006980     libvcruntime:exsup4.obj
 0001:00005995       ReturnPoint                10006995     libvcruntime:exsup4.obj
 0001:000059a0       $$000000                   100069a0     libvcruntime:exsup4.obj
 0001:000059b7       ?try_get_first_available_module@@YAPAUHINSTANCE__@@QBW4module_id@?A0x26f6bd02@@0@Z 100069b7 f   libvcruntime:winapi_downlevel.obj
 0001:00005a51       ?try_get_function@@YAPAXW4function_id@?A0x26f6bd02@@QBDQBW4module_id@2@2@Z 10006a51 f   libvcruntime:winapi_downlevel.obj
 0001:00005c20       $$000000                   10006c20     libvcruntime:memcpy.obj
 0001:00005c20       $$000000                   10006c20     libvcruntime:memmove.obj
 0001:00005c40       CopyUp                     10006c40     libvcruntime:memcpy.obj
 0001:00005c40       CopyUp                     10006c40     libvcruntime:memmove.obj
 0001:00005c64       CopyUpLargeMov             10006c64     libvcruntime:memcpy.obj
 0001:00005c64       CopyUpLargeMov             10006c64     libvcruntime:memmove.obj
 0001:00005c77       CopyUpSSE2Check            10006c77     libvcruntime:memcpy.obj
 0001:00005c77       CopyUpSSE2Check            10006c77     libvcruntime:memmove.obj
 0001:00005c90       AtomChk                    10006c90     libvcruntime:memcpy.obj
 0001:00005c90       AtomChk                    10006c90     libvcruntime:memmove.obj
 0001:00005cb6       PalignHead4                10006cb6     libvcruntime:memcpy.obj
 0001:00005cb6       PalignHead4                10006cb6     libvcruntime:memmove.obj
 0001:00005cc9       PalignHead8                10006cc9     libvcruntime:memcpy.obj
 0001:00005cc9       PalignHead8                10006cc9     libvcruntime:memmove.obj
 0001:00005ce0       PalignLoop                 10006ce0     libvcruntime:memcpy.obj
 0001:00005ce0       PalignLoop                 10006ce0     libvcruntime:memmove.obj
 0001:00005cf2       MovPalign12                10006cf2     libvcruntime:memcpy.obj
 0001:00005cf2       MovPalign12                10006cf2     libvcruntime:memmove.obj
 0001:00005cfc       PalignLoop12               10006cfc     libvcruntime:memcpy.obj
 0001:00005cfc       PalignLoop12               10006cfc     libvcruntime:memmove.obj
 0001:00005d4d       MovPalign8                 10006d4d     libvcruntime:memcpy.obj
 0001:00005d4d       MovPalign8                 10006d4d     libvcruntime:memmove.obj
 0001:00005d58       PalignLoop8                10006d58     libvcruntime:memcpy.obj
 0001:00005d58       PalignLoop8                10006d58     libvcruntime:memmove.obj
 0001:00005da6       MovPalign4                 10006da6     libvcruntime:memcpy.obj
 0001:00005da6       MovPalign4                 10006da6     libvcruntime:memmove.obj
 0001:00005db0       PalignLoop4                10006db0     libvcruntime:memcpy.obj
 0001:00005db0       PalignLoop4                10006db0     libvcruntime:memmove.obj
 0001:00005dfc       PalignTail                 10006dfc     libvcruntime:memcpy.obj
 0001:00005dfc       PalignTail                 10006dfc     libvcruntime:memmove.obj
 0001:00005e14       PalignTail4                10006e14     libvcruntime:memcpy.obj
 0001:00005e14       PalignTail4                10006e14     libvcruntime:memmove.obj
 0001:00005e27       PalignTail8                10006e27     libvcruntime:memcpy.obj
 0001:00005e27       PalignTail8                10006e27     libvcruntime:memmove.obj
 0001:00005e3e       PalignTailLE3              10006e3e     libvcruntime:memcpy.obj
 0001:00005e3e       PalignTailLE3              10006e3e     libvcruntime:memmove.obj
 0001:00005e47       Dword_align                10006e47     libvcruntime:memcpy.obj
 0001:00005e47       Dword_align                10006e47     libvcruntime:memmove.obj
 0001:00005e4f       Dword_up_align_loop        10006e4f     libvcruntime:memcpy.obj
 0001:00005e4f       Dword_up_align_loop        10006e4f     libvcruntime:memmove.obj
 0001:00005e62       Dword_align_Ok             10006e62     libvcruntime:memcpy.obj
 0001:00005e62       Dword_align_Ok             10006e62     libvcruntime:memmove.obj
 0001:00005e7c       ByteCopyUp                 10006e7c     libvcruntime:memcpy.obj
 0001:00005e7c       ByteCopyUp                 10006e7c     libvcruntime:memmove.obj
 0001:00005e84       TrailingUpVec              10006e84     libvcruntime:memcpy.obj
 0001:00005e84       TrailingUpVec              10006e84     libvcruntime:memmove.obj
 0001:00005e94       TrailingUp0                10006e94     libvcruntime:memcpy.obj
 0001:00005e94       TrailingUp0                10006e94     libvcruntime:memmove.obj
 0001:00005e9c       TrailingUp1                10006e9c     libvcruntime:memcpy.obj
 0001:00005e9c       TrailingUp1                10006e9c     libvcruntime:memmove.obj
 0001:00005ea8       TrailingUp2                10006ea8     libvcruntime:memcpy.obj
 0001:00005ea8       TrailingUp2                10006ea8     libvcruntime:memmove.obj
 0001:00005ebc       TrailingUp3                10006ebc     libvcruntime:memcpy.obj
 0001:00005ebc       TrailingUp3                10006ebc     libvcruntime:memmove.obj
 0001:00005ed4       CopyDown                   10006ed4     libvcruntime:memcpy.obj
 0001:00005ed4       CopyDown                   10006ed4     libvcruntime:memmove.obj
 0001:00005ef9       CopyDownNotAligned         10006ef9     libvcruntime:memcpy.obj
 0001:00005ef9       CopyDownNotAligned         10006ef9     libvcruntime:memmove.obj
 0001:00005f00       CopyDownAlignLoop          10006f00     libvcruntime:memcpy.obj
 0001:00005f00       CopyDownAlignLoop          10006f00     libvcruntime:memmove.obj
 0001:00005f0d       CopyDownAligned            10006f0d     libvcruntime:memcpy.obj
 0001:00005f0d       CopyDownAligned            10006f0d     libvcruntime:memmove.obj
 0001:00005f30       TrailingDownVec            10006f30     libvcruntime:memcpy.obj
 0001:00005f30       TrailingDownVec            10006f30     libvcruntime:memmove.obj
 0001:00005f40       TrailingDown0              10006f40     libvcruntime:memcpy.obj
 0001:00005f40       TrailingDown0              10006f40     libvcruntime:memmove.obj
 0001:00005f48       TrailingDown1              10006f48     libvcruntime:memcpy.obj
 0001:00005f48       TrailingDown1              10006f48     libvcruntime:memmove.obj
 0001:00005f58       TrailingDown2              10006f58     libvcruntime:memcpy.obj
 0001:00005f58       TrailingDown2              10006f58     libvcruntime:memmove.obj
 0001:00005f6c       TrailingDown3              10006f6c     libvcruntime:memcpy.obj
 0001:00005f6c       TrailingDown3              10006f6c     libvcruntime:memmove.obj
 0001:00005f85       XmmMovLargeAlignTest       10006f85     libvcruntime:memcpy.obj
 0001:00005f85       XmmMovLargeAlignTest       10006f85     libvcruntime:memmove.obj
 0001:00005f8d       XmmMovAlignLoop            10006f8d     libvcruntime:memcpy.obj
 0001:00005f8d       XmmMovAlignLoop            10006f8d     libvcruntime:memmove.obj
 0001:00005f9c       XmmMovLargeLoop            10006f9c     libvcruntime:memcpy.obj
 0001:00005f9c       XmmMovLargeLoop            10006f9c     libvcruntime:memmove.obj
 0001:0000600c       XmmMovSmallTest            1000700c     libvcruntime:memcpy.obj
 0001:0000600c       XmmMovSmallTest            1000700c     libvcruntime:memmove.obj
 0001:00006011       XmmMovSmallLoop            10007011     libvcruntime:memcpy.obj
 0001:00006011       XmmMovSmallLoop            10007011     libvcruntime:memmove.obj
 0001:00006034       CopyDownSmall              10007034     libvcruntime:memcpy.obj
 0001:00006034       CopyDownSmall              10007034     libvcruntime:memmove.obj
 0001:0000603c       CopyDownDwordLoop          1000703c     libvcruntime:memcpy.obj
 0001:0000603c       CopyDownDwordLoop          1000703c     libvcruntime:memmove.obj
 0001:00006051       CopyDownByteTest           10007051     libvcruntime:memcpy.obj
 0001:00006051       CopyDownByteTest           10007051     libvcruntime:memmove.obj
 0001:00006055       CopyDownByteLoop           10007055     libvcruntime:memcpy.obj
 0001:00006055       CopyDownByteLoop           10007055     libvcruntime:memmove.obj
 0001:00006064       CopyDownReturn             10007064     libvcruntime:memcpy.obj
 0001:00006064       CopyDownReturn             10007064     libvcruntime:memmove.obj
 0001:00006070       XmmCopy                    10007070     libvcruntime:memcpy.obj
 0001:00006070       XmmCopy                    10007070     libvcruntime:memmove.obj
 0001:0000607d       XmmCopyAligned             1000707d     libvcruntime:memcpy.obj
 0001:0000607d       XmmCopyAligned             1000707d     libvcruntime:memmove.obj
 0001:00006090       XmmCopyLargeLoop           10007090     libvcruntime:memcpy.obj
 0001:00006090       XmmCopyLargeLoop           10007090     libvcruntime:memmove.obj
 0001:000060ed       XmmCopySmallTest           100070ed     libvcruntime:memcpy.obj
 0001:000060ed       XmmCopySmallTest           100070ed     libvcruntime:memmove.obj
 0001:00006100       XmmCopySmallLoop           10007100     libvcruntime:memcpy.obj
 0001:00006100       XmmCopySmallLoop           10007100     libvcruntime:memmove.obj
 0001:0000611b       CopyUpDwordMov             1000711b     libvcruntime:memcpy.obj
 0001:0000611b       CopyUpDwordMov             1000711b     libvcruntime:memmove.obj
 0001:00006120       CopyUpDwordTest            10007120     libvcruntime:memcpy.obj
 0001:00006120       CopyUpDwordTest            10007120     libvcruntime:memmove.obj
 0001:00006127       CopyUpDwordLoop            10007127     libvcruntime:memcpy.obj
 0001:00006127       CopyUpDwordLoop            10007127     libvcruntime:memmove.obj
 0001:00006136       CopyUpByteTest             10007136     libvcruntime:memcpy.obj
 0001:00006136       CopyUpByteTest             10007136     libvcruntime:memmove.obj
 0001:0000613d       CopyUpByteLoop             1000713d     libvcruntime:memcpy.obj
 0001:0000613d       CopyUpByteLoop             1000713d     libvcruntime:memmove.obj
 0001:00006150       CopyUpReturn               10007150     libvcruntime:memcpy.obj
 0001:00006150       CopyUpReturn               10007150     libvcruntime:memmove.obj
 0001:00006160       XmmCopyUnaligned           10007160     libvcruntime:memcpy.obj
 0001:00006160       XmmCopyUnaligned           10007160     libvcruntime:memmove.obj
 0001:00006173       XmmAlignByte               10007173     libvcruntime:memcpy.obj
 0001:00006173       XmmAlignByte               10007173     libvcruntime:memmove.obj
 0001:0000617c       XmmAlignDwordTest          1000717c     libvcruntime:memcpy.obj
 0001:0000617c       XmmAlignDwordTest          1000717c     libvcruntime:memmove.obj
 0001:00006181       XmmAlignDwordLoop          10007181     libvcruntime:memcpy.obj
 0001:00006181       XmmAlignDwordLoop          10007181     libvcruntime:memmove.obj
 0001:0000618e       XmmAlignAdjustCnt          1000718e     libvcruntime:memcpy.obj
 0001:0000618e       XmmAlignAdjustCnt          1000718e     libvcruntime:memmove.obj
 0001:000061a0       $$000000                   100071a0     libvcruntime:exsup.obj
 0001:000061b0       $$000000                   100071b0     libvcruntime:exsup.obj
 0001:000061bb       __NLG_Go                   100071bb     libvcruntime:exsup.obj
 0001:000061d0       $$000000                   100071d0     libvcruntime:exsup.obj
 0001:00006623       ??$?RV<lambda_03b1d95aef87969028cfba75ccab2455>@@AAV<lambda_6e4b09c48022b2350581041d5f6b0c4c>@@V<lambda_22bdf7517842c4b3e53723af5aa32b9e>@@@?$__crt_seh_guarded_call@X@@QAEX$$QAV<lambda_03b1d95aef87969028cfba75ccab2455>@@AAV<lambda_6e4b09c48022b2350581041d5f6b0c4c>@@$$QAV<lambda_22bdf7517842c4b3e53723af5aa32b9e>@@@Z 10007623 f   libucrt:exit.obj
 0001:00006670       ??R<lambda_6e4b09c48022b2350581041d5f6b0c4c>@@QBE@XZ 10007670 f   libucrt:exit.obj
 0001:0000674a       ?atexit_exception_filter@@YAHK@Z 1000774a f   libucrt:exit.obj
 0001:0000675d       ?common_exit@@YAXHW4_crt_exit_cleanup_mode@@W4_crt_exit_return_mode@@@Z 1000775d f   libucrt:exit.obj
 0001:000067c1       ?exit_or_terminate_process@@YAXI@Z 100077c1 f   libucrt:exit.obj
 0001:00006803       ?is_managed_app@@YA_NXZ    10007803 f   libucrt:exit.obj
 0001:00006846       ?try_cor_exit_process@@YAXI@Z 10007846 f   libucrt:exit.obj
 0001:000068d4       ??$common_configure_argv@D@@YAHW4_crt_argv_mode@@@Z 100078d4 f   libucrt:argv_parsing.obj
 0001:00006a0a       ??$parse_command_line@D@@YAXPADPAPAD0PAI2@Z 10007a0a f   libucrt:argv_parsing.obj
 0001:00006bdb       ??$common_initialize_environment_nolock@D@@YAHXZ 10007bdb f   libucrt:environment_initialization.obj
 0001:00006c2e       ??$create_environment@D@@YAQAPADQAD@Z 10007c2e f   libucrt:environment_initialization.obj
 0001:00006cfe       ??$free_environment@D@@YAXQAPAD@Z 10007cfe f   libucrt:environment_initialization.obj
 0001:00006cfe       ??$free_environment@_W@@YAXQAPA_W@Z 10007cfe f   libucrt:environment_initialization.obj
 0001:00006d56       ??$uninitialize_environment_internal@D@@YAXAAPAPAD@Z 10007d56 f   libucrt:environment_initialization.obj
 0001:00006d71       ??$uninitialize_environment_internal@_W@@YAXAAPAPA_W@Z 10007d71 f   libucrt:environment_initialization.obj
 0001:00006dc8       ??$?RV<lambda_69a2805e680e0e292e8ba93315fe43a8>@@AAV<lambda_f03950bc5685219e0bcd2087efbe011e>@@V<lambda_03fcd07e894ec930e3f35da366ca99d6>@@@?$__crt_seh_guarded_call@H@@QAEH$$QAV<lambda_69a2805e680e0e292e8ba93315fe43a8>@@AAV<lambda_f03950bc5685219e0bcd2087efbe011e>@@$$QAV<lambda_03fcd07e894ec930e3f35da366ca99d6>@@@Z 10007dc8 f   libucrt:onexit.obj
 0001:00006e23       ??$?RV<lambda_8e746cf0007f6ed984d6f78af1fec997>@@AAV<lambda_22ebabd17bc4fa466a2aca6d8deb888d>@@V<lambda_18ed0c0b38a6dc0daf1e7ac6d6adf05e>@@@?$__crt_seh_guarded_call@H@@QAEH$$QAV<lambda_8e746cf0007f6ed984d6f78af1fec997>@@AAV<lambda_22ebabd17bc4fa466a2aca6d8deb888d>@@$$QAV<lambda_18ed0c0b38a6dc0daf1e7ac6d6adf05e>@@@Z 10007e23 f   libucrt:onexit.obj
 0001:00006e9d       ??R<lambda_22ebabd17bc4fa466a2aca6d8deb888d>@@QBEHXZ 10007e9d f   libucrt:onexit.obj
 0001:00006fc6       ??R<lambda_f03950bc5685219e0bcd2087efbe011e>@@QBEHXZ 10007fc6 f   libucrt:onexit.obj
 0001:0000713f       _initialize_environment    1000813f f   libucrt:initialization.obj
 0001:0000713f       _initialize_global_state_isolation 1000813f f   libucrt:initialization.obj
 0001:0000713f       _report_memory_leaks       1000813f f   libucrt:initialization.obj
 0001:0000713f       _uninitialize_c            1000813f f   libucrt:initialization.obj
 0001:0000713f       _uninitialize_global_state_isolation 1000813f f   libucrt:initialization.obj
 0001:00007142       _initialize_global_variables 10008142 f   libucrt:initialization.obj
 0001:0000714f       _initialize_c              1000814f f   libucrt:initialization.obj
 0001:00007169       _uninitialize_environment  10008169 f   libucrt:initialization.obj
 0001:00007171       _initialize_pointers       10008171 f   libucrt:initialization.obj
 0001:0000719f       _uninitialize_vcruntime    1000819f f   libucrt:initialization.obj
 0001:000071a8       _uninitialize_allocated_memory 100081a8 f   libucrt:initialization.obj
 0001:000071bf       _uninitialize_allocated_io_buffers 100081bf f   libucrt:initialization.obj
 0001:0000720f       ??R<lambda_af42a3ee9806e9a7305d451646e05244>@@QBEXAAPAU__crt_multibyte_data@@@Z 1000820f f   libucrt:initialization.obj
 0001:000074b0       $$000000                   100084b0     libucrt:strncmp.obj
 0001:00007562       ??$?RV<lambda_15ade71b0218206bbe3333a0c9b79046>@@AAV<lambda_da44e0f8b0f19ba52fefafb335991732>@@V<lambda_207f2d024fc103971653565357d6cd41>@@@?$__crt_seh_guarded_call@X@@QAEX$$QAV<lambda_15ade71b0218206bbe3333a0c9b79046>@@AAV<lambda_da44e0f8b0f19ba52fefafb335991732>@@$$QAV<lambda_207f2d024fc103971653565357d6cd41>@@@Z 10008562 f   libucrt:per_thread_data.obj
 0001:000075b4       ??$?RV<lambda_38edbb1296d33220d7e4dd0ed76b244a>@@AAV<lambda_5ce1d447e08cb34b2473517608e21441>@@V<lambda_fb385d3da700c9147fc39e65dd577a8c>@@@?$__crt_seh_guarded_call@X@@QAEX$$QAV<lambda_38edbb1296d33220d7e4dd0ed76b244a>@@AAV<lambda_5ce1d447e08cb34b2473517608e21441>@@$$QAV<lambda_fb385d3da700c9147fc39e65dd577a8c>@@@Z 100085b4 f   libucrt:per_thread_data.obj
 0001:0000761f       ??$?RV<lambda_6affb1475c98b40b75cdec977db92e3c>@@AAV<lambda_b8d4b9c228a6ecc3f80208dbb4b4a104>@@V<lambda_608742c3c92a14382c1684fc64f96c88>@@@?$__crt_seh_guarded_call@X@@QAEX$$QAV<lambda_6affb1475c98b40b75cdec977db92e3c>@@AAV<lambda_b8d4b9c228a6ecc3f80208dbb4b4a104>@@$$QAV<lambda_608742c3c92a14382c1684fc64f96c88>@@@Z 1000861f f   libucrt:per_thread_data.obj
 0001:00007674       ??$?RV<lambda_a7e850c220f1c8d1e6efeecdedd162c6>@@AAV<lambda_46720907175c18b6c9d2717bc0d2d362>@@V<lambda_9048902d66e8d99359bc9897bbb930a8>@@@?$__crt_seh_guarded_call@X@@QAEX$$QAV<lambda_a7e850c220f1c8d1e6efeecdedd162c6>@@AAV<lambda_46720907175c18b6c9d2717bc0d2d362>@@$$QAV<lambda_9048902d66e8d99359bc9897bbb930a8>@@@Z 10008674 f   libucrt:per_thread_data.obj
 0001:000076ce       ?construct_ptd@@YAXQAU__acrt_ptd@@QAPAU__crt_locale_data@@@Z 100086ce f   libucrt:per_thread_data.obj
 0001:00007767       ?destroy_fls@@YGXPAX@Z     10008767 f   libucrt:per_thread_data.obj
 0001:00007788       ?destroy_ptd@@YAXQAU__acrt_ptd@@@Z 10008788 f   libucrt:per_thread_data.obj
 0001:00007855       ?replace_current_thread_locale_nolock@@YAXQAU__acrt_ptd@@QAU__crt_locale_data@@@Z 10008855 f   libucrt:per_thread_data.obj
 0001:00007d60       ?<lambda_invoker_cdecl>@<lambda_838c7f62c73c983481e27c09e84b0b5d>@@CAHPBX0@Z 10008d60 f   libucrt:argv_wildcards.obj
 0001:00007d78       ??$__acrt_convert_wcs_mbs_cp@D_WV<lambda_62f6974d9771e494a5ea317cc32e971c>@@U__crt_win32_buffer_internal_dynamic_resizing@@@@YAHQBDAAV?$__crt_win32_buffer@_WU__crt_win32_buffer_internal_dynamic_resizing@@@@ABV<lambda_62f6974d9771e494a5ea317cc32e971c>@@I@Z 10008d78 f   libucrt:argv_wildcards.obj
 0001:00007e2a       ??$__acrt_convert_wcs_mbs_cp@_WDV<lambda_28bda7af82a03b66c1cb3803a755f95d>@@U__crt_win32_buffer_internal_dynamic_resizing@@@@YAHQB_WAAV?$__crt_win32_buffer@DU__crt_win32_buffer_internal_dynamic_resizing@@@@ABV<lambda_28bda7af82a03b66c1cb3803a755f95d>@@I@Z 10008e2a f   libucrt:argv_wildcards.obj
 0001:00007f16       ??$common_expand_argv_wildcards@D@@YAHQAPADQAPAPAD@Z 10008f16 f   libucrt:argv_wildcards.obj
 0001:00008105       ??$copy_and_add_argument_to_buffer@D@@YAHQBD0IAAV?$argument_list@D@?A0x5f5c8891@@@Z 10009105 f   libucrt:argv_wildcards.obj
 0001:000081b6       ??$expand_argument_wildcards@D@@YAHQAD0AAV?$argument_list@D@?A0x5f5c8891@@@Z 100091b6 f   libucrt:argv_wildcards.obj
 0001:00008500       ?expand_if_necessary@?$argument_list@D@?A0x5f5c8891@@AAEHXZ 10009500 f   libucrt:argv_wildcards.obj
 0001:00008592       ??$__acrt_convert_wcs_mbs_cp@_WDV<lambda_0fec1a7b3f42a53036604e18c2d5e07e>@@U__crt_win32_buffer_no_resizing@@@@YAHQB_WAAV?$__crt_win32_buffer@DU__crt_win32_buffer_no_resizing@@@@ABV<lambda_0fec1a7b3f42a53036604e18c2d5e07e>@@I@Z 10009592 f   libucrt:getmodulefilenamea.obj
 0001:00008735       ??$?RV<lambda_ceb1ee4838e85a9d631eb091e2fbe199>@@AAV<lambda_ae742caa10f662c28703da3d2ea5e57e>@@V<lambda_cd08b5d6af4937fe54fc07d0c9bf6b37>@@@?$__crt_seh_guarded_call@X@@QAEX$$QAV<lambda_ceb1ee4838e85a9d631eb091e2fbe199>@@AAV<lambda_ae742caa10f662c28703da3d2ea5e57e>@@$$QAV<lambda_cd08b5d6af4937fe54fc07d0c9bf6b37>@@@Z 10009735 f   libucrt:mbctype.obj
 0001:00008782       ??R<lambda_ae742caa10f662c28703da3d2ea5e57e>@@QBEXXZ 10009782 f   libucrt:mbctype.obj
 0001:00008805       ?CPtoLocaleName@@YAPB_WH@Z 10009805 f   libucrt:mbctype.obj
 0001:00008843       ?getSystemCP@@YAHH@Z       10009843 f   libucrt:mbctype.obj
 0001:000088b4       ?setSBCS@@YAXPAU__crt_multibyte_data@@@Z 100098b4 f   libucrt:mbctype.obj
 0001:00008919       ?setSBUpLow@@YAXPAU__crt_multibyte_data@@@Z 10009919 f   libucrt:mbctype.obj
 0001:00008a9a       ?setmbcp_internal@@YAHH_NQAU__acrt_ptd@@QAPAU__crt_multibyte_data@@@Z 10009a9a f   libucrt:mbctype.obj
 0001:00008bb3       ?update_thread_multibyte_data_internal@@YAPAU__crt_multibyte_data@@QAU__acrt_ptd@@QAPAU1@@Z 10009bb3 f   libucrt:mbctype.obj
 0001:00008ea1       _memcpy_s                  10009ea1 f   libucrt:mbctype.obj
 0001:00008f22       ?x_ismbbtype_l@@YAHPAU__crt_locale_pointers@@IHH@Z 10009f22 f   libucrt:ismbbyte.obj
 0001:000090d3       ?find_end_of_double_null_terminated_sequence@@YAPB_WQB_W@Z 1000a0d3 f   libucrt:get_environment_from_os.obj
 0001:000091fb       ?try_get_AreFileApisANSI@@YAP6GHXZXZ 1000a1fb f   libucrt:winapi_thunks.obj
 0001:00009215       ?try_get_LCMapStringEx@@YAP6GHPB_WK0HPA_WHPAU_nlsversioninfo@@PAXJ@ZXZ 1000a215 f   libucrt:winapi_thunks.obj
 0001:0000922f       ?try_get_LocaleNameToLCID@@YAP6GKPB_WK@ZXZ 1000a22f f   libucrt:winapi_thunks.obj
 0001:00009249       ?try_get_first_available_module@@YAPAUHINSTANCE__@@QBW4module_id@?A0x391cf84c@@0@Z 1000a249 f   libucrt:winapi_thunks.obj
 0001:00009310       ?try_get_function@@YAPAXW4function_id@?A0x391cf84c@@QBDQBW4module_id@2@2@Z 1000a310 f   libucrt:winapi_thunks.obj
 0001:00009646       ?initialize_inherited_file_handles_nolock@@YAXXZ 1000a646 f   libucrt:ioinit.obj
 0001:000096fc       ?initialize_stdio_handles_nolock@@YAXXZ 1000a6fc f   libucrt:ioinit.obj
 0001:000098d5       ??$?RV<lambda_cbab9ec6f41b0180b23cc171c22676b0>@@AAV<lambda_44731a7d0e6d81c3e6aa82d741081786>@@V<lambda_4b292cb8dd18144e164572427af410ab>@@@?$__crt_seh_guarded_call@P6AXH@Z@@QAEP6AXH@Z$$QAV<lambda_cbab9ec6f41b0180b23cc171c22676b0>@@AAV<lambda_44731a7d0e6d81c3e6aa82d741081786>@@$$QAV<lambda_4b292cb8dd18144e164572427af410ab>@@@Z 1000a8d5 f   libucrt:signal.obj
 0001:00009939       ?get_global_action_nolock@@YAPAP6AXH@ZH@Z 1000a939 f   libucrt:signal.obj
 0001:0000997b       ?siglookup@@YAPAU__crt_signal_action_t@@HQAU1@@Z 1000a97b f   libucrt:signal.obj
 0001:00009c45       ??$?RV<lambda_2866be3712abc81a800a822484c830d8>@@AAV<lambda_39ca0ed439415581b5b15c265174cece>@@V<lambda_2b24c74d71094a6cd0cb82e44167d71b>@@@?$__crt_seh_guarded_call@X@@QAEX$$QAV<lambda_2866be3712abc81a800a822484c830d8>@@AAV<lambda_39ca0ed439415581b5b15c265174cece>@@$$QAV<lambda_2b24c74d71094a6cd0cb82e44167d71b>@@@Z 1000ac45 f   libucrt:fflush.obj
 0001:00009cd1       ??$?RV<lambda_2cc53f568c5a2bb6f192f930a45d44ea>@@AAV<lambda_ab61a845afdef5b7c387490eaf3616ee>@@V<lambda_c2ffc0b7726aa6be21d5f0026187e748>@@@?$__crt_seh_guarded_call@X@@QAEX$$QAV<lambda_2cc53f568c5a2bb6f192f930a45d44ea>@@AAV<lambda_ab61a845afdef5b7c387490eaf3616ee>@@$$QAV<lambda_c2ffc0b7726aa6be21d5f0026187e748>@@@Z 1000acd1 f   libucrt:fflush.obj
 0001:00009d7d       ?common_flush_all@@YAH_N@Z 1000ad7d f   libucrt:fflush.obj
 0001:00009dca       ?common_flush_all_should_try_to_flush_stream@@YA_NV__crt_stdio_stream@@QAH@Z 1000adca f   libucrt:fflush.obj
 0001:00009dfd       ?is_stream_flushable_or_commitable@@YA_NJ@Z 1000adfd f   libucrt:fflush.obj
 0001:0000a1f1       ??$?RV<lambda_e5124f882df8998aaf41531e079ba474>@@AAV<lambda_3e16ef9562a7dcce91392c22ab16ea36>@@V<lambda_e25ca0880e6ef98be67edffd8c599615>@@@?$__crt_seh_guarded_call@X@@QAEX$$QAV<lambda_e5124f882df8998aaf41531e079ba474>@@AAV<lambda_3e16ef9562a7dcce91392c22ab16ea36>@@$$QAV<lambda_e25ca0880e6ef98be67edffd8c599615>@@@Z 1000b1f1 f   libucrt:wsetlocale.obj
 0001:0000a660       ?swap@@YAXPAD0I@Z          1000b660 f   libucrt:qsort.obj
 0001:0000aae4       ??$common_tcsncpy_s@D@@YAHQADIQBDI@Z 1000bae4 f   libucrt:strncpy_s.obj
 0001:0000abb0       $$000000                   1000bbb0     libucrt:strpbrk.obj
 0001:0000adb7       ?__acrt_LCMapStringA_stat@@YAHPAU__crt_locale_pointers@@PB_WKPBDHPADHHH@Z 1000bdb7 f   libucrt:lcmapstringa.obj
 0001:0000afea       ?initialize_multibyte@@YAHXZ 1000bfea f   libucrt:multibyte_initializer.obj
 0001:0000b095       ?GetTableIndexFromLocaleName@@YAHPB_W@Z 1000c095 f   libucrt:lcidtoname_downlevel.obj
 0001:0000b3a0       ??$?RV<lambda_9e9de3de5fa147e2223d7db92bc10aa6>@@AAV<lambda_38ce7e780aa69e748d6df282ebc68efe>@@V<lambda_8ca6da459f0f6780f1cff60fdc3d00e5>@@@?$__crt_seh_guarded_call@H@@QAEH$$QAV<lambda_9e9de3de5fa147e2223d7db92bc10aa6>@@AAV<lambda_38ce7e780aa69e748d6df282ebc68efe>@@$$QAV<lambda_8ca6da459f0f6780f1cff60fdc3d00e5>@@@Z 1000c3a0 f   libucrt:commit.obj
 0001:0000b4bf       ?write_double_translated_ansi_nolock@@YA?AUwrite_result@?A0x17268360@@HQBDI@Z 1000c4bf f   libucrt:write.obj
 0001:0000b869       ?write_double_translated_unicode_nolock@@YA?AUwrite_result@?A0x17268360@@QBDI@Z 1000c869 f   libucrt:write.obj
 0001:0000b8d1       ?write_requires_double_translation_nolock@@YA_NH@Z 1000c8d1 f   libucrt:write.obj
 0001:0000b942       ?write_text_ansi_nolock@@YA?AUwrite_result@?A0x17268360@@HQBDI@Z 1000c942 f   libucrt:write.obj
 0001:0000ba1d       ?write_text_utf16le_nolock@@YA?AUwrite_result@?A0x17268360@@HQBDI@Z 1000ca1d f   libucrt:write.obj
 0001:0000bb06       ?write_text_utf8_nolock@@YA?AUwrite_result@?A0x17268360@@HQBDI@Z 1000cb06 f   libucrt:write.obj
 0001:0000c087       ??R<lambda_3d301b9e52f5099be73030e1f0bf487e>@@QBEIPBD@Z 1000d087 f   libucrt:mbrtowc.obj
 0001:0000c374       ?free_crt_array_internal@@YAXQAPBXI@Z 1000d374 f   libucrt:inittime.obj
 0001:0000c501       ??$common_lseek_nolock@_J@@YA_JH_JH@Z 1000d501 f   libucrt:lseek.obj
 0001:0000c870       $$000000                   1000d870     libucrt:log10_impl.obj
 0001:0000c980       $$000000                   1000d980     libucrt:ceil_pentium4.obj
 0001:0000caa0       $$000000                   1000daa0     libucrt:_strnicm.obj
 0001:0000cb01       ?__dcrt_lowio_initialize_console_output@@YAXXZ 1000db01 f   libucrt:initcon.obj
 0001:0000cbab       ??$?RV<lambda_218ce3db14220d0be481dae8ef3383b6>@@AAV<lambda_628dfdc04ba53c8bfc02c9951375f3f5>@@V<lambda_57dc472bd5c9d5f3b2cbca59b8a843ae>@@@?$__crt_seh_guarded_call@H@@QAEH$$QAV<lambda_218ce3db14220d0be481dae8ef3383b6>@@AAV<lambda_628dfdc04ba53c8bfc02c9951375f3f5>@@$$QAV<lambda_57dc472bd5c9d5f3b2cbca59b8a843ae>@@@Z 1000dbab f   libucrt:close.obj
 0001:0000cdb0       $$000000                   1000ddb0     libucrt:log10_pentium4.obj
 0001:0000d040       $$000000                   1000e040     libucrt:87tran.obj
 0001:0000d250       $$000000                   1000e250     libucrt:87disp.obj
 0001:0000d4b0       $$000000                   1000e4b0     libucrt:common.obj
 0001:0000d640       $$000000                   1000e640     libucrt:genexcep.obj
 0001:0000e6f0       $$000000                   1000f6f0     LIBCMT:alloca16.obj
 0001:0000e706       alloca_8                   1000f706     LIBCMT:alloca16.obj
 0001:0000e720       $$000000                   1000f720     LIBCMT:chkstk.obj
 0001:0000e734       cs10                       1000f734     LIBCMT:chkstk.obj
 0001:0000e742       cs20                       1000f742     LIBCMT:chkstk.obj
 0001:0000e7d0       __ehhandler$??1PluginSettings@@QAE@XZ 1000f7d0 f   HlfViewer.obj
 0001:0000e7f0       __ehhandler$_ConfigureW@4  1000f7f0 f   HlfViewer.obj
 0001:0000e820       __unwindfunclet$?GetPluginConfig@@YAXXZ$0 1000f820 f   HlfViewer.obj
 0001:0000e82d       __ehhandler$?GetPluginConfig@@YAXXZ 1000f82d f   HlfViewer.obj
 0001:0000e854       __ehhandler$?CallUnexpected@@YAXPBU_s_ESTypeList@@@Z 1000f854 f   libvcruntime:frame.obj
 0001:0000e880       ??__FDeleter@?1??InitializeSListHead@implementation@slist@@YGXPAT_SLIST_HEADER@@@Z@YAXXZ 1000f880 f   vc_crt_fix_impl.obj
 0002:000001f0       _GS_ExceptionPointers      100101f0     LIBCMT:gs_report.obj
 0002:00000230       ?tokenTable@@3QBUStringLiteral@@B 10010230     libvcruntime:undname.obj
 0002:000002b0       ?nameTable@@3QBUStringLiteral@@B 100102b0     libvcruntime:undname.obj
 0002:00000548       ?rttiTable@@3QBUStringLiteral@@B 10010548     libvcruntime:undname.obj
 0002:00000570       ?IndirectionName@@3QBUStringLiteral@@B 10010570     libvcruntime:undname.obj
 0002:000005a0       ?PrefixName@@3QBUStringLiteral@@B 100105a0     libvcruntime:undname.obj
 0002:00000bd0       ?module_names@?A0x26f6bd02@@3QBQB_WB 10010bd0     libvcruntime:winapi_downlevel.obj
 0002:00000c78       ?candidate_modules@?1??try_get_FlsAlloc@@YAP6GKP6GXPAX@Z@ZXZ@4QBW4module_id@?A0x26f6bd02@@B 10010c78     libvcruntime:winapi_downlevel.obj
 0002:00000c8c       ?candidate_modules@?1??try_get_FlsFree@@YAP6GHK@ZXZ@4QBW4module_id@?A0x26f6bd02@@B 10010c8c     libvcruntime:winapi_downlevel.obj
 0002:00000c9c       ?candidate_modules@?1??try_get_FlsGetValue@@YAP6GPAXK@ZXZ@4QBW4module_id@?A0x26f6bd02@@B 10010c9c     libvcruntime:winapi_downlevel.obj
 0002:00000cb0       ?candidate_modules@?1??try_get_FlsSetValue@@YAP6GHKPAX@ZXZ@4QBW4module_id@?A0x26f6bd02@@B 10010cb0     libvcruntime:winapi_downlevel.obj
 0002:00000cc4       ?candidate_modules@?1??try_get_InitializeCriticalSectionEx@@YAP6GHPAU_RTL_CRITICAL_SECTION@@KK@ZXZ@4QBW4module_id@?A0x26f6bd02@@B 10010cc4     libvcruntime:winapi_downlevel.obj
 0002:00000d98       ___acrt_initializers       10010d98     libucrt:initialization.obj
 0002:00000e18       ?errtable@@3QBUerrentry@?A0x31fdb9ec@@B 10010e18     libucrt:errno.obj
 0002:00000f80       ?_mb_locale_names@@3QBQB_WB 10010f80     libucrt:mbctype.obj
 0002:00000fc0       ?module_names@?A0x391cf84c@@3QBQB_WB 10010fc0     libucrt:winapi_thunks.obj
 0002:00001438       ?candidate_modules@?1??try_get_AreFileApisANSI@@YAP6GHXZXZ@4QBW4module_id@?A0x391cf84c@@B 10011438     libucrt:winapi_thunks.obj
 0002:0000144c       ?candidate_modules@?1??try_get_FlsAlloc@@YAP6GKP6GXPAX@Z@ZXZ@4QBW4module_id@?A0x391cf84c@@B 1001144c     libucrt:winapi_thunks.obj
 0002:00001454       ?candidate_modules@?1??try_get_FlsFree@@YAP6GHK@ZXZ@4QBW4module_id@?A0x391cf84c@@B 10011454     libucrt:winapi_thunks.obj
 0002:0000145c       ?candidate_modules@?1??try_get_FlsGetValue@@YAP6GPAXK@ZXZ@4QBW4module_id@?A0x391cf84c@@B 1001145c     libucrt:winapi_thunks.obj
 0002:00001464       ?candidate_modules@?1??try_get_FlsSetValue@@YAP6GHKPAX@ZXZ@4QBW4module_id@?A0x391cf84c@@B 10011464     libucrt:winapi_thunks.obj
 0002:0000146c       ?candidate_modules@?1??try_get_InitializeCriticalSectionEx@@YAP6GHPAU_RTL_CRITICAL_SECTION@@KK@ZXZ@4QBW4module_id@?A0x391cf84c@@B 1001146c     libucrt:winapi_thunks.obj
 0002:00001474       ?candidate_modules@?1??try_get_LCMapStringEx@@YAP6GHPB_WK0HPA_WHPAU_nlsversioninfo@@PAXJ@ZXZ@4QBW4module_id@?A0x391cf84c@@B 10011474     libucrt:winapi_thunks.obj
 0002:0000148c       ?candidate_modules@?1??try_get_LocaleNameToLCID@@YAP6GKPB_WK@ZXZ@4QBW4module_id@?A0x391cf84c@@B 1001148c     libucrt:winapi_thunks.obj
 0002:000014a8       ?candidate_modules@?1??try_get_AppPolicyGetProcessTerminationMethod@@YAP6GJPAXPAW4AppPolicyProcessTerminationMethod@@@ZXZ@4QBW4module_id@?A0x391cf84c@@B 100114a8     libucrt:winapi_thunks.obj
 0002:00001f98       ?LcidToLocaleNameTable@?A0x881e4c05@@3QBULcidToLocaleName@1@B 10011f98     libucrt:lcidtoname_downlevel.obj
 0002:000030c0       ?LocaleNameToIndexTable@?A0x881e4c05@@3QBULocaleNameIndex@1@B 100130c0     libucrt:lcidtoname_downlevel.obj
 0002:00004010       LOG_name                   10014010     libucrt:log10_impl.obj
 0002:00004020       _One                       10014020     libucrt:ceil_pentium4.obj
 0002:00004030       _Bns                       10014030     libucrt:ceil_pentium4.obj
 0002:00004040       _Zero                      10014040     libucrt:ceil_pentium4.obj
 0002:00004050       _S                         10014050     libucrt:ceil_pentium4.obj
 0002:00004060       _NegZero                   10014060     libucrt:ceil_pentium4.obj
 0002:00004080       emask                      10014080     libucrt:log10_pentium4.obj
 0002:00004090       CC                         10014090     libucrt:log10_pentium4.obj
 0002:000040a0       Magic                      100140a0     libucrt:log10_pentium4.obj
 0002:000040b0       hi_mask                    100140b0     libucrt:log10_pentium4.obj
 0002:000040c0       LOG10_2                    100140c0     libucrt:log10_pentium4.obj
 0002:000040d0       place_L                    100140d0     libucrt:log10_pentium4.obj
 0002:000040f0       One                        100140f0     libucrt:log10_pentium4.obj
 0002:00004100       Zero                       10014100     libucrt:log10_pentium4.obj
 0002:00004110       Two52                      10014110     libucrt:log10_pentium4.obj
 0002:00004120       Infs                       10014120     libucrt:log10_pentium4.obj
 0002:00004130       NaN                        10014130     libucrt:log10_pentium4.obj
 0002:00004140       coeff                      10014140     libucrt:log10_pentium4.obj
 0002:0000419e       _log2max                   1001419e     libucrt:87tran.obj
 0002:000041a8       _smallarg                  100141a8     libucrt:87tran.obj
 0002:000041b2       _half                      100141b2     libucrt:87tran.obj
 0002:000041fe       One                        100141fe     libucrt:87disp.obj
 0002:00004206       Three                      10014206     libucrt:87disp.obj
 0002:0000420e       XAMtoTagTab                1001420e     libucrt:87disp.obj
 0002:00004220       One                        10014220     libucrt:common.obj
 0002:00004234       DblMax                     10014234     libucrt:common.obj
 0002:0000423c       DblMin                     1001423c     libucrt:common.obj
 0002:00004244       IeeeAdjO                   10014244     libucrt:common.obj
 0002:0000424c       IeeeAdjU                   1001424c     libucrt:common.obj
 0002:00004254       _infinity                  10014254     libucrt:common.obj
 0002:0000425c       _zero                      1001425c     libucrt:common.obj
 0002:00004298       _over                      10014298     libucrt:fpctrl.obj
 0002:000042a4       _under                     100142a4     libucrt:fpctrl.obj
 0002:00004ad8       ?_names@?1??_get_fname@@9@9 10014ad8     libucrt:fpexcept.obj
 0002:00004c80       two32                      10014c80     LIBCMT:ftol2.obj
 0002:00004c84       two63                      10014c84     LIBCMT:ftol2.obj
 0002:00004c88       _NaN                       10014c88     LIBCMT:ftol2.obj
 0002:00004e70       ?_DefKey@@3U_INPUT_RECORD@@A 10014e70     HlfViewer.obj
 0002:00005004       ?ntdll@modules@@3QB_WB     10015004     vc_crt_fix_impl.obj
 0002:00005010       ?kernel32@modules@@3QB_WB  10015010     vc_crt_fix_impl.obj
 0002:000057e0       __ehfuncinfo$??1PluginSettings@@QAE@XZ 100157e0     HlfViewer.obj
 0002:00005804       __ehfuncinfo$_ConfigureW@4 10015804     HlfViewer.obj
 0002:00005828       __unwindtable$_ConfigureW@4 10015828     HlfViewer.obj
 0002:00005838       __ehfuncinfo$?GetPluginConfig@@YAXXZ 10015838     HlfViewer.obj
 0002:0000585c       __unwindtable$?GetPluginConfig@@YAXXZ 1001585c     HlfViewer.obj
 0002:000058e0       __sehtable$___scrt_is_nonwritable_in_current_image 100158e0     LIBCMT:utility.obj
 0002:00005900       __sehtable$?dllmain_crt_process_attach@@YAHQAUHINSTANCE__@@QAX@Z 10015900     LIBCMT:dll_dllmain.obj
 0002:00005920       __sehtable$?dllmain_crt_process_detach@@YAH_N@Z 10015920     LIBCMT:dll_dllmain.obj
 0002:00005948       __sehtable$?dllmain_dispatch@@YAHQAUHINSTANCE__@@KQAX@Z 10015948     LIBCMT:dll_dllmain.obj
 0002:00005968       __sehtable$___DestructExceptionObject 10015968     libvcruntime:ehhelpers.obj
 0002:00005988       __sehtable$?FrameUnwindToState@__FrameHandler3@@SAXPAUEHRegistrationNode@@PAXPBU_s_FuncInfo@@H@Z 10015988     libvcruntime:frame.obj
 0002:000059b0       __sehtable$?CallCatchBlock@@YAPAXPAUEHExceptionRecord@@PAUEHRegistrationNode@@PAU_CONTEXT@@PBU_s_FuncInfo@@PAXHK@Z 100159b0     libvcruntime:frame.obj
 0002:000059d8       __catchsym$?CallUnexpected@@YAXPBU_s_ESTypeList@@@Z$2 100159d8     libvcruntime:frame.obj
 0002:000059e8       __unwindtable$?CallUnexpected@@YAXPBU_s_ESTypeList@@@Z 100159e8     libvcruntime:frame.obj
 0002:000059f8       __tryblocktable$?CallUnexpected@@YAXPBU_s_ESTypeList@@@Z 100159f8     libvcruntime:frame.obj
 0002:00005a0c       __ehfuncinfo$?CallUnexpected@@YAXPBU_s_ESTypeList@@@Z 10015a0c     libvcruntime:frame.obj
 0002:00005a30       __sehtable$??$BuildCatchObjectHelperInternal@V__FrameHandler3@@@@YAHPAUEHExceptionRecord@@PAXPBU_s_HandlerType@@PBU_s_CatchableType@@@Z 10015a30     libvcruntime:frame.obj
 0002:00005a50       __sehtable$??$BuildCatchObjectInternal@V__FrameHandler3@@@@YAXPAUEHExceptionRecord@@PAXPBU_s_HandlerType@@PBU_s_CatchableType@@@Z 10015a50     libvcruntime:frame.obj
 0002:00005aa8       __sehtable$__query_new_handler 10015aa8     libucrt:new_handler.obj
 0002:00005ac8       __sehtable$??R<lambda_6e4b09c48022b2350581041d5f6b0c4c>@@QBE@XZ 10015ac8     libucrt:exit.obj
 0002:00005ae8       __sehtable$??$?RV<lambda_03b1d95aef87969028cfba75ccab2455>@@AAV<lambda_6e4b09c48022b2350581041d5f6b0c4c>@@V<lambda_22bdf7517842c4b3e53723af5aa32b9e>@@@?$__crt_seh_guarded_call@X@@QAEX$$QAV<lambda_03b1d95aef87969028cfba75ccab2455>@@AAV<lambda_6e4b09c48022b2350581041d5f6b0c4c>@@$$QAV<lambda_22bdf7517842c4b3e53723af5aa32b9e>@@@Z 10015ae8     libucrt:exit.obj
 0002:00005b08       __sehtable$??$?RV<lambda_8e746cf0007f6ed984d6f78af1fec997>@@AAV<lambda_22ebabd17bc4fa466a2aca6d8deb888d>@@V<lambda_18ed0c0b38a6dc0daf1e7ac6d6adf05e>@@@?$__crt_seh_guarded_call@H@@QAEH$$QAV<lambda_8e746cf0007f6ed984d6f78af1fec997>@@AAV<lambda_22ebabd17bc4fa466a2aca6d8deb888d>@@$$QAV<lambda_18ed0c0b38a6dc0daf1e7ac6d6adf05e>@@@Z 10015b08     libucrt:onexit.obj
 0002:00005b28       __sehtable$??$?RV<lambda_69a2805e680e0e292e8ba93315fe43a8>@@AAV<lambda_f03950bc5685219e0bcd2087efbe011e>@@V<lambda_03fcd07e894ec930e3f35da366ca99d6>@@@?$__crt_seh_guarded_call@H@@QAEH$$QAV<lambda_69a2805e680e0e292e8ba93315fe43a8>@@AAV<lambda_f03950bc5685219e0bcd2087efbe011e>@@$$QAV<lambda_03fcd07e894ec930e3f35da366ca99d6>@@@Z 10015b28     libucrt:onexit.obj
 0002:00005b48       __sehtable$_terminate      10015b48     libucrt:terminate.obj
 0002:00005b68       __sehtable$??$?RV<lambda_15ade71b0218206bbe3333a0c9b79046>@@AAV<lambda_da44e0f8b0f19ba52fefafb335991732>@@V<lambda_207f2d024fc103971653565357d6cd41>@@@?$__crt_seh_guarded_call@X@@QAEX$$QAV<lambda_15ade71b0218206bbe3333a0c9b79046>@@AAV<lambda_da44e0f8b0f19ba52fefafb335991732>@@$$QAV<lambda_207f2d024fc103971653565357d6cd41>@@@Z 10015b68     libucrt:per_thread_data.obj
 0002:00005b88       __sehtable$??$?RV<lambda_a7e850c220f1c8d1e6efeecdedd162c6>@@AAV<lambda_46720907175c18b6c9d2717bc0d2d362>@@V<lambda_9048902d66e8d99359bc9897bbb930a8>@@@?$__crt_seh_guarded_call@X@@QAEX$$QAV<lambda_a7e850c220f1c8d1e6efeecdedd162c6>@@AAV<lambda_46720907175c18b6c9d2717bc0d2d362>@@$$QAV<lambda_9048902d66e8d99359bc9897bbb930a8>@@@Z 10015b88     libucrt:per_thread_data.obj
 0002:00005ba8       __sehtable$??$?RV<lambda_38edbb1296d33220d7e4dd0ed76b244a>@@AAV<lambda_5ce1d447e08cb34b2473517608e21441>@@V<lambda_fb385d3da700c9147fc39e65dd577a8c>@@@?$__crt_seh_guarded_call@X@@QAEX$$QAV<lambda_38edbb1296d33220d7e4dd0ed76b244a>@@AAV<lambda_5ce1d447e08cb34b2473517608e21441>@@$$QAV<lambda_fb385d3da700c9147fc39e65dd577a8c>@@@Z 10015ba8     libucrt:per_thread_data.obj
 0002:00005bc8       __sehtable$??$?RV<lambda_6affb1475c98b40b75cdec977db92e3c>@@AAV<lambda_b8d4b9c228a6ecc3f80208dbb4b4a104>@@V<lambda_608742c3c92a14382c1684fc64f96c88>@@@?$__crt_seh_guarded_call@X@@QAEX$$QAV<lambda_6affb1475c98b40b75cdec977db92e3c>@@AAV<lambda_b8d4b9c228a6ecc3f80208dbb4b4a104>@@$$QAV<lambda_608742c3c92a14382c1684fc64f96c88>@@@Z 10015bc8     libucrt:per_thread_data.obj
 0002:00005be8       __sehtable$?update_thread_multibyte_data_internal@@YAPAU__crt_multibyte_data@@QAU__acrt_ptd@@QAPAU1@@Z 10015be8     libucrt:mbctype.obj
 0002:00005c08       __sehtable$??$?RV<lambda_ceb1ee4838e85a9d631eb091e2fbe199>@@AAV<lambda_ae742caa10f662c28703da3d2ea5e57e>@@V<lambda_cd08b5d6af4937fe54fc07d0c9bf6b37>@@@?$__crt_seh_guarded_call@X@@QAEX$$QAV<lambda_ceb1ee4838e85a9d631eb091e2fbe199>@@AAV<lambda_ae742caa10f662c28703da3d2ea5e57e>@@$$QAV<lambda_cd08b5d6af4937fe54fc07d0c9bf6b37>@@@Z 10015c08     libucrt:mbctype.obj
 0002:00005c28       __sehtable$___acrt_initialize_lowio 10015c28     libucrt:ioinit.obj
 0002:00005c48       __sehtable$_raise          10015c48     libucrt:signal.obj
 0002:00005c68       __sehtable$??$?RV<lambda_cbab9ec6f41b0180b23cc171c22676b0>@@AAV<lambda_44731a7d0e6d81c3e6aa82d741081786>@@V<lambda_4b292cb8dd18144e164572427af410ab>@@@?$__crt_seh_guarded_call@P6AXH@Z@@QAEP6AXH@Z$$QAV<lambda_cbab9ec6f41b0180b23cc171c22676b0>@@AAV<lambda_44731a7d0e6d81c3e6aa82d741081786>@@$$QAV<lambda_4b292cb8dd18144e164572427af410ab>@@@Z 10015c68     libucrt:signal.obj
 0002:00005c88       __sehtable$??$?RV<lambda_2866be3712abc81a800a822484c830d8>@@AAV<lambda_39ca0ed439415581b5b15c265174cece>@@V<lambda_2b24c74d71094a6cd0cb82e44167d71b>@@@?$__crt_seh_guarded_call@X@@QAEX$$QAV<lambda_2866be3712abc81a800a822484c830d8>@@AAV<lambda_39ca0ed439415581b5b15c265174cece>@@$$QAV<lambda_2b24c74d71094a6cd0cb82e44167d71b>@@@Z 10015c88     libucrt:fflush.obj
 0002:00005ca8       __sehtable$??$?RV<lambda_2cc53f568c5a2bb6f192f930a45d44ea>@@AAV<lambda_ab61a845afdef5b7c387490eaf3616ee>@@V<lambda_c2ffc0b7726aa6be21d5f0026187e748>@@@?$__crt_seh_guarded_call@X@@QAEX$$QAV<lambda_2cc53f568c5a2bb6f192f930a45d44ea>@@AAV<lambda_ab61a845afdef5b7c387490eaf3616ee>@@$$QAV<lambda_c2ffc0b7726aa6be21d5f0026187e748>@@@Z 10015ca8     libucrt:fflush.obj
 0002:00005cc8       __sehtable$??$?RV<lambda_e5124f882df8998aaf41531e079ba474>@@AAV<lambda_3e16ef9562a7dcce91392c22ab16ea36>@@V<lambda_e25ca0880e6ef98be67edffd8c599615>@@@?$__crt_seh_guarded_call@X@@QAEX$$QAV<lambda_e5124f882df8998aaf41531e079ba474>@@AAV<lambda_3e16ef9562a7dcce91392c22ab16ea36>@@$$QAV<lambda_e25ca0880e6ef98be67edffd8c599615>@@@Z 10015cc8     libucrt:wsetlocale.obj
 0002:00005ce8       __sehtable$___acrt_update_thread_locale_data 10015ce8     libucrt:locale_refcounting.obj
 0002:00005d08       __sehtable$___acrt_lowio_ensure_fh_exists 10015d08     libucrt:osfinfo.obj
 0002:00005d28       __sehtable$??$?RV<lambda_9e9de3de5fa147e2223d7db92bc10aa6>@@AAV<lambda_38ce7e780aa69e748d6df282ebc68efe>@@V<lambda_8ca6da459f0f6780f1cff60fdc3d00e5>@@@?$__crt_seh_guarded_call@H@@QAEH$$QAV<lambda_9e9de3de5fa147e2223d7db92bc10aa6>@@AAV<lambda_38ce7e780aa69e748d6df282ebc68efe>@@$$QAV<lambda_8ca6da459f0f6780f1cff60fdc3d00e5>@@@Z 10015d28     libucrt:commit.obj
 0002:00005d48       __sehtable$__write         10015d48     libucrt:write.obj
 0002:00005d68       __sehtable$__fcloseall     10015d68     libucrt:closeall.obj
 0002:00005d88       __sehtable$_fclose         10015d88     libucrt:fclose.obj
 0002:00005da8       __sehtable$??$?RV<lambda_218ce3db14220d0be481dae8ef3383b6>@@AAV<lambda_628dfdc04ba53c8bfc02c9951375f3f5>@@V<lambda_57dc472bd5c9d5f3b2cbca59b8a843ae>@@@?$__crt_seh_guarded_call@H@@QAEH$$QAV<lambda_218ce3db14220d0be481dae8ef3383b6>@@AAV<lambda_628dfdc04ba53c8bfc02c9951375f3f5>@@$$QAV<lambda_57dc472bd5c9d5f3b2cbca59b8a843ae>@@@Z 10015da8     libucrt:close.obj
 0002:00005dc8       __sehtable$__IsNonwritableInCurrentImage 10015dc8     LIBCMT:pesect.obj
 0002:00005e60       .edata                     10015e60     HlfViewer.exp
 0002:00005e88       rgpv                       10015e88     HlfViewer.exp
 0002:00005ea0       rgszName                   10015ea0     HlfViewer.exp
 0002:00005eb8       rgwOrd                     10015eb8     HlfViewer.exp
 0002:00005ec4       szName                     10015ec4     HlfViewer.exp
 0002:00005ed2       $N00001                    10015ed2     HlfViewer.exp
 0002:00005edd       $N00002                    10015edd     HlfViewer.exp
 0002:00005eec       $N00003                    10015eec     HlfViewer.exp
 0002:00005efb       $N00004                    10015efb     HlfViewer.exp
 0002:00005f01       $N00005                    10015f01     HlfViewer.exp
 0002:00005f15       $N00006                    10015f15     HlfViewer.exp
 0002:0000625c       .idata$6                   1001625c     kernel32:KERNEL32.dll
 0002:0000627c       .idata$6                   1001627c     rpcrt4:RPCRT4.dll
 0003:00000010       ?__vcrt_flsindex@@3KA      10017010     libvcruntime:per_thread_data.obj
 0003:00000040       ?__acrt_flsindex@@3KA      10017040     libucrt:per_thread_data.obj
 0003:00000044       ?errno_no_memory@@3HA      10017044     libucrt:errno.obj
 0003:00000048       ?doserrno_no_memory@@3KA   10017048     libucrt:errno.obj
 0003:00000270       __mbctypes                 10017270     libucrt:mbctype.obj
 0003:00000378       __mbcasemaps               10017378     libucrt:mbctype.obj
 0003:00000478       ?__rgctypeflag@@3PADA      10017478     libucrt:mbctype.obj
 0003:00000480       ?__rgcode_page_info@@3PAUcode_page_info@@A 10017480     libucrt:mbctype.obj
 0003:00000840       ?__dcrt_lowio_console_output_handle@@3PAXA 10017840     libucrt:initcon.obj
 0003:000009d0       _GS_ExceptionRecord        100179d0     LIBCMT:gs_report.obj
 0003:00000a20       _GS_ContextRecord          10017a20     LIBCMT:gs_report.obj
 0003:00000cf4       ?is_initialized_as_dll@@3_NA 10017cf4     LIBCMT:utility.obj
 0003:00000cf5       ?module_local_atexit_table_initialized@@3_NA 10017cf5     LIBCMT:utility.obj
 0003:00000cf8       ?module_local_atexit_table@@3U_onexit_table_t@@A 10017cf8     LIBCMT:utility.obj
 0003:00000d04       ?module_local_at_quick_exit_table@@3U_onexit_table_t@@A 10017d04     LIBCMT:utility.obj
 0003:00000d10       ?__proc_attached@@3HA      10017d10     LIBCMT:dll_dllmain.obj
 0003:00000d44       ?__vcrt_startup_thread_ptd@@3U__vcrt_ptd@@A 10017d44     libvcruntime:per_thread_data.obj
 0003:00000d70       ___vcrt_lock_table         10017d70     libvcruntime:locks.obj
 0003:00000d88       ___vcrt_locks_initialized  10017d88     libvcruntime:locks.obj
 0003:00000db4       ?heap@@3V_HeapManager@@A   10017db4     libvcruntime:undname.obj
 0003:00000dc8       ?module_handles@@3PAPAUHINSTANCE__@@A 10017dc8     libvcruntime:winapi_downlevel.obj
 0003:00000dd4       ?function_pointers@@3PAPAXA 10017dd4     libvcruntime:winapi_downlevel.obj
 0003:00000de8       ?__acrt_invalid_parameter_handler@@3V?$dual_state_global@P6AXPB_W00II@Z@__crt_state_management@@A 10017de8     libucrt:invalid_parameter.obj
 0003:00000dec       ?__acrt_new_handler@@3V?$dual_state_global@P6AHI@Z@__crt_state_management@@A 10017dec     libucrt:new_handler.obj
 0003:00000df0       ?c_termination_complete@@3JA 10017df0     libucrt:exit.obj
 0003:00000df4       ?thread_local_exit_callback_func@@3P6GXPAXK0@ZA 10017df4     libucrt:exit.obj
 0003:00000e00       ?program_name@?1???$common_configure_argv@D@@YAHW4_crt_argv_mode@@@Z@4PADA 10017e00     libucrt:argv_parsing.obj
 0003:00000f30       ?__acrt_lock_table@@3PAU_RTL_CRITICAL_SECTION@@A 10017f30     libucrt:locks.obj
 0003:00001080       ?__acrt_locks_initialized@@3IA 10018080     libucrt:locks.obj
 0003:00001090       ?fSystemSet@@3HA           10018090     libucrt:mbctype.obj
 0003:00001094       ?initialized@?1??__acrt_initialize_multibyte@@9@4_NA 10018094     libucrt:mbctype.obj
 0003:000010b0       ?module_handles@@3PAPAUHINSTANCE__@@A 100180b0     libucrt:winapi_thunks.obj
 0003:00001100       ?encoded_function_pointers@@3PAPAXA 10018100     libucrt:winapi_thunks.obj
 0003:00001394       ?ctrlc_action@@3V?$dual_state_global@P6AXH@Z@__crt_state_management@@A 10018394     libucrt:signal.obj
 0003:00001398       ?ctrlbreak_action@@3V?$dual_state_global@P6AXH@Z@__crt_state_management@@A 10018398     libucrt:signal.obj
 0003:0000139c       ?abort_action@@3V?$dual_state_global@P6AXH@Z@__crt_state_management@@A 1001839c     libucrt:signal.obj
 0003:000013a0       ?term_action@@3V?$dual_state_global@P6AXH@Z@__crt_state_management@@A 100183a0     libucrt:signal.obj
 0003:000013a4       ?user_matherr@@3V?$dual_state_global@P6AHPAU_exception@@@Z@__crt_state_management@@A 100183a4     libucrt:matherr.obj
 0003:000013bc       ?internal_state@?1??_mbtowc_l@@9@4U_Mbstatet@@A 100183bc     libucrt:mbtowc.obj
 0003:000013c8       ?__acrt_global_new_mode@@3V?$dual_state_global@J@__crt_state_management@@A 100183c8     libucrt:new_mode.obj
 0003:000013d4       ?__acrt_app_type@@3W4_crt_app_type@@A 100183d4     libucrt:report_runtime_error.obj
 0003:000013d8       ?internal_pst@?1??__mbrtoc32_utf8@__crt_mbstring@@YAIPA_UPBDIPAU_Mbstatet@@@Z@4U3@A 100183d8     libucrt:mbrtoc32.obj
 0003:000013e4       __pmatherr_set             100183e4     libucrt:libm_error.obj
 0003:000013e8       ?ptrName@?BB@??OpenW@@9@4@4PA_WA 100183e8     HlfViewer.obj
 0003:000013ec       ?ptrTopic@?BB@??OpenW@@9@4@4PA_WA 100183ec     HlfViewer.obj
 0003:000013f0       ?PluginConfigStrings@?1??GetPluginInfoW@@9@4@4PAPB_WA 100183f0     HlfViewer.obj
 0003:000013f4       ?PluginMenuStrings@?4??GetPluginInfoW@@9@4@4PAPB_WA 100183f4     HlfViewer.obj
 0003:00001400       ?FSF@@3UFarStandardFunctions@@A 10018400     HlfViewer.obj
 0003:000014c8       ?PsInfo@@3UPluginStartupInfo@@A 100184c8     HlfViewer.obj
 0003:00001560       ?Opt@@3UOptions@@A         10018560     HlfViewer.obj
 0003:00001810       ?cmdbuf@?BB@??OpenW@@9@4@4PA_WA 10018810     HlfViewer.obj
 0003:00002010       ?FileName@?BB@??OpenW@@9@4@4PA_WA 10019010     HlfViewer.obj
 0003:00002218       ?Function@?1??RtlFirstEntrySListWrapper@@9@4@4Q6GPAU_SINGLE_LIST_ENTRY@@PAT_SLIST_HEADER@@@ZA 10019218     vc_crt_fix_impl.obj
 0003:0000221c       ?$S17@?1??CompareStringExWrapper@@9@36@4IA 1001921c     vc_crt_fix_impl.obj
 0003:00002220       ?Cookie@?1??XorPointer@@YAPAXPAX@Z@4IB 10019220     vc_crt_fix_impl.obj
 0003:00002224       ?$S1@?1??XorPointer@@YAPAXPAX@Z@4IA 10019224     vc_crt_fix_impl.obj
 0003:00002228       ?Function@?1??CompareStringExWrapper@@9@36@4Q6GHPB_WK0H0HPAU_nlsversioninfo@@PAXJ@ZA 10019228     vc_crt_fix_impl.obj
 0003:0000222c       ?Function@?1??InterlockedPushEntrySListWrapper@@9@8@4Q6GPAU_SINGLE_LIST_ENTRY@@PAT_SLIST_HEADER@@PAU2@@ZA 1001922c     vc_crt_fix_impl.obj
 0003:00002230       ?Function@?1??EncodePointerWrapper@@9@4@4Q6GPAXPAX@ZA 10019230     vc_crt_fix_impl.obj
 0003:00002234       ?Function@?1??DecodePointerWrapper@@9@4@4Q6GPAXPAX@ZA 10019234     vc_crt_fix_impl.obj
 0003:00002238       ?Function@?1??QueryDepthSListWrapper@@9@4@4Q6GGPAT_SLIST_HEADER@@@ZA 10019238     vc_crt_fix_impl.obj
 0003:0000223c       ?$S9@?1??InterlockedPushEntrySListWrapper@@9@8@4IA 1001923c     vc_crt_fix_impl.obj
 0003:00002240       ?$S11@?1??RtlFirstEntrySListWrapper@@9@4@4IA 10019240     vc_crt_fix_impl.obj
 0003:00002244       ?$S12@?1??QueryDepthSListWrapper@@9@4@4IA 10019244     vc_crt_fix_impl.obj
 0003:00002248       ?Deleter@?1??InitializeSListHead@implementation@slist@@YGXPAT_SLIST_HEADER@@@Z@4Vservice_deleter@23@A 10019248     vc_crt_fix_impl.obj
 0003:00002268       ?$S15@?1??SetThreadStackGuaranteeWrapper@@9@4@4IA 10019268     vc_crt_fix_impl.obj
 0003:0000226c       ?Function@?1??SetThreadStackGuaranteeWrapper@@9@4@4Q6GHPAK@ZA 1001926c     vc_crt_fix_impl.obj
 0003:00002270       ?Function@?1??LCMapStringExWrapper@@9@36@4Q6GHPB_WK0HPA_WHPAU_nlsversioninfo@@PAXJ@ZA 10019270     vc_crt_fix_impl.obj
 0003:00002274       ?$S3@?1??DecodePointerWrapper@@9@4@4IA 10019274     vc_crt_fix_impl.obj
 0003:00002278       ?Function@?1??InterlockedPushListSListExWrapper@@9@16@4Q6GPAU_SINGLE_LIST_ENTRY@@PAT_SLIST_HEADER@@PAU2@1K@ZA 10019278     vc_crt_fix_impl.obj
 0003:0000227c       ?Function@?1??GetModuleHandleExWWrapper@@9@12@4Q6GHKPB_WPAPAUHINSTANCE__@@@ZA 1001927c     vc_crt_fix_impl.obj
 0003:00002280       ?$S2@?1??EncodePointerWrapper@@9@4@4IA 10019280     vc_crt_fix_impl.obj
 0003:00002284       ?Function@?1??GetLogicalProcessorInformationWrapper@@9@8@4Q6GHPAU_SYSTEM_LOGICAL_PROCESSOR_INFORMATION@@PAK@ZA 10019284     vc_crt_fix_impl.obj
 0003:00002288       ?$S18@?1??LCMapStringExWrapper@@9@36@4IA 10019288     vc_crt_fix_impl.obj
 0003:0000228c       ?$S6@?1??InitializeSListHeadWrapper@@9@4@4IA 1001928c     vc_crt_fix_impl.obj
 0003:00002290       ?Function@?1??InitializeCriticalSectionExWrapper@@9@12@4Q6GHPAU_RTL_CRITICAL_SECTION@@KK@ZA 10019290     vc_crt_fix_impl.obj
 0003:00002294       ?Function@?1??InterlockedFlushSListWrapper@@9@4@4Q6GPAU_SINGLE_LIST_ENTRY@@PAT_SLIST_HEADER@@@ZA 10019294     vc_crt_fix_impl.obj
 0003:00002298       ?$S14@?1??GetLogicalProcessorInformationWrapper@@9@8@4IA 10019298     vc_crt_fix_impl.obj
 0003:0000229c       ?$S13@?1??GetNumaHighestNodeNumberWrapper@@9@4@4IA 1001929c     vc_crt_fix_impl.obj
 0003:000022a0       ?Function@?1??InterlockedPopEntrySListWrapper@@9@4@4Q6GPAU_SINGLE_LIST_ENTRY@@PAT_SLIST_HEADER@@@ZA 100192a0     vc_crt_fix_impl.obj
 0003:000022a4       ?Function@?1??InitializeSListHeadWrapper@@9@4@4Q6GXPAT_SLIST_HEADER@@@ZA 100192a4     vc_crt_fix_impl.obj
 0003:000022a8       ?$S8@?1??InterlockedPopEntrySListWrapper@@9@4@4IA 100192a8     vc_crt_fix_impl.obj
 0003:000022ac       ?$S5@?1??InitializeSListHead@implementation@slist@@YGXPAT_SLIST_HEADER@@@Z@4IA 100192ac     vc_crt_fix_impl.obj
 0003:000022b0       ?$S7@?1??InterlockedFlushSListWrapper@@9@4@4IA 100192b0     vc_crt_fix_impl.obj
 0003:000022b4       ?$S10@?1??InterlockedPushListSListExWrapper@@9@16@4IA 100192b4     vc_crt_fix_impl.obj
 0003:000022b8       ?$S16@?1??InitializeCriticalSectionExWrapper@@9@12@4IA 100192b8     vc_crt_fix_impl.obj
 0003:000022bc       ?$S4@?1??GetModuleHandleExWWrapper@@9@12@4IA 100192bc     vc_crt_fix_impl.obj
 0003:000022c0       ?Ptr@?1???R<lambda_1>@?1??XorPointer@@YAPAXPAX@Z@QBE@XZ@4PAXA 100192c0     vc_crt_fix_impl.obj
 0003:000022c4       ?Function@?1??GetNumaHighestNodeNumberWrapper@@9@4@4Q6GHPAK@ZA 100192c4     vc_crt_fix_impl.obj
 0004:00000060       $R000000                   1001a060     HlfViewer.res
